******************************************************************************
               TMS320C6x Linker PC v7.4.0                      
******************************************************************************
>> Linked Mon Mar 04 15:36:43 2013

OUTPUT FILE NAME:   <SRIOSingleSRIO.out>
ENTRY POINT SYMBOL: "_c_int00"  address: 0082c600


MEMORY CONFIGURATION

         name            origin    length      used     unused   attr    fill
----------------------  --------  ---------  --------  --------  ----  --------
  L2SRAM                00800000   00080000  00072444  0000dbbc  RW X
  MSMCSRAM              0c000000   00400000  00202784  001fd87c  RW X
  DDR3                  80000000   20000000  00012f80  1ffed080  RWIX


SEGMENT ALLOCATION MAP

run origin  load origin   length   init length attrs members
----------  ----------- ---------- ----------- ----- -------
00800000    00800000    000334c0   000334c0    r-x
  00800000    00800000    000334c0   000334c0    r-x .text
008334c0    008334c0    00030000   00000000    rw-
  008334c0    008334c0    00030000   00000000    rw- systemHeap
008634c0    008634c0    00000040   00000040    r--
  008634c0    008634c0    00000040   00000040    r-- .const.1
00863500    00863500    00005be8   00000000    rw-
  00863500    00863500    00005be8   00000000    rw- .far
008690e8    008690e8    00000008   00000008    rw-
  008690e8    008690e8    00000008   00000008    rw- .fardata.1
008690f0    008690f0    0000510a   0000510a    r--
  008690f0    008690f0    0000510a   0000510a    r-- .const.2
0086e200    0086e200    00001e9a   00001e9a    rw-
  0086e200    0086e200    00001e9a   00001e9a    rw- .fardata.2
008700a0    008700a0    00001178   00000000    rw-
  008700a0    008700a0    00001000   00000000    rw- .stack
  008710a0    008710a0    00000120   00000000    rw- .cio
  008711c0    008711c0    00000058   00000000    rw- .bss
00871218    00871218    00000029   00000029    rw-
  00871218    00871218    00000029   00000029    rw- .neardata
00871244    00871244    00000040   00000040    r--
  00871244    00871244    00000040   00000040    r-- .rodata
00871284    00871284    00000080   00000080    r--
  00871284    00871284    00000080   00000080    r-- .switch
00871400    00871400    0000114c   0000114c    r-x
  00871400    00871400    00000200   00000200    r-x .vecs
  00871600    00871600    00000f4c   00000f4c    r-- .cinit
0c000000    0c000000    00002400   00000000    rw-
  0c000000    0c000000    00002400   00000000    rw- .qmss
0c002400    0c002400    00000184   00000184    rw-
  0c002400    0c002400    00000184   00000184    rw- .srioSharedMem
0c002600    0c002600    00000200   00000000    rw-
  0c002600    0c002600    00000200   00000000    rw- .cppi
80000000    80000000    00012f80   00000000    rw-
  80000000    80000000    00011000   00000000    rw- .fftInput
  80011000    80011000    00001f80   00000000    rw- .twiddleFactor


SECTION ALLOCATION MAP

 output                                  attributes/
section   page    origin      length       input sections
--------  ----  ----------  ----------   ----------------
.init_array 
*          0    00800000    00000000     UNINITIALIZED

.init_array 
*          0    00800000    00000000     UNINITIALIZED

xdc.meta   0    00800000    00000100     COPY SECTION
                  00800000    00000100     SRIOMulticore_fft_1_pe66.oe66 (xdc.meta)

.text      0    00800000    000334c0     
                  00800000    000045a0     srio_drv.obj (.text)
                  008045a0    00001b60     device_srio_loopback.obj (.text)
                  00806100    000011c0     ipc.lib : Ipc.obj (.text:ti_sdo_ipc_GateMP_Instance_init__F)
                  008072c0    00000bc0     initialization.obj (.text)
                  00807e80    00000a60     ipc.lib : Ipc.obj (.text:ti_sdo_ipc_heaps_HeapMemMP_alloc__E)
                  008088e0    000009e0             : Ipc.obj (.text:ti_sdo_ipc_heaps_HeapMemMP_free__E)
                  008092c0    000009a0             : Ipc.obj (.text:Ipc_attach)
                  00809c60    000009a0     ti.targets.rts6000.ae66 : System.oe66 (.text:xdc_runtime_System_doPrint__I)
                  0080a600    00000920     ipc.lib : Ipc.obj (.text:ti_sdo_ipc_transports_TransportShm_Instance_init__F)
                  0080af20    000008a0             : Ipc.obj (.text:ti_sdo_ipc_ListMP_Instance_init__F)
                  0080b7c0    00000860             : Ipc.obj (.text:ti_sdo_ipc_GateMP_Instance_finalize__F)
                  0080c020    00000840             : Ipc.obj (.text:MessageQ_put)
                  0080c860    000007e0     ti.drv.qmss.ae66 : qmss_drv.oe66 (.text:Qmss_insertMemoryRegion)
                  0080d040    00000780     ipc.lib : Ipc.obj (.text:ti_sdo_ipc_heaps_HeapMemMP_Instance_init__F)
                  0080d7c0    00000780     sysbios.lib : BIOS.obj (.text:ti_sysbios_family_c64p_Exception_handler__I)
                  0080df40    00000740     multicoreLoopback_osal.obj (.text)
                  0080e680    00000720     device_srio_loopback.obj (.text:SrioDevice_init)
                  0080eda0    000006c0     ipc.lib : Ipc.obj (.text:ti_sdo_ipc_nsremote_NameServerRemoteNotify_Instance_init__F)
                  0080f460    000006a0             : Ipc.obj (.text:NameServer_add)
                  0080fb00    00000660     ti.drv.cppi.ae66 : cppi_drv.oe66 (.text:Cppi_configureRxFlow)
                  00810160    00000660     sysbios.lib : BIOS.obj (.text:ti_sysbios_heaps_HeapMem_free__E)
                  008107c0    00000620     ipc.lib : Ipc.obj (.text:Notify_sendEvent)
                  00810de0    00000620     sysbios.lib : BIOS.obj (.text:ti_sysbios_heaps_HeapMem_alloc__E)
                  00811400    000005e0     ipc.lib : Ipc.obj (.text:Notify_registerEventSingle)
                  008119e0    000005c0             : Ipc.obj (.text:ListMP_getHead)
                  00811fa0    000005c0             : Ipc.obj (.text:Notify_unregisterEventSingle)
                  00812560    000005c0     rts6600_elf.lib : divd.obj (.text:__c6xabi_divd)
                  00812b20    000005c0     dsplib.ae66 : DSP_fft16x16.obj (.text:optimized)
                  008130e0    000005c0     ipc.lib : Ipc.obj (.text:ti_sdo_ipc_SharedRegion_start__F)
                  008136a0    000005c0     sysbios.lib : BIOS.obj (.text:ti_sysbios_timers_timer64_Timer_Module_startup__F)
                  00813c60    00000580     ipc.lib : Ipc.obj (.text:ti_sdo_ipc_nsremote_NameServerRemoteNotify_get__F)
                  008141e0    00000580             : Ipc.obj (.text:ti_sdo_ipc_transports_TransportShm_put__E)
                  00814760    00000540             : Ipc.obj (.text:ti_sdo_ipc_Ipc_procSyncStart__I)
                  00814ca0    00000500     sysbios.lib : BIOS.obj (.text:ti_sysbios_knl_Task_Instance_finalize__F)
                  008151a0    000004e0     ipc.lib : Ipc.obj (.text:ti_sdo_ipc_notifyDrivers_NotifyDriverShm_Instance_init__F)
                  00815680    000004c0     ti.drv.cppi.ae66 : cppi_drv.oe66 (.text:Cppi_txChannelOpen)
                  00815b40    000004a0     ipc.lib : Ipc.obj (.text:ti_sdo_ipc_gates_GatePeterson_Instance_init__F)
                  00815fe0    00000460     masterTask.obj (.text)
                  00816440    00000460     ipc.lib : Ipc.obj (.text:ti_sdo_ipc_GateMP_setRegion0Reserved__F)
                  008168a0    00000460             : Ipc.obj (.text:ti_sdo_ipc_Ipc_procSyncFinish__I)
                  00816d00    00000440     ti.drv.cppi.ae66 : cppi_drv.oe66 (.text:Cppi_rxChannelOpen)
                  00817140    00000440     ipc.lib : Ipc.obj (.text:ListMP_putTail)
                  00817580    00000440             : Ipc.obj (.text:ti_sdo_ipc_heaps_HeapMemMP_getStats__E)
                  008179c0    00000440             : Ipc.obj (.text:ti_sdo_ipc_heaps_HeapMemMP_postInit__I)
                  00817e00    00000400             : Ipc.obj (.text:ti_sdo_ipc_Notify_Instance_init__F)
                  00818200    00000400     sysbios.lib : BIOS.obj (.text:ti_sysbios_knl_Semaphore_pend__E)
                  00818600    000003e0     bioMain.obj (.text)
                  008189e0    000003e0     slaveTask.obj (.text)
                  00818dc0    000003c0     ti.drv.cppi.ae66 : cppi_desc.oe66 (.text:Cppi_initDescriptor)
                  00819180    000003c0     ipc.lib : Ipc.obj (.text:ti_sdo_ipc_SharedRegion_reserveMemory__F)
                  00819540    000003c0     sysbios.lib : BIOS.obj (.text:ti_sysbios_knl_Task_Instance_init__F)
                  00819900    000003c0                 : BIOS.obj (.text:ti_sysbios_knl_Task_setPri__E)
                  00819cc0    000003a0     bioUtilityAndGlobals.obj (.text)
                  0081a060    00000380     ipc.lib : Ipc.obj (.text:HeapMemMP_sharedMemReq)
                  0081a3e0    00000360     SRIOMulticore_fft_1_pe66.oe66 (.text:xdc_runtime_System_printfExtend__I)
                  0081a740    00000340     ipc.lib : Ipc.obj (.text:GateMP_sharedMemReq)
                  0081aa80    00000340     ti.drv.qmss.ae66 : qmss_drv.oe66 (.text:Qmss_init)
                  0081adc0    00000340     ipc.lib : Ipc.obj (.text:ti_sdo_ipc_nsremote_NameServerRemoteNotify_swiFxn__I)
                  0081b100    00000300             : Ipc.obj (.text:GateMP_openByAddr)
                  0081b400    00000300             : Ipc.obj (.text:ti_sdo_ipc_transports_TransportShm_openByAddr__F)
                  0081b700    00000300     sysbios.lib : BIOS.obj (.text:ti_sysbios_family_c64p_Hwi_dispatchC__I)
                  0081ba00    000002e0     ipc.lib : Ipc.obj (.text:SharedRegion_getEntry)
                  0081bce0    000002e0             : Ipc.obj (.text:SharedRegion_getPtr)
                  0081bfc0    000002e0     gen_twiddle_fft16x16.obj (.text)
                  0081c2a0    000002e0     requestProcessingData.obj (.text)
                  0081c580    000002e0     sysbios.lib : BIOS.obj (.text:ti_sysbios_gates_GateMutexPri_enter__E)
                  0081c860    000002e0                 : BIOS.obj (.text:ti_sysbios_knl_Task_Module_startup__F)
                  0081cb40    000002c0     rts6600_elf.lib : cos.obj (.text:cos)
                  0081ce00    000002c0     fftRoutines.obj (.text)
                  0081d0c0    000002c0     ipc.lib : Ipc.obj (.text:ti_sdo_ipc_notifyDrivers_NotifyDriverShm_isr__I)
                  0081d380    000002a0             : Ipc.obj (.text:Ipc_start)
                  0081d620    000002a0             : Ipc.obj (.text:NameServer_getLocal)
                  0081d8c0    000002a0     sysbios.lib : BIOS.obj (.text:ti_sysbios_knl_Clock_workFunc__E)
                  0081db60    00000280     ipc.lib : Ipc.obj (.text:SharedRegion_getSRPtr)
                  0081dde0    00000280     rts6600_elf.lib : divf.obj (.text:__c6xabi_divf)
                  0081e060    00000280     sysbios.lib : BIOS.obj (.text:deviceConfig$44)
                  0081e2e0    00000280     rts6600_elf.lib : sin.obj (.text:sin)
                  0081e560    00000280     ipc.lib : Ipc.obj (.text:ti_sdo_ipc_notifyDrivers_NotifyDriverShm_sharedMemReq__F)
                  0081e7e0    00000280     sysbios.lib : BIOS.obj (.text:ti_sysbios_knl_Clock_Instance_init__F)
                  0081ea60    00000280                 : BIOS.obj (.text:ti_sysbios_knl_Task_exit__E)
                  0081ece0    00000280     ti.targets.rts6000.ae66 : Core-mem.oe66 (.text:xdc_runtime_Core_createObject__I)
                  0081ef60    00000280                             : Error.oe66 (.text:xdc_runtime_Error_raiseX__F)
                  0081f1e0    00000260     ipc.lib : Ipc.obj (.text:ListMP_sharedMemReq)
                  0081f440    00000260             : Ipc.obj (.text:ti_sdo_ipc_ListMP_Instance_finalize__F)
                  0081f6a0    00000260             : Ipc.obj (.text:ti_sdo_ipc_heaps_HeapMemMP_Instance_finalize__F)
                  0081f900    00000260             : Ipc.obj (.text:ti_sdo_ipc_notifyDrivers_NotifyDriverShm_disableEvent__E)
                  0081fb60    00000260     ti.targets.rts6000.ae66 : Startup.oe66 (.text:xdc_runtime_Startup_startMods__I)
                  0081fdc0    00000240     ti.drv.cppi.ae66 : cppi_drv.oe66 (.text:Cppi_open)
                  00820000    00000240     rts6600_elf.lib : imath64.obj (.text:__c6xabi_divull)
                  00820240    00000240     sysbios.lib : BIOS.obj (.text:ti_sysbios_family_c64p_Exception_internalHandler__I)
                  00820480    00000240                 : BIOS.obj (.text:ti_sysbios_knl_Semaphore_post__E)
                  008206c0    00000220     rts6600_elf.lib : fputc.obj (.text:fputc)
                  008208e0    00000220     sysbios.lib : BIOS.obj (.text:ti_sysbios_family_c64p_Hwi_reconfig__E)
                  00820b00    00000220                 : BIOS.obj (.text:ti_sysbios_knl_Swi_run__I)
                  00820d20    00000220                 : BIOS.obj (.text:ti_sysbios_knl_Task_schedule__I)
                  00820f40    00000220                 : BIOS.obj (.text:ti_sysbios_knl_Task_startup__E)
                  00821160    00000200     ipc.lib : Ipc.obj (.text:GateMP_enter)
                  00821360    00000200             : Ipc.obj (.text:GateMP_leave)
                  00821560    00000200             : Ipc.obj (.text:ListMP_openByAddr)
                  00821760    00000200     ti.drv.qmss.ae66 : qmss_drv.oe66 (.text:Qmss_internalQueueOpen)
                  00821960    00000200                      : qmss_acc.oe66 (.text:Qmss_programAccumulator)
                  00821b60    00000200     sysbios.lib : c64p_Hwi_disp_always.obj (.text:_ti_sysbios_family_c64p_Hwi_dispatchAlways)
                  00821d60    00000200                 : BIOS.obj (.text:block$56)
                  00821f60    00000200     ti.drv.cppi.ae66 : cppi_heap.oe66 (.text:cppi_internal_heap_add)
                  00822160    00000200     rts6600_elf.lib : setvbuf.obj (.text:setvbuf)
                  00822360    00000200     ipc.lib : Ipc.obj (.text:ti_sdo_ipc_family_c647x_MultiProcSetup_init__I)
                  00822560    00000200             : Ipc.obj (.text:ti_sdo_ipc_notifyDrivers_NotifyDriverShm_sendEvent__E)
                  00822760    00000200             : Ipc.obj (.text:ti_sdo_ipc_transports_TransportShm_Instance_finalize__F)
                  00822960    000001e0             : Ipc.obj (.text:ti_sdo_ipc_GateMP_attach__F)
                  00822b40    000001e0             : Ipc.obj (.text:ti_sdo_ipc_GateMP_getFreeResource__I)
                  00822d20    000001e0     sysbios.lib : BIOS.obj (.text:ti_sysbios_knl_Task_postInit__I)
                  00822f00    000001e0                 : BIOS.obj (.text:ti_sysbios_timers_timer64_Timer_getFreq__E)
                  008230e0    000001c0     ti.drv.cppi.ae66 : cppi_drv.oe66 (.text:Cppi_initCfg)
                  008232a0    000001c0     ipc.lib : Ipc.obj (.text:HeapMemMP_openByAddr)
                  00823460    000001c0     ti.drv.qmss.ae66 : qmss_drv.oe66 (.text:Qmss_internaldownloadFirmware)
                  00823620    000001c0     rts6600_elf.lib : atan.obj (.text:atan)
                  008237e0    000001c0     ipc.lib : Ipc.obj (.text:ti_sdo_ipc_notifyDrivers_NotifyDriverShm_registerEvent__E)
                  008239a0    000001c0     sysbios.lib : BIOS.obj (.text:ti_sysbios_knl_Swi_Instance_init__F)
                  00823b60    000001c0                 : BIOS.obj (.text:ti_sysbios_knl_Task_checkStacks__E)
                  00823d20    000001c0                 : BIOS.obj (.text:ti_sysbios_timers_timer64_Timer_setPeriodMicroSecs__E)
                  00823ee0    000001a0     rts6600_elf.lib : trgdrv.obj (.text:HOSTrename)
                  00824080    000001a0     ipc.lib : Ipc.obj (.text:SharedRegion_getCacheLineSize)
                  00824220    000001a0             : Ipc.obj (.text:SharedRegion_getHeap)
                  008243c0    000001a0             : Ipc.obj (.text:SharedRegion_isCacheEnabled)
                  00824560    000001a0             : Ipc.obj (.text:ti_sdo_ipc_GateMP_openRegion0Reserved__F)
                  00824700    000001a0             : Ipc.obj (.text:ti_sdo_ipc_notifyDrivers_NotifyDriverShm_enableEvent__E)
                  008248a0    000001a0             : Ipc.obj (.text:ti_sdo_ipc_notifyDrivers_NotifyDriverShm_unregisterEvent__E)
                  00824a40    000001a0             : Ipc.obj (.text:ti_sdo_ipc_nsremote_NameServerRemoteNotify_attach__E)
                  00824be0    000001a0     sysbios.lib : BIOS.obj (.text:ti_sysbios_gates_GateMutex_enter__E)
                  00824d80    000001a0                 : BIOS.obj (.text:ti_sysbios_timers_timer64_Timer_start__E)
                  00824f20    00000180     ipc.lib : Ipc.obj (.text:MultiProc_setLocalId)
                  008250a0    00000180             : Ipc.obj (.text:NameServer_getHandle)
                  00825220    00000180             : Ipc.obj (.text:Notify_intLineRegistered)
                  008253a0    00000180     rts6600_elf.lib : copy_decompress_rle.obj (.text:__TI_decompress_rle_core)
                  00825520    00000180     sysbios.lib : c64p_Exception_asm.obj (.text)
                  008256a0    00000180     ipc.lib : Ipc.obj (.text:ti_sdo_ipc_MessageQ_registerTransport__F)
                  00825820    00000180             : Ipc.obj (.text:ti_sdo_ipc_Notify_Module_startup__F)
                  008259a0    00000180             : Ipc.obj (.text:ti_sdo_ipc_gates_GatePeterson_enter__E)
                  00825b20    00000180             : Ipc.obj (.text:ti_sdo_utils_NameServer_Module_startup__F)
                  00825ca0    00000180     sysbios.lib : BIOS.obj (.text:ti_sysbios_heaps_HeapBuf_Module_startup__F)
                  00825e20    00000180                 : BIOS.obj (.text:ti_sysbios_heaps_HeapMem_Instance_init__F)
                  00825fa0    00000180                 : BIOS.obj (.text:ti_sysbios_knl_Swi_schedule__I)
                  00826120    00000180                 : BIOS.obj (.text:ti_sysbios_knl_Task_unblockI__E)
                  008262a0    00000180     ti.targets.rts6000.ae66 : Text.oe66 (.text:xdc_runtime_Text_putSite__F)
                  00826420    00000160     ti.drv.qmss.ae66 : qmss_drv.oe66 (.text:Qmss_getMemoryRegionCfg)
                  00826580    00000160     ipc.lib : Ipc.obj (.text:ti_sdo_ipc_GateMP_createLocal__F)
                  008266e0    00000160             : Ipc.obj (.text:ti_sdo_ipc_MessageQ_unregisterTransport__F)
                  00826840    00000160             : Ipc.obj (.text:ti_sdo_ipc_gates_GateHWSem_Instance_init__F)
                  008269a0    00000160             : Ipc.obj (.text:ti_sdo_ipc_transports_TransportShm_sharedMemReq__F)
                  00826b00    00000160             : Ipc.obj (.text:ti_sdo_utils_NameServer_isRegistered__E)
                  00826c60    00000160             : Ipc.obj (.text:ti_sdo_utils_NameServer_registerRemoteDriver__E)
                  00826dc0    00000160             : Ipc.obj (.text:ti_sdo_utils_NameServer_unregisterRemoteDriver__E)
                  00826f20    00000140     ti.csl.ae66 : csl_chip.oe66 (.text:CSL_chipReadReg)
                  00827060    00000140     ipc.lib : Ipc.obj (.text:GateMP_close)
                  008271a0    00000140             : Ipc.obj (.text:Notify_attach)
                  008272e0    00000140     boot.ae66 : autoinit.oe66 (.text:_auto_init_elf)
                  00827420    00000140     rts6600_elf.lib : lowlev.obj (.text:getdevice)
                  00827560    00000140     ipc.lib : Ipc.obj (.text:ti_sdo_ipc_Notify_exec__F)
                  008276a0    00000140     sysbios.lib : BIOS.obj (.text:ti_sysbios_family_c64p_Hwi_Module_startup__F)
                  008277e0    00000140                 : BIOS.obj (.text:ti_sysbios_family_c66_Cache_Module_startup__F)
                  00827920    00000140                 : BIOS.obj (.text:ti_sysbios_gates_GateSwi_enter__E)
                  00827a60    00000140                 : BIOS.obj (.text:ti_sysbios_knl_Clock_Instance_finalize__F)
                  00827ba0    00000140                 : BIOS.obj (.text:ti_sysbios_knl_Semaphore_Instance_init__F)
                  00827ce0    00000140                 : BIOS.obj (.text:ti_sysbios_knl_Swi_post__E)
                  00827e20    00000140                 : BIOS.obj (.text:ti_sysbios_knl_Task_blockI__E)
                  00827f60    00000140                 : BIOS.obj (.text:ti_sysbios_knl_Task_yield__E)
                  008280a0    00000120     rts6600_elf.lib : fclose.obj (.text:_closefile)
                  008281c0    00000120                     : fseek.obj (.text:fseek)
                  008282e0    00000120     sysbios.lib : BIOS.obj (.text:rtsUnlock$0)
                  00828400    00000120     ipc.lib : Ipc.obj (.text:ti_sdo_ipc_MessageQ_Module_startup__F)
                  00828520    00000120             : Ipc.obj (.text:ti_sdo_ipc_family_c647x_Interrupt_intRegister__E)
                  00828640    00000120             : Ipc.obj (.text:ti_sdo_ipc_nsremote_NameServerRemoteNotify_Instance_finalize__F)
                  00828760    00000120     ti.targets.rts6000.ae66 : Text.oe66 (.text:xdc_runtime_Text_putLab__F)
                  00828880    00000100     rts6600_elf.lib : trgdrv.obj (.text:HOSTlseek)
                  00828980    00000100                     : _io_perm.obj (.text:_wrt_ok)
                  00828a80    00000100     sysbios.lib : BIOS.obj (.text:initDevice$44)
                  00828b80    00000100     ipc.lib : Ipc.obj (.text:ti_sdo_ipc_GateMP_start__F)
                  00828c80    00000100             : Ipc.obj (.text:ti_sdo_ipc_Notify_Instance_finalize__F)
                  00828d80    00000100             : Ipc.obj (.text:ti_sdo_ipc_SharedRegion_attach__F)
                  00828e80    00000100             : Ipc.obj (.text:ti_sdo_ipc_SharedRegion_clearReservedMemory__F)
                  00828f80    00000100             : Ipc.obj (.text:ti_sdo_ipc_family_c647x_Interrupt_Module_startup__F)
                  00829080    00000100             : Ipc.obj (.text:ti_sdo_ipc_gates_GateHWSem_Module_startup__F)
                  00829180    00000100             : Ipc.obj (.text:ti_sdo_ipc_gates_GateMPSupportNull_enter__E)
                  00829280    00000100             : Ipc.obj (.text:ti_sdo_ipc_gates_GateMPSupportNull_leave__E)
                  00829380    00000100             : Ipc.obj (.text:ti_sdo_ipc_transports_TransportShmSetup_attach__E)
                  00829480    00000100     sysbios.lib : BIOS.obj (.text:ti_sysbios_family_c64p_EventCombiner_dispatch__F)
                  00829580    00000100                 : BIOS.obj (.text:ti_sysbios_gates_GateMutexPri_leave__E)
                  00829680    00000100                 : BIOS.obj (.text:ti_sysbios_knl_Clock_startI__E)
                  00829780    00000100                 : BIOS.obj (.text:ti_sysbios_knl_Swi_restoreHwi__E)
                  00829880    00000100     ti.targets.rts6000.ae66 : Core-mem.oe66 (.text:xdc_runtime_Core_deleteObject__I)
                  00829980    00000100                             : Startup.oe66 (.text:xdc_runtime_Startup_exec__F)
                  00829a80    00000100                             : Text.oe66 (.text:xdc_runtime_Text_putMod__F)
                  00829b80    00000100                             : Text.oe66 (.text:xdc_runtime_Text_visitRope2__I)
                  00829c80    000000e0     rts6600_elf.lib : trgdrv.obj (.text:HOSTopen)
                  00829d60    000000e0                     : lowlev.obj (.text:close)
                  00829e40    000000e0                     : copy_zero_init.obj (.text:decompress:ZI:__TI_zero_init)
                  00829f20    000000e0                     : fflush.obj (.text:fflush)
                  0082a000    000000e0                     : memset.obj (.text:memset)
                  0082a0e0    000000e0     SRIOMulticore_fft_1_pe66.oe66 (.text:ti_sdo_ipc_Notify_Object__create__S)
                  0082a1c0    000000e0     ipc.lib : Ipc.obj (.text:ti_sdo_ipc_family_c647x_NotifySetup_attach__E)
                  0082a2a0    000000e0             : Ipc.obj (.text:ti_sdo_ipc_gates_GateHWSem_enter__E)
                  0082a380    000000e0     sysbios.lib : BIOS.obj (.text:ti_sysbios_family_c64p_Hwi_Instance_finalize__F)
                  0082a460    000000e0                 : BIOS.obj (.text:ti_sysbios_family_c64p_Hwi_Instance_init__F)
                  0082a540    000000e0     SRIOMulticore_fft_1_pe66.oe66 (.text:ti_sysbios_family_c64p_Hwi_Object__create__S)
                  0082a620    000000e0     sysbios.lib : BIOS.obj (.text:ti_sysbios_knl_Clock_start__E)
                  0082a700    000000e0                 : BIOS.obj (.text:ti_sysbios_timers_timer64_Timer_startup__E)
                  0082a7e0    000000e0     ti.targets.rts6000.ae66 : Error.oe66 (.text:xdc_runtime_Error_print__F)
                  0082a8c0    000000e0                             : Memory.oe66 (.text:xdc_runtime_Memory_alloc__F)
                  0082a9a0    000000c0     rts6600_elf.lib : trgdrv.obj (.text:HOSTread)
                  0082aa60    000000c0                     : trgdrv.obj (.text:HOSTunlink)
                  0082ab20    000000c0                     : trgdrv.obj (.text:HOSTwrite)
                  0082abe0    000000c0     ipc.lib : Ipc.obj (.text:HeapMemMP_create)
                  0082aca0    000000c0             : Ipc.obj (.text:ListMP_create)
                  0082ad60    000000c0     ti.drv.qmss.ae66 : qmss_drv.oe66 (.text:Qmss_setEoiVector)
                  0082ae20    000000c0                      : qmss_drv.oe66 (.text:Qmss_setQueueThreshold)
                  0082aee0    000000c0     rts6600_elf.lib : dtor_list.obj (.text:_Z11__TI_atexitPFYvPvES_S_)
                  0082afa0    000000c0                     : dtor_list.obj (.text:__cxa_finalize)
                  0082b060    000000c0                     : divu.obj (.text:__divu)
                  0082b120    000000c0                     : remi.obj (.text:__remi)
                  0082b1e0    000000c0                     : fflush.obj (.text:_doflush)
                  0082b2a0    000000c0                     : exit.obj (.text:exit)
                  0082b360    000000c0     SRIOMulticore_fft_1_pe66.oe66 (.text:ti_sdo_ipc_GateMP_Object__create__S)
                  0082b420    000000c0     ipc.lib : Ipc.obj (.text:ti_sdo_ipc_GateMP_getRegion0ReservedSize__F)
                  0082b4e0    000000c0     SRIOMulticore_fft_1_pe66.oe66 (.text:ti_sdo_ipc_ListMP_Object__create__S)
                  0082b5a0    000000c0     ipc.lib : Ipc.obj (.text:ti_sdo_ipc_family_c647x_Interrupt_intShmStub__I)
                  0082b660    000000c0     SRIOMulticore_fft_1_pe66.oe66 (.text:ti_sdo_ipc_gates_GatePeterson_Object__create__S)
                  0082b720    000000c0     SRIOMulticore_fft_1_pe66.oe66 (.text:ti_sdo_ipc_heaps_HeapMemMP_Object__create__S)
                  0082b7e0    000000c0     SRIOMulticore_fft_1_pe66.oe66 (.text:ti_sdo_ipc_notifyDrivers_NotifyDriverShm_Object__create__S)
                  0082b8a0    000000c0     SRIOMulticore_fft_1_pe66.oe66 (.text:ti_sdo_ipc_nsremote_NameServerRemoteNotify_Object__create__S)
                  0082b960    000000c0     SRIOMulticore_fft_1_pe66.oe66 (.text:ti_sdo_ipc_transports_TransportShm_Object__create__S)
                  0082ba20    000000c0     sysbios.lib : BIOS.obj (.text:ti_sysbios_BIOS_errorRaiseHook__I)
                  0082bae0    000000c0                 : BIOS.obj (.text:ti_sysbios_gates_GateAll_leave__E)
                  0082bba0    000000c0                 : BIOS.obj (.text:ti_sysbios_heaps_HeapMem_getStats__E)
                  0082bc60    000000c0                 : BIOS.obj (.text:ti_sysbios_knl_Clock_logTick__E)
                  0082bd20    000000c0                 : BIOS.obj (.text:ti_sysbios_knl_Swi_Instance_finalize__F)
                  0082bde0    000000c0     SRIOMulticore_fft_1_pe66.oe66 (.text:ti_sysbios_knl_Swi_Object__create__S)
                  0082bea0    000000c0     SRIOMulticore_fft_1_pe66.oe66 (.text:ti_sysbios_knl_Task_Object__create__S)
                  0082bf60    000000c0     sysbios.lib : BIOS.obj (.text:ti_sysbios_timers_timer64_Timer_stop__E)
                  0082c020    000000c0     ti.targets.rts6000.ae66 : System.oe66 (.text:xdc_runtime_System_formatNum__I)
                  0082c0e0    000000c0     SRIOMulticore_fft_1_pe66.oe66 (.text:xdc_runtime_knl_GateThread_Object__create__S)
                  0082c1a0    000000a0     ti.drv.cppi.ae66 : cppi_drv.oe66 (.text:Cppi_channelEnable)
                  0082c240    000000a0     rts6600_elf.lib : trgdrv.obj (.text:HOSTclose)
                  0082c2e0    000000a0                     : trgdrv.obj (.text:HOSTtime)
                  0082c380    000000a0     ti.drv.qmss.ae66 : qmss_drv.oe66 (.text:Qmss_queueClose)
                  0082c420    000000a0                      : qmss_drv.oe66 (.text:Qmss_startCfg)
                  0082c4c0    000000a0     rts6600_elf.lib : round.obj (.text:__c6xabi_nround)
                  0082c560    000000a0                     : remu.obj (.text:__remu)
                  0082c600    000000a0     boot.ae66 : boot.oe66 (.text:_c_int00)
                  0082c6a0    000000a0     rts6600_elf.lib : fopen.obj (.text:_cleanup)
                  0082c740    000000a0     sysbios.lib : c64p_Hwi_asm.obj (.text:_ti_sysbios_family_c64p_Hwi_plug__E)
                  0082c7e0    000000a0     ti.drv.cppi.ae66 : cppi_heap.oe66 (.text:cppi_internal_heap_malloc)
                  0082c880    000000a0                      : cppi_listlib.oe66 (.text:cppi_list_cat)
                  0082c920    000000a0     rts6600_elf.lib : lowlev.obj (.text:finddevice)
                  0082c9c0    000000a0                     : lowlev.obj (.text:lseek)
                  0082ca60    000000a0                     : memcpy64.obj (.text:memcpy)
                  0082cb00    000000a0                     : modf.obj (.text:modf)
                  0082cba0    000000a0     ipc.lib : Ipc.obj (.text:ti_sdo_ipc_family_c647x_Interrupt_intUnregister__E)
                  0082cc40    000000a0             : Ipc.obj (.text:ti_sdo_ipc_gates_GatePeterson_leave__E)
                  0082cce0    000000a0             : Ipc.obj (.text:ti_sdo_ipc_notifyDrivers_NotifyDriverShm_Instance_finalize__F)
                  0082cd80    000000a0     sysbios.lib : BIOS.obj (.text:ti_sysbios_heaps_HeapMem_init__I)
                  0082ce20    000000a0     rts6600_elf.lib : lowlev.obj (.text:write)
                  0082cec0    000000a0     ti.targets.rts6000.ae66 : Assert.oe66 (.text:xdc_runtime_Assert_raise__I)
                  0082cf60    00000080     ti.drv.cppi.ae66 : cppi_drv.oe66 (.text:Cppi_setCpdmaLoopback)
                  0082cfe0    00000080     ti.drv.qmss.ae66 : qmss_drv.oe66 (.text:Qmss_getMemRegQueueHandle)
                  0082d060    00000080                      : qmss_drv.oe66 (.text:Qmss_queueOpen)
                  0082d0e0    00000080     rts6600_elf.lib : llshift.obj (.text:__c6xabi_llshl)
                  0082d160    00000080     sysbios.lib : c62_TaskSupport_asm.obj (.text:_ti_sysbios_family_c62_TaskSupport_swap__E)
                  0082d1e0    00000080     ti.drv.cppi.ae66 : cppi_heap.oe66 (.text:cppi_internal_heap_cache_begin)
                  0082d260    00000080                      : cppi_listlib.oe66 (.text:cppi_list_remove)
                  0082d2e0    00000080     SRIOMulticore_fft_1_pe66.oe66 (.text:malloc)
                  0082d360    00000080     rts6600_elf.lib : rand.obj (.text:rand)
                  0082d3e0    00000080                     : trgmsg.obj (.text:readmsg)
                  0082d460    00000080     SRIOMulticore_fft_1_pe66.oe66 (.text:ti_sdo_ipc_gates_GateHWSem_Object__create__S)
                  0082d4e0    00000080     SRIOMulticore_fft_1_pe66.oe66 (.text:ti_sdo_ipc_gates_GateMPSupportNull_Object__create__S)
                  0082d560    00000080     ipc.lib : Ipc.obj (.text:ti_sdo_ipc_nsremote_NameServerRemoteNotify_detach__E)
                  0082d5e0    00000080             : Ipc.obj (.text:ti_sdo_ipc_transports_TransportShm_swiFxn__I)
                  0082d660    00000080     SRIOMulticore_fft_1_pe66.oe66 (.text:ti_sdo_utils_List_Object__create__S)
                  0082d6e0    00000080     sysbios.lib : BIOS.obj (.text:ti_sysbios_family_c62_TaskSupport_start__E)
                  0082d760    00000080                 : BIOS.obj (.text:ti_sysbios_family_c64p_Exception_Module_startup__F)
                  0082d7e0    00000080                 : BIOS.obj (.text:ti_sysbios_family_c64p_Hwi_eventMap__E)
                  0082d860    00000080                 : BIOS.obj (.text:ti_sysbios_family_c66_Cache_invL1pAll__E)
                  0082d8e0    00000080     SRIOMulticore_fft_1_pe66.oe66 (.text:ti_sysbios_gates_GateAll_Object__create__S)
                  0082d960    00000080     SRIOMulticore_fft_1_pe66.oe66 (.text:ti_sysbios_gates_GateHwi_Object__create__S)
                  0082d9e0    00000080     SRIOMulticore_fft_1_pe66.oe66 (.text:ti_sysbios_gates_GateMutexPri_Object__create__S)
                  0082da60    00000080     SRIOMulticore_fft_1_pe66.oe66 (.text:ti_sysbios_gates_GateMutex_Object__create__S)
                  0082dae0    00000080     SRIOMulticore_fft_1_pe66.oe66 (.text:ti_sysbios_gates_GateSwi_Object__create__S)
                  0082db60    00000080     sysbios.lib : BIOS.obj (.text:ti_sysbios_gates_GateSwi_leave__E)
                  0082dbe0    00000080                 : BIOS.obj (.text:ti_sysbios_hal_Hwi_checkStack:ti_sysbios_hal_Hwi_checkStack)
                  0082dc60    00000080     SRIOMulticore_fft_1_pe66.oe66 (.text:ti_sysbios_heaps_HeapMem_Object__create__S)
                  0082dce0    00000080     sysbios.lib : BIOS.obj (.text:ti_sysbios_knl_Clock_Module_startup__F)
                  0082dd60    00000080     SRIOMulticore_fft_1_pe66.oe66 (.text:ti_sysbios_knl_Clock_Object__create__S)
                  0082dde0    00000080     sysbios.lib : BIOS.obj (.text:ti_sysbios_knl_Clock_getTicks__E)
                  0082de60    00000080                 : BIOS.obj (.text:ti_sysbios_knl_Idle_loop__E)
                  0082dee0    00000080     SRIOMulticore_fft_1_pe66.oe66 (.text:ti_sysbios_knl_Queue_Object__create__S)
                  0082df60    00000080     SRIOMulticore_fft_1_pe66.oe66 (.text:ti_sysbios_knl_Semaphore_Object__create__S)
                  0082dfe0    00000080     sysbios.lib : BIOS.obj (.text:ti_sysbios_knl_Semaphore_pendTimeout__I)
                  0082e060    00000080                 : BIOS.obj (.text:ti_sysbios_knl_Swi_startup__E)
                  0082e0e0    00000080                 : BIOS.obj (.text:ti_sysbios_knl_Task_restore__E)
                  0082e160    00000080                 : BIOS.obj (.text:ti_sysbios_timers_timer64_Timer_getCount__E)
                  0082e1e0    00000080                 : BIOS.obj (.text:ti_sysbios_timers_timer64_Timer_getPeriod__E)
                  0082e260    00000080     SRIOMulticore_fft_1_pe66.oe66 (.text:ti_sysbios_xdcruntime_GateThreadSupport_Object__create__S)
                  0082e2e0    00000080     rts6600_elf.lib : lowlev.obj (.text:unlink)
                  0082e360    00000080     ti.targets.rts6000.ae66 : Core-label.oe66 (.text:xdc_runtime_Core_assignLabel__I)
                  0082e3e0    00000080                             : Core-params.oe66 (.text:xdc_runtime_Core_assignParams__I)
                  0082e460    00000080                             : System.oe66 (.text:xdc_runtime_System_atexit__F)
                  0082e4e0    00000080                             : System.oe66 (.text:xdc_runtime_System_rtsExit__I)
                  0082e560    00000080                             : Text.oe66 (.text:xdc_runtime_Text_printVisFxn__I)
                  0082e5e0    00000080                             : Text.oe66 (.text:xdc_runtime_Text_xprintf__I)
                  0082e660    00000060     ipc.lib : Ipc.obj (.text:GateMP_Params_init)
                  0082e6c0    00000060             : Ipc.obj (.text:HeapMemMP_Params_init)
                  0082e720    00000060     ti.drv.srio.ae66 : listlib.oe66 (.text:Srio_listCat)
                  0082e780    00000060                      : listlib.oe66 (.text:Srio_listRemoveNode)
                  0082e7e0    00000060     rts6600_elf.lib : frcmpyd_div.obj (.text:__c6xabi_frcmpyd_div)
                  0082e840    00000060                     : llshift.obj (.text:__c6xabi_llshru)
                  0082e8a0    00000060                     : imath64.obj (.text:_subcull)
                  0082e900    00000060     ti.drv.cppi.ae66 : cppi_listlib.oe66 (.text:cppi_list_add)
                  0082e960    00000060                      : cppi_listlib.oe66 (.text:cppi_list_cache_invalidate)
                  0082e9c0    00000060     rts6600_elf.lib : rand.obj (.text:srand)
                  0082ea20    00000060     SRIOMulticore_fft_1_pe66.oe66 (.text:ti_sdo_ipc_MessageQ_Object__get__S)
                  0082ea80    00000060     ipc.lib : Ipc.obj (.text:ti_sdo_ipc_family_c647x_NotifySetup_sharedMemReq__E)
                  0082eae0    00000060             : Ipc.obj (.text:ti_sdo_ipc_gates_GateHWSem_leave__E)
                  0082eb40    00000060             : Ipc.obj (.text:ti_sdo_ipc_gates_GatePeterson_Instance_finalize__F)
                  0082eba0    00000060             : Ipc.obj (.text:ti_sdo_ipc_gates_GatePeterson_sharedMemReq__E)
                  0082ec00    00000060             : Ipc.obj (.text:ti_sdo_ipc_notifyDrivers_NotifyDriverShm_setNotifyHandle__E)
                  0082ec60    00000060             : Ipc.obj (.text:ti_sdo_ipc_transports_TransportShmSetup_sharedMemReq__E)
                  0082ecc0    00000060     SRIOMulticore_fft_1_pe66.oe66 (.text:ti_sdo_utils_List_Object__get__S)
                  0082ed20    00000060     SRIOMulticore_fft_1_pe66.oe66 (.text:ti_sdo_utils_NameServer_Object__get__S)
                  0082ed80    00000060     SRIOMulticore_fft_1_pe66.oe66 (.text:ti_sysbios_BIOS_exitFunc__I)
                  0082ede0    00000060     sysbios.lib : BIOS.obj (.text:ti_sysbios_BIOS_registerRTSLock__I)
                  0082ee40    00000060                 : BIOS.obj (.text:ti_sysbios_family_c64p_EventCombiner_Module_startup__F)
                  0082eea0    00000060                 : BIOS.obj (.text:ti_sysbios_family_c64p_EventCombiner_dispatchPlug__F)
                  0082ef00    00000060                 : BIOS.obj (.text:ti_sysbios_family_c64p_EventCombiner_unused__F)
                  0082ef60    00000060                 : BIOS.obj (.text:ti_sysbios_gates_GateAll_enter__E)
                  0082efc0    00000060                 : BIOS.obj (.text:ti_sysbios_gates_GateMutex_Instance_init__F)
                  0082f020    00000060                 : BIOS.obj (.text:ti_sysbios_hal_Hwi_initStack:ti_sysbios_hal_Hwi_initStack)
                  0082f080    00000060     SRIOMulticore_fft_1_pe66.oe66 (.text:ti_sysbios_heaps_HeapBuf_Object__get__S)
                  0082f0e0    00000060     SRIOMulticore_fft_1_pe66.oe66 (.text:ti_sysbios_heaps_HeapMem_Object__get__S)
                  0082f140    00000060     SRIOMulticore_fft_1_pe66.oe66 (.text:ti_sysbios_knl_Clock_doTick__I)
                  0082f1a0    00000060     SRIOMulticore_fft_1_pe66.oe66 (.text:ti_sysbios_knl_Queue_Object__get__S)
                  0082f200    00000060     sysbios.lib : BIOS.obj (.text:ti_sysbios_knl_Swi_Module_startup__F)
                  0082f260    00000060     SRIOMulticore_fft_1_pe66.oe66 (.text:ti_sysbios_knl_Swi_Object__get__S)
                  0082f2c0    00000060     SRIOMulticore_fft_1_pe66.oe66 (.text:ti_sysbios_knl_Task_Object__get__S)
                  0082f320    00000060     sysbios.lib : BIOS.obj (.text:ti_sysbios_knl_Task_allBlockedFunction__I)
                  0082f380    00000060                 : BIOS.obj (.text:ti_sysbios_knl_Task_enter__I)
                  0082f3e0    00000060     rts6600_elf.lib : trgmsg.obj (.text:writemsg)
                  0082f440    00000060     SRIOMulticore_fft_1_pe66.oe66 (.text:xdc_runtime_GateNull_Object__create__S)
                  0082f4a0    00000060     ti.targets.rts6000.ae66 : Memory.oe66 (.text:xdc_runtime_Memory_calloc__F)
                  0082f500    00000060                             : Memory.oe66 (.text:xdc_runtime_Memory_valloc__F)
                  0082f560    00000060                             : SysStd.oe66 (.text:xdc_runtime_SysStd_abort__F)
                  0082f5c0    00000060                             : System.oe66 (.text:xdc_runtime_System_avprintf__F)
                  0082f620    00000060                             : System.oe66 (.text:xdc_runtime_System_vprintf__F)
                  0082f680    00000060                             : Text.oe66 (.text:xdc_runtime_Text_cordText__F)
                  0082f6e0    00000040     ti.drv.qmss.ae66 : qmss_drv.oe66 (.text:Qmss_ackInterrupt)
                  0082f720    00000040                      : qmss_drv.oe66 (.text:Qmss_getMemRegDescSize)
                  0082f760    00000040     ti.drv.srio.ae66 : listlib.oe66 (.text:Srio_listAdd)
                  0082f7a0    00000040                      : listlib.oe66 (.text:Srio_listRemove)
                  0082f7e0    00000040     rts6600_elf.lib : strasg.obj (.text:__strasgi_64plus)
                  0082f820    00000040                     : args_main.obj (.text:_args_main)
                  0082f860    00000040     sysbios.lib : c62_TaskSupport_asm.obj (.text:_ti_sysbios_family_c62_TaskSupport_buildTaskStack)
                  0082f8a0    00000040                 : c64p_Hwi_asm_switch.obj (.text:_ti_sysbios_family_xxx_Hwi_switchToIsrStack)
                  0082f8e0    00000040     rts6600_elf.lib : floor.obj (.text:floor)
                  0082f920    00000040     SRIOMulticore_fft_1_pe66.oe66 (.text:free)
                  0082f960    00000040     sysbios.lib : BIOS.obj (.text:rtsLock$0)
                  0082f9a0    00000040     SRIOMulticore_fft_1_pe66.oe66 (.text:ti_sdo_ipc_GateMP_Object__delete__S)
                  0082f9e0    00000040     SRIOMulticore_fft_1_pe66.oe66 (.text:ti_sdo_ipc_GateMP_Params__init__S)
                  0082fa20    00000040     SRIOMulticore_fft_1_pe66.oe66 (.text:ti_sdo_ipc_GateMP_RemoteCustom1Proxy_Object__create__S)
                  0082fa60    00000040     SRIOMulticore_fft_1_pe66.oe66 (.text:ti_sdo_ipc_GateMP_RemoteCustom2Proxy_Object__create__S)
                  0082faa0    00000040     SRIOMulticore_fft_1_pe66.oe66 (.text:ti_sdo_ipc_GateMP_RemoteSystemProxy_Object__create__S)
                  0082fae0    00000040     SRIOMulticore_fft_1_pe66.oe66 (.text:ti_sdo_ipc_ListMP_Object__delete__S)
                  0082fb20    00000040     SRIOMulticore_fft_1_pe66.oe66 (.text:ti_sdo_ipc_ListMP_Params__init__S)
                  0082fb60    00000040     SRIOMulticore_fft_1_pe66.oe66 (.text:ti_sdo_ipc_MessageQ_registerTransport__E)
                  0082fba0    00000040     ipc.lib : Ipc.obj (.text:ti_sdo_ipc_family_c647x_Interrupt_intClear__E)
                  0082fbe0    00000040             : Ipc.obj (.text:ti_sdo_ipc_family_c647x_Interrupt_intSend__E)
                  0082fc20    00000040     SRIOMulticore_fft_1_pe66.oe66 (.text:ti_sdo_ipc_gates_GateHWSem_Handle__label__S)
                  0082fc60    00000040     SRIOMulticore_fft_1_pe66.oe66 (.text:ti_sdo_ipc_gates_GateHWSem_Object__delete__S)
                  0082fca0    00000040     SRIOMulticore_fft_1_pe66.oe66 (.text:ti_sdo_ipc_gates_GateHWSem_Params__init__S)
                  0082fce0    00000040     SRIOMulticore_fft_1_pe66.oe66 (.text:ti_sdo_ipc_gates_GateMPSupportNull_Handle__label__S)
                  0082fd20    00000040     SRIOMulticore_fft_1_pe66.oe66 (.text:ti_sdo_ipc_gates_GateMPSupportNull_Object__delete__S)
                  0082fd60    00000040     SRIOMulticore_fft_1_pe66.oe66 (.text:ti_sdo_ipc_gates_GateMPSupportNull_Params__init__S)
                  0082fda0    00000040     SRIOMulticore_fft_1_pe66.oe66 (.text:ti_sdo_ipc_gates_GatePeterson_Handle__label__S)
                  0082fde0    00000040     SRIOMulticore_fft_1_pe66.oe66 (.text:ti_sdo_ipc_gates_GatePeterson_Object__delete__S)
                  0082fe20    00000040     SRIOMulticore_fft_1_pe66.oe66 (.text:ti_sdo_ipc_gates_GatePeterson_Params__init__S)
                  0082fe60    00000040     SRIOMulticore_fft_1_pe66.oe66 (.text:ti_sdo_ipc_heaps_HeapMemMP_Handle__label__S)
                  0082fea0    00000040     SRIOMulticore_fft_1_pe66.oe66 (.text:ti_sdo_ipc_heaps_HeapMemMP_Object__delete__S)
                  0082fee0    00000040     SRIOMulticore_fft_1_pe66.oe66 (.text:ti_sdo_ipc_heaps_HeapMemMP_Params__init__S)
                  0082ff20    00000040     SRIOMulticore_fft_1_pe66.oe66 (.text:ti_sdo_ipc_notifyDrivers_NotifyDriverShm_Handle__label__S)
                  0082ff60    00000040     SRIOMulticore_fft_1_pe66.oe66 (.text:ti_sdo_ipc_notifyDrivers_NotifyDriverShm_InterruptProxy_intRegister__E)
                  0082ffa0    00000040     SRIOMulticore_fft_1_pe66.oe66 (.text:ti_sdo_ipc_notifyDrivers_NotifyDriverShm_Object__delete__S)
                  0082ffe0    00000040     SRIOMulticore_fft_1_pe66.oe66 (.text:ti_sdo_ipc_notifyDrivers_NotifyDriverShm_Params__init__S)
                  00830020    00000040     ipc.lib : Ipc.obj (.text:ti_sdo_ipc_notifyDrivers_NotifyDriverShm_disable__E)
                  00830060    00000040             : Ipc.obj (.text:ti_sdo_ipc_notifyDrivers_NotifyDriverShm_enable__E)
                  008300a0    00000040     SRIOMulticore_fft_1_pe66.oe66 (.text:ti_sdo_ipc_nsremote_NameServerRemoteNotify_Handle__label__S)
                  008300e0    00000040     SRIOMulticore_fft_1_pe66.oe66 (.text:ti_sdo_ipc_nsremote_NameServerRemoteNotify_Object__delete__S)
                  00830120    00000040     SRIOMulticore_fft_1_pe66.oe66 (.text:ti_sdo_ipc_nsremote_NameServerRemoteNotify_Object__first__S)
                  00830160    00000040     SRIOMulticore_fft_1_pe66.oe66 (.text:ti_sdo_ipc_nsremote_NameServerRemoteNotify_Object__next__S)
                  008301a0    00000040     SRIOMulticore_fft_1_pe66.oe66 (.text:ti_sdo_ipc_nsremote_NameServerRemoteNotify_Params__init__S)
                  008301e0    00000040     SRIOMulticore_fft_1_pe66.oe66 (.text:ti_sdo_ipc_nsremote_NameServerRemoteNotify_get__E)
                  00830220    00000040     ipc.lib : Ipc.obj (.text:ti_sdo_ipc_nsremote_NameServerRemoteNotify_sharedMemReq__E)
                  00830260    00000040     SRIOMulticore_fft_1_pe66.oe66 (.text:ti_sdo_ipc_transports_TransportShm_Handle__label__S)
                  008302a0    00000040     SRIOMulticore_fft_1_pe66.oe66 (.text:ti_sdo_ipc_transports_TransportShm_Object__delete__S)
                  008302e0    00000040     SRIOMulticore_fft_1_pe66.oe66 (.text:ti_sdo_ipc_transports_TransportShm_Params__init__S)
                  00830320    00000040     SRIOMulticore_fft_1_pe66.oe66 (.text:ti_sdo_utils_List_Object__destruct__S)
                  00830360    00000040     SRIOMulticore_fft_1_pe66.oe66 (.text:ti_sdo_utils_NameServer_Module__startupDone__F)
                  008303a0    00000040     SRIOMulticore_fft_1_pe66.oe66 (.text:ti_sdo_utils_NameServer_Object__first__S)
                  008303e0    00000040     SRIOMulticore_fft_1_pe66.oe66 (.text:ti_sdo_utils_NameServer_Object__next__S)
                  00830420    00000040     SRIOMulticore_fft_1_pe66.oe66 (.text:ti_sysbios_BIOS_startFunc__I)
                  00830460    00000040     sysbios.lib : BIOS.obj (.text:ti_sysbios_BIOS_start__E)
                  008304a0    00000040     SRIOMulticore_fft_1_pe66.oe66 (.text:ti_sysbios_family_c64p_EventCombiner_dispatchPlug__E)
                  008304e0    00000040     sysbios.lib : BIOS.obj (.text:ti_sysbios_family_c64p_EventCombiner_enableEvent__F)
                  00830520    00000040     SRIOMulticore_fft_1_pe66.oe66 (.text:ti_sysbios_family_c64p_Hwi_Module__startupDone__F)
                  00830560    00000040     SRIOMulticore_fft_1_pe66.oe66 (.text:ti_sysbios_family_c64p_Hwi_Object__delete__S)
                  008305a0    00000040     SRIOMulticore_fft_1_pe66.oe66 (.text:ti_sysbios_family_c64p_Hwi_Params__init__S)
                  008305e0    00000040     sysbios.lib : BIOS.obj (.text:ti_sysbios_family_c64p_Hwi_disableInterrupt__E)
                  00830620    00000040                 : BIOS.obj (.text:ti_sysbios_family_c64p_Hwi_enableInterrupt__E)
                  00830660    00000040     SRIOMulticore_fft_1_pe66.oe66 (.text:ti_sysbios_gates_GateAll_Handle__label__S)
                  008306a0    00000040     SRIOMulticore_fft_1_pe66.oe66 (.text:ti_sysbios_gates_GateAll_Object__delete__S)
                  008306e0    00000040     SRIOMulticore_fft_1_pe66.oe66 (.text:ti_sysbios_gates_GateHwi_Handle__label__S)
                  00830720    00000040     SRIOMulticore_fft_1_pe66.oe66 (.text:ti_sysbios_gates_GateHwi_Object__delete__S)
                  00830760    00000040     SRIOMulticore_fft_1_pe66.oe66 (.text:ti_sysbios_gates_GateMutexPri_Handle__label__S)
                  008307a0    00000040     sysbios.lib : BIOS.obj (.text:ti_sysbios_gates_GateMutexPri_Instance_finalize__F)
                  008307e0    00000040                 : BIOS.obj (.text:ti_sysbios_gates_GateMutexPri_Instance_init__F)
                  00830820    00000040     SRIOMulticore_fft_1_pe66.oe66 (.text:ti_sysbios_gates_GateMutexPri_Object__delete__S)
                  00830860    00000040     SRIOMulticore_fft_1_pe66.oe66 (.text:ti_sysbios_gates_GateMutexPri_Object__destruct__S)
                  008308a0    00000040     SRIOMulticore_fft_1_pe66.oe66 (.text:ti_sysbios_gates_GateMutex_Handle__label__S)
                  008308e0    00000040     sysbios.lib : BIOS.obj (.text:ti_sysbios_gates_GateMutex_Instance_finalize__F)
                  00830920    00000040     SRIOMulticore_fft_1_pe66.oe66 (.text:ti_sysbios_gates_GateMutex_Object__delete__S)
                  00830960    00000040     sysbios.lib : BIOS.obj (.text:ti_sysbios_gates_GateMutex_leave__E)
                  008309a0    00000040     SRIOMulticore_fft_1_pe66.oe66 (.text:ti_sysbios_gates_GateSwi_Handle__label__S)
                  008309e0    00000040     SRIOMulticore_fft_1_pe66.oe66 (.text:ti_sysbios_gates_GateSwi_Object__delete__S)
                  00830a20    00000040     SRIOMulticore_fft_1_pe66.oe66 (.text:ti_sysbios_hal_Cache_CacheProxy_inv__E)
                  00830a60    00000040     SRIOMulticore_fft_1_pe66.oe66 (.text:ti_sysbios_hal_Cache_CacheProxy_wbInv__E)
                  00830aa0    00000040     SRIOMulticore_fft_1_pe66.oe66 (.text:ti_sysbios_hal_Timer_Module__startupDone__F)
                  00830ae0    00000040     SRIOMulticore_fft_1_pe66.oe66 (.text:ti_sysbios_heaps_HeapMem_Handle__label__S)
                  00830b20    00000040     SRIOMulticore_fft_1_pe66.oe66 (.text:ti_sysbios_heaps_HeapMem_Object__delete__S)
                  00830b60    00000040     SRIOMulticore_fft_1_pe66.oe66 (.text:ti_sysbios_knl_Clock_Object__destruct__S)
                  00830ba0    00000040     SRIOMulticore_fft_1_pe66.oe66 (.text:ti_sysbios_knl_Clock_Params__init__S)
                  00830be0    00000040     SRIOMulticore_fft_1_pe66.oe66 (.text:ti_sysbios_knl_Queue_Object__destruct__S)
                  00830c20    00000040     sysbios.lib : BIOS.obj (.text:ti_sysbios_knl_Semaphore_Instance_finalize__F)
                  00830c60    00000040     SRIOMulticore_fft_1_pe66.oe66 (.text:ti_sysbios_knl_Semaphore_Object__delete__S)
                  00830ca0    00000040     SRIOMulticore_fft_1_pe66.oe66 (.text:ti_sysbios_knl_Semaphore_Object__destruct__S)
                  00830ce0    00000040     SRIOMulticore_fft_1_pe66.oe66 (.text:ti_sysbios_knl_Semaphore_Params__init__S)
                  00830d20    00000040     SRIOMulticore_fft_1_pe66.oe66 (.text:ti_sysbios_knl_Swi_Object__destruct__S)
                  00830d60    00000040     SRIOMulticore_fft_1_pe66.oe66 (.text:ti_sysbios_knl_Swi_Params__init__S)
                  00830da0    00000040     SRIOMulticore_fft_1_pe66.oe66 (.text:ti_sysbios_knl_Task_Object__first__S)
                  00830de0    00000040     SRIOMulticore_fft_1_pe66.oe66 (.text:ti_sysbios_knl_Task_Object__next__S)
                  00830e20    00000040     SRIOMulticore_fft_1_pe66.oe66 (.text:ti_sysbios_knl_Task_Params__init__S)
                  00830e60    00000040     SRIOMulticore_fft_1_pe66.oe66 (.text:ti_sysbios_timers_timer64_Timer_Module__startupDone__F)
                  00830ea0    00000040     sysbios.lib : BIOS.obj (.text:ti_sysbios_xdcruntime_GateThreadSupport_Instance_finalize__F)
                  00830ee0    00000040                 : BIOS.obj (.text:ti_sysbios_xdcruntime_GateThreadSupport_Instance_init__F)
                  00830f20    00000040     SRIOMulticore_fft_1_pe66.oe66 (.text:ti_sysbios_xdcruntime_GateThreadSupport_Object__delete__S)
                  00830f60    00000040     sysbios.lib : BIOS.obj (.text:ti_sysbios_xdcruntime_GateThreadSupport_enter__F)
                  00830fa0    00000040                 : BIOS.obj (.text:ti_sysbios_xdcruntime_GateThreadSupport_leave__F)
                  00830fe0    00000040     rts6600_elf.lib : time.obj (.text:time)
                  00831020    00000040     ti.targets.rts6000.ae66 : Error.oe66 (.text:xdc_runtime_Error_check__F)
                  00831060    00000040                             : Error.oe66 (.text:xdc_runtime_Error_init__F)
                  008310a0    00000040     SRIOMulticore_fft_1_pe66.oe66 (.text:xdc_runtime_Error_raiseX__E)
                  008310e0    00000040     SRIOMulticore_fft_1_pe66.oe66 (.text:xdc_runtime_GateNull_Handle__label__S)
                  00831120    00000040     SRIOMulticore_fft_1_pe66.oe66 (.text:xdc_runtime_GateNull_Object__delete__S)
                  00831160    00000040     ti.targets.rts6000.ae66 : Gate.oe66 (.text:xdc_runtime_Gate_leaveSystem__F)
                  008311a0    00000040     SRIOMulticore_fft_1_pe66.oe66 (.text:xdc_runtime_IHeap_alloc)
                  008311e0    00000040     SRIOMulticore_fft_1_pe66.oe66 (.text:xdc_runtime_IHeap_free)
                  00831220    00000040     ti.targets.rts6000.ae66 : Memory.oe66 (.text:xdc_runtime_Memory_free__F)
                  00831260    00000040     SRIOMulticore_fft_1_pe66.oe66 (.text:xdc_runtime_Memory_valloc__E)
                  008312a0    00000040     ti.targets.rts6000.ae66 : Registry.oe66 (.text:xdc_runtime_Registry_findById__F)
                  008312e0    00000040     SRIOMulticore_fft_1_pe66.oe66 (.text:xdc_runtime_Startup_exec__I)
                  00831320    00000040     ti.targets.rts6000.ae66 : System.oe66 (.text:xdc_runtime_System_abort__F)
                  00831360    00000040     SRIOMulticore_fft_1_pe66.oe66 (.text:xdc_runtime_System_aprintf__E)
                  008313a0    00000040     SRIOMulticore_fft_1_pe66.oe66 (.text:xdc_runtime_System_printf__E)
                  008313e0    00000040     ti.targets.rts6000.ae66 : Text.oe66 (.text:xdc_runtime_Text_ropeText__F)
                  00831420    00000040     SRIOMulticore_fft_1_pe66.oe66 (.text:xdc_runtime_Text_visitRope__I)
                  00831460    00000040     SRIOMulticore_fft_1_pe66.oe66 (.text:xdc_runtime_knl_GateThread_Handle__label__S)
                  008314a0    00000040     ti.targets.rts6000.ae66 : GateThread.oe66 (.text:xdc_runtime_knl_GateThread_Instance_finalize__F)
                  008314e0    00000040                             : GateThread.oe66 (.text:xdc_runtime_knl_GateThread_Instance_init__F)
                  00831520    00000040     SRIOMulticore_fft_1_pe66.oe66 (.text:xdc_runtime_knl_GateThread_Object__delete__S)
                  00831560    00000040     SRIOMulticore_fft_1_pe66.oe66 (.text:xdc_runtime_knl_GateThread_Proxy_Object__create__S)
                  008315a0    00000020     ti.csl.ae66 : csl_srioGetBaseAddress.oe66 (.text:CSL_SRIO_Open)
                  008315c0    00000020     ti.drv.cppi.ae66 : cppi_drv.oe66 (.text:Cppi_getFlowId)
                  008315e0    00000020                      : cppi_drv.oe66 (.text:Cppi_init)
                  00831600    00000020     ti.drv.qmss.ae66 : qmss_drv.oe66 (.text:Qmss_getQueueHandle)
                  00831620    00000020                      : qmss_drv.oe66 (.text:Qmss_getQueueNumber)
                  00831640    00000020                      : qmss_drv.oe66 (.text:Qmss_start)
                  00831660    00000020     ti.drv.srio.ae66 : listlib.oe66 (.text:Srio_listGetHead)
                  00831680    00000020                      : listlib.oe66 (.text:Srio_listGetNext)
                  008316a0    00000020     rts6600_elf.lib : trunc.obj (.text:__c6xabi_trunc)
                  008316c0    00000020                     : dtor_list.obj (.text:__cxa_atexit)
                  008316e0    00000020                     : dtor_list.obj (.text:__cxa_ia64_exit)
                  00831700    00000020     ti.targets.rts6000.ae66 : xdc_noinit.oe66 (.text:__xdc__init)
                  00831720    00000020     rts6600_elf.lib : _lock.obj (.text:_nop)
                  00831740    00000020                     : _lock.obj (.text:_register_lock)
                  00831760    00000020                     : _lock.obj (.text:_register_unlock)
                  00831780    00000020     sysbios.lib : c62_TaskSupport_asm.obj (.text:_ti_sysbios_family_c62_TaskSupport_glue)
                  008317a0    00000020                 : c64p_Hwi_asm_switch.obj (.text:_ti_sysbios_family_xxx_Hwi_switchToTaskStack)
                  008317c0    00000020     rts6600_elf.lib : exit.obj (.text:abort)
                  008317e0    00000020                     : dtor_list.obj (.text:atexit)
                  00831800    00000020     ti.drv.cppi.ae66 : cppi_listlib.oe66 (.text:cppi_list_get_head)
                  00831820    00000020                      : cppi_listlib.oe66 (.text:cppi_list_get_next)
                  00831840    00000020     rts6600_elf.lib : copy_decompress_none.obj (.text:decompress:none:__TI_decompress_none)
                  00831860    00000020                     : copy_decompress_rle.obj (.text:decompress:rle24:__TI_decompress_rle24)
                  00831880    00000020     sysbios.lib : BIOS.obj (.text:nullFunc$0)
                  008318a0    00000020     rts6600_elf.lib : fputc.obj (.text:putc)
                  008318c0    00000020                     : fputc.obj (.text:putchar)
                  008318e0    00000020     SRIOMulticore_fft_1_pe66.oe66 (.text:ti_sdo_ipc_GateMP_RemoteCustom1Proxy_Object__delete__S)
                  00831900    00000020     SRIOMulticore_fft_1_pe66.oe66 (.text:ti_sdo_ipc_GateMP_RemoteCustom1Proxy_Params__init__S)
                  00831920    00000020     SRIOMulticore_fft_1_pe66.oe66 (.text:ti_sdo_ipc_GateMP_RemoteCustom1Proxy_Proxy__abstract__S)
                  00831940    00000020     SRIOMulticore_fft_1_pe66.oe66 (.text:ti_sdo_ipc_GateMP_RemoteCustom1Proxy_Proxy__delegate__S)
                  00831960    00000020     SRIOMulticore_fft_1_pe66.oe66 (.text:ti_sdo_ipc_GateMP_RemoteCustom1Proxy_getReservedMask__E)
                  00831980    00000020     SRIOMulticore_fft_1_pe66.oe66 (.text:ti_sdo_ipc_GateMP_RemoteCustom1Proxy_sharedMemReq__E)
                  008319a0    00000020     SRIOMulticore_fft_1_pe66.oe66 (.text:ti_sdo_ipc_GateMP_RemoteCustom2Proxy_Object__delete__S)
                  008319c0    00000020     SRIOMulticore_fft_1_pe66.oe66 (.text:ti_sdo_ipc_GateMP_RemoteCustom2Proxy_Params__init__S)
                  008319e0    00000020     SRIOMulticore_fft_1_pe66.oe66 (.text:ti_sdo_ipc_GateMP_RemoteCustom2Proxy_Proxy__abstract__S)
                  00831a00    00000020     SRIOMulticore_fft_1_pe66.oe66 (.text:ti_sdo_ipc_GateMP_RemoteCustom2Proxy_Proxy__delegate__S)
                  00831a20    00000020     SRIOMulticore_fft_1_pe66.oe66 (.text:ti_sdo_ipc_GateMP_RemoteCustom2Proxy_getReservedMask__E)
                  00831a40    00000020     SRIOMulticore_fft_1_pe66.oe66 (.text:ti_sdo_ipc_GateMP_RemoteCustom2Proxy_sharedMemReq__E)
                  00831a60    00000020     SRIOMulticore_fft_1_pe66.oe66 (.text:ti_sdo_ipc_GateMP_RemoteSystemProxy_Object__delete__S)
                  00831a80    00000020     SRIOMulticore_fft_1_pe66.oe66 (.text:ti_sdo_ipc_GateMP_RemoteSystemProxy_Params__init__S)
                  00831aa0    00000020     SRIOMulticore_fft_1_pe66.oe66 (.text:ti_sdo_ipc_GateMP_RemoteSystemProxy_Proxy__abstract__S)
                  00831ac0    00000020     SRIOMulticore_fft_1_pe66.oe66 (.text:ti_sdo_ipc_GateMP_RemoteSystemProxy_Proxy__delegate__S)
                  00831ae0    00000020     SRIOMulticore_fft_1_pe66.oe66 (.text:ti_sdo_ipc_GateMP_RemoteSystemProxy_getReservedMask__E)
                  00831b00    00000020     SRIOMulticore_fft_1_pe66.oe66 (.text:ti_sdo_ipc_GateMP_RemoteSystemProxy_sharedMemReq__E)
                  00831b20    00000020     SRIOMulticore_fft_1_pe66.oe66 (.text:ti_sdo_ipc_GateMP_attach__E)
                  00831b40    00000020     SRIOMulticore_fft_1_pe66.oe66 (.text:ti_sdo_ipc_GateMP_getRegion0ReservedSize__E)
                  00831b60    00000020     SRIOMulticore_fft_1_pe66.oe66 (.text:ti_sdo_ipc_GateMP_getSharedAddr__E)
                  00831b80    00000020     ipc.lib : Ipc.obj (.text:ti_sdo_ipc_GateMP_getSharedAddr__F)
                  00831ba0    00000020     SRIOMulticore_fft_1_pe66.oe66 (.text:ti_sdo_ipc_GateMP_start__E)
                  00831bc0    00000020     SRIOMulticore_fft_1_pe66.oe66 (.text:ti_sdo_ipc_MessageQ_Module_startup__E)
                  00831be0    00000020     SRIOMulticore_fft_1_pe66.oe66 (.text:ti_sdo_ipc_MessageQ_SetupTransportProxy_attach__E)
                  00831c00    00000020     SRIOMulticore_fft_1_pe66.oe66 (.text:ti_sdo_ipc_MessageQ_SetupTransportProxy_isRegistered__E)
                  00831c20    00000020     SRIOMulticore_fft_1_pe66.oe66 (.text:ti_sdo_ipc_MessageQ_SetupTransportProxy_sharedMemReq__E)
                  00831c40    00000020     SRIOMulticore_fft_1_pe66.oe66 (.text:ti_sdo_ipc_MessageQ_unregisterTransport__E)
                  00831c60    00000020     SRIOMulticore_fft_1_pe66.oe66 (.text:ti_sdo_ipc_Notify_Module_GateProxy_enter__E)
                  00831c80    00000020     SRIOMulticore_fft_1_pe66.oe66 (.text:ti_sdo_ipc_Notify_Module_GateProxy_leave__E)
                  00831ca0    00000020     SRIOMulticore_fft_1_pe66.oe66 (.text:ti_sdo_ipc_Notify_Module_startup__E)
                  00831cc0    00000020     SRIOMulticore_fft_1_pe66.oe66 (.text:ti_sdo_ipc_Notify_SetupProxy_attach__E)
                  00831ce0    00000020     SRIOMulticore_fft_1_pe66.oe66 (.text:ti_sdo_ipc_Notify_SetupProxy_numIntLines__E)
                  00831d00    00000020     SRIOMulticore_fft_1_pe66.oe66 (.text:ti_sdo_ipc_Notify_SetupProxy_sharedMemReq__E)
                  00831d20    00000020     SRIOMulticore_fft_1_pe66.oe66 (.text:ti_sdo_ipc_Notify_exec__E)
                  00831d40    00000020     SRIOMulticore_fft_1_pe66.oe66 (.text:ti_sdo_ipc_SharedRegion_attach__E)
                  00831d60    00000020     SRIOMulticore_fft_1_pe66.oe66 (.text:ti_sdo_ipc_SharedRegion_clearReservedMemory__E)
                  00831d80    00000020     SRIOMulticore_fft_1_pe66.oe66 (.text:ti_sdo_ipc_SharedRegion_reserveMemory__E)
                  00831da0    00000020     SRIOMulticore_fft_1_pe66.oe66 (.text:ti_sdo_ipc_SharedRegion_start__E)
                  00831dc0    00000020     SRIOMulticore_fft_1_pe66.oe66 (.text:ti_sdo_ipc_family_c647x_Interrupt_Module_startup__E)
                  00831de0    00000020     ipc.lib : Ipc.obj (.text:ti_sdo_ipc_family_c647x_Interrupt_intDisable__E)
                  00831e00    00000020             : Ipc.obj (.text:ti_sdo_ipc_family_c647x_Interrupt_intEnable__E)
                  00831e20    00000020             : Ipc.obj (.text:ti_sdo_ipc_family_c647x_NotifySetup_numIntLines__E)
                  00831e40    00000020     SRIOMulticore_fft_1_pe66.oe66 (.text:ti_sdo_ipc_gates_GateHWSem_Module_startup__E)
                  00831e60    00000020     ipc.lib : Ipc.obj (.text:ti_sdo_ipc_gates_GateHWSem_getReservedMask__E)
                  00831e80    00000020     SRIOMulticore_fft_1_pe66.oe66 (.text:ti_sdo_ipc_gates_GateHWSem_query__E)
                  00831ea0    00000020     ipc.lib : Ipc.obj (.text:ti_sdo_ipc_gates_GateHWSem_query__F)
                  00831ec0    00000020             : Ipc.obj (.text:ti_sdo_ipc_gates_GateHWSem_sharedMemReq__E)
                  00831ee0    00000020             : Ipc.obj (.text:ti_sdo_ipc_gates_GateMPSupportNull_Instance_init__F)
                  00831f00    00000020             : Ipc.obj (.text:ti_sdo_ipc_gates_GateMPSupportNull_getReservedMask__E)
                  00831f20    00000020     SRIOMulticore_fft_1_pe66.oe66 (.text:ti_sdo_ipc_gates_GateMPSupportNull_query__E)
                  00831f40    00000020     ipc.lib : Ipc.obj (.text:ti_sdo_ipc_gates_GateMPSupportNull_query__F)
                  00831f60    00000020             : Ipc.obj (.text:ti_sdo_ipc_gates_GateMPSupportNull_sharedMemReq__E)
                  00831f80    00000020             : Ipc.obj (.text:ti_sdo_ipc_gates_GatePeterson_getReservedMask__E)
                  00831fa0    00000020     SRIOMulticore_fft_1_pe66.oe66 (.text:ti_sdo_ipc_gates_GatePeterson_query__E)
                  00831fc0    00000020     ipc.lib : Ipc.obj (.text:ti_sdo_ipc_gates_GatePeterson_query__F)
                  00831fe0    00000020     SRIOMulticore_fft_1_pe66.oe66 (.text:ti_sdo_ipc_heaps_HeapMemMP_isBlocking__E)
                  00832000    00000020     ipc.lib : Ipc.obj (.text:ti_sdo_ipc_heaps_HeapMemMP_isBlocking__F)
                  00832020    00000020     SRIOMulticore_fft_1_pe66.oe66 (.text:ti_sdo_ipc_notifyDrivers_NotifyDriverShm_InterruptProxy_intClear__E)
                  00832040    00000020     SRIOMulticore_fft_1_pe66.oe66 (.text:ti_sdo_ipc_notifyDrivers_NotifyDriverShm_InterruptProxy_intDisable__E)
                  00832060    00000020     SRIOMulticore_fft_1_pe66.oe66 (.text:ti_sdo_ipc_notifyDrivers_NotifyDriverShm_InterruptProxy_intEnable__E)
                  00832080    00000020     SRIOMulticore_fft_1_pe66.oe66 (.text:ti_sdo_ipc_notifyDrivers_NotifyDriverShm_InterruptProxy_intSend__E)
                  008320a0    00000020     SRIOMulticore_fft_1_pe66.oe66 (.text:ti_sdo_ipc_notifyDrivers_NotifyDriverShm_InterruptProxy_intUnregister__E)
                  008320c0    00000020     SRIOMulticore_fft_1_pe66.oe66 (.text:ti_sdo_ipc_notifyDrivers_NotifyDriverShm_sharedMemReq__E)
                  008320e0    00000020     ipc.lib : Ipc.obj (.text:ti_sdo_ipc_nsremote_NameServerRemoteNotify_cbFxn__I)
                  00832100    00000020             : Ipc.obj (.text:ti_sdo_ipc_transports_TransportShmSetup_isRegistered__E)
                  00832120    00000020             : Ipc.obj (.text:ti_sdo_ipc_transports_TransportShm_control__E)
                  00832140    00000020             : Ipc.obj (.text:ti_sdo_ipc_transports_TransportShm_getStatus__E)
                  00832160    00000020             : Ipc.obj (.text:ti_sdo_ipc_transports_TransportShm_notifyFxn__I)
                  00832180    00000020     SRIOMulticore_fft_1_pe66.oe66 (.text:ti_sdo_ipc_transports_TransportShm_openByAddr__E)
                  008321a0    00000020     SRIOMulticore_fft_1_pe66.oe66 (.text:ti_sdo_ipc_transports_TransportShm_setErrFxn__E)
                  008321c0    00000020     ipc.lib : Ipc.obj (.text:ti_sdo_ipc_transports_TransportShm_setErrFxn__F)
                  008321e0    00000020     SRIOMulticore_fft_1_pe66.oe66 (.text:ti_sdo_ipc_transports_TransportShm_sharedMemReq__E)
                  00832200    00000020     ipc.lib : Ipc.obj (.text:ti_sdo_utils_List_Instance_init__F)
                  00832220    00000020     SRIOMulticore_fft_1_pe66.oe66 (.text:ti_sdo_utils_MultiProc_getClusterId__E)
                  00832240    00000020     ipc.lib : Ipc.obj (.text:ti_sdo_utils_MultiProc_getClusterId__F)
                  00832260    00000020     SRIOMulticore_fft_1_pe66.oe66 (.text:ti_sdo_utils_NameServer_Module__startupDone__S)
                  00832280    00000020     SRIOMulticore_fft_1_pe66.oe66 (.text:ti_sdo_utils_NameServer_Module_startup__E)
                  008322a0    00000020     SRIOMulticore_fft_1_pe66.oe66 (.text:ti_sdo_utils_NameServer_SetupProxy_attach__E)
                  008322c0    00000020     SRIOMulticore_fft_1_pe66.oe66 (.text:ti_sdo_utils_NameServer_SetupProxy_sharedMemReq__E)
                  008322e0    00000020     SRIOMulticore_fft_1_pe66.oe66 (.text:ti_sysbios_BIOS_RtsGateProxy_enter__E)
                  00832300    00000020     SRIOMulticore_fft_1_pe66.oe66 (.text:ti_sysbios_BIOS_RtsGateProxy_leave__E)
                  00832320    00000020     sysbios.lib : BIOS.obj (.text:ti_sysbios_BIOS_getThreadType__E)
                  00832340    00000020                 : BIOS.obj (.text:ti_sysbios_BIOS_setThreadType__E)
                  00832360    00000020     SRIOMulticore_fft_1_pe66.oe66 (.text:ti_sysbios_family_c62_TaskSupport_Module__startupDone__S)
                  00832380    00000020     sysbios.lib : BIOS.obj (.text:ti_sysbios_family_c62_TaskSupport_checkStack__E)
                  008323a0    00000020                 : BIOS.obj (.text:ti_sysbios_family_c62_TaskSupport_getStackAlignment__E)
                  008323c0    00000020     SRIOMulticore_fft_1_pe66.oe66 (.text:ti_sysbios_family_c64p_EventCombiner_Module_startup__E)
                  008323e0    00000020     SRIOMulticore_fft_1_pe66.oe66 (.text:ti_sysbios_family_c64p_EventCombiner_dispatch__E)
                  00832400    00000020     SRIOMulticore_fft_1_pe66.oe66 (.text:ti_sysbios_family_c64p_EventCombiner_enableEvent__E)
                  00832420    00000020     SRIOMulticore_fft_1_pe66.oe66 (.text:ti_sysbios_family_c64p_EventCombiner_unused__E)
                  00832440    00000020     SRIOMulticore_fft_1_pe66.oe66 (.text:ti_sysbios_family_c64p_Exception_Module_startup__E)
                  00832460    00000020     SRIOMulticore_fft_1_pe66.oe66 (.text:ti_sysbios_family_c64p_Hwi_Module__startupDone__S)
                  00832480    00000020     SRIOMulticore_fft_1_pe66.oe66 (.text:ti_sysbios_family_c64p_Hwi_Module_startup__E)
                  008324a0    00000020     sysbios.lib : BIOS.obj (.text:ti_sysbios_family_c64p_Hwi_clearInterrupt__E)
                  008324c0    00000020                 : BIOS.obj (.text:ti_sysbios_family_c64p_Hwi_getHandle__E)
                  008324e0    00000020                 : BIOS.obj (.text:ti_sysbios_family_c64p_Hwi_startup__E)
                  00832500    00000020                 : BIOS.obj (.text:ti_sysbios_family_c64p_Hwi_switchFromBootStack__E)
                  00832520    00000020                 : BIOS.obj (.text:ti_sysbios_family_c64p_Hwi_unPluggedInterrupt__I)
                  00832540    00000020                 : BIOS.obj (.text:ti_sysbios_family_c64p_tci6488_TimerSupport_enable__E)
                  00832560    00000020     SRIOMulticore_fft_1_pe66.oe66 (.text:ti_sysbios_family_c66_Cache_Module_startup__E)
                  00832580    00000020     sysbios.lib : BIOS.obj (.text:ti_sysbios_family_c66_Cache_inv__E)
                  008325a0    00000020                 : BIOS.obj (.text:ti_sysbios_family_c66_Cache_wbInv__E)
                  008325c0    00000020                 : BIOS.obj (.text:ti_sysbios_gates_GateAll_Instance_init__F)
                  008325e0    00000020     SRIOMulticore_fft_1_pe66.oe66 (.text:ti_sysbios_gates_GateAll_query__E)
                  00832600    00000020     sysbios.lib : BIOS.obj (.text:ti_sysbios_gates_GateAll_query__F)
                  00832620    00000020                 : BIOS.obj (.text:ti_sysbios_gates_GateHwi_Instance_init__F)
                  00832640    00000020                 : BIOS.obj (.text:ti_sysbios_gates_GateHwi_enter__E)
                  00832660    00000020                 : BIOS.obj (.text:ti_sysbios_gates_GateHwi_leave__E)
                  00832680    00000020     SRIOMulticore_fft_1_pe66.oe66 (.text:ti_sysbios_gates_GateHwi_query__E)
                  008326a0    00000020     sysbios.lib : BIOS.obj (.text:ti_sysbios_gates_GateHwi_query__F)
                  008326c0    00000020     SRIOMulticore_fft_1_pe66.oe66 (.text:ti_sysbios_gates_GateMutexPri_query__E)
                  008326e0    00000020     sysbios.lib : BIOS.obj (.text:ti_sysbios_gates_GateMutexPri_query__F)
                  00832700    00000020     SRIOMulticore_fft_1_pe66.oe66 (.text:ti_sysbios_gates_GateMutex_query__E)
                  00832720    00000020     sysbios.lib : BIOS.obj (.text:ti_sysbios_gates_GateMutex_query__F)
                  00832740    00000020                 : BIOS.obj (.text:ti_sysbios_gates_GateSwi_Instance_init__F)
                  00832760    00000020     SRIOMulticore_fft_1_pe66.oe66 (.text:ti_sysbios_gates_GateSwi_query__E)
                  00832780    00000020     sysbios.lib : BIOS.obj (.text:ti_sysbios_gates_GateSwi_query__F)
                  008327a0    00000020     SRIOMulticore_fft_1_pe66.oe66 (.text:ti_sysbios_hal_Hwi_HwiProxy_Module__startupDone__S)
                  008327c0    00000020     SRIOMulticore_fft_1_pe66.oe66 (.text:ti_sysbios_hal_Hwi_HwiProxy_clearInterrupt__E)
                  008327e0    00000020     SRIOMulticore_fft_1_pe66.oe66 (.text:ti_sysbios_hal_Hwi_HwiProxy_disableInterrupt__E)
                  00832800    00000020     SRIOMulticore_fft_1_pe66.oe66 (.text:ti_sysbios_hal_Hwi_HwiProxy_enableInterrupt__E)
                  00832820    00000020     SRIOMulticore_fft_1_pe66.oe66 (.text:ti_sysbios_hal_Hwi_HwiProxy_startup__E)
                  00832840    00000020     SRIOMulticore_fft_1_pe66.oe66 (.text:ti_sysbios_hal_Hwi_HwiProxy_switchFromBootStack__E)
                  00832860    00000020     SRIOMulticore_fft_1_pe66.oe66 (.text:ti_sysbios_hal_Hwi_Module_startup__E)
                  00832880    00000020     sysbios.lib : BIOS.obj (.text:ti_sysbios_hal_Hwi_Module_startup__F)
                  008328a0    00000020     SRIOMulticore_fft_1_pe66.oe66 (.text:ti_sysbios_hal_Timer_Module__startupDone__S)
                  008328c0    00000020     SRIOMulticore_fft_1_pe66.oe66 (.text:ti_sysbios_hal_Timer_Module_startup__E)
                  008328e0    00000020     sysbios.lib : BIOS.obj (.text:ti_sysbios_hal_Timer_Module_startup__F)
                  00832900    00000020     SRIOMulticore_fft_1_pe66.oe66 (.text:ti_sysbios_hal_Timer_TimerProxy_Module__startupDone__S)
                  00832920    00000020     SRIOMulticore_fft_1_pe66.oe66 (.text:ti_sysbios_hal_Timer_TimerProxy_getExpiredCounts__E)
                  00832940    00000020     SRIOMulticore_fft_1_pe66.oe66 (.text:ti_sysbios_hal_Timer_TimerProxy_getPeriod__E)
                  00832960    00000020     SRIOMulticore_fft_1_pe66.oe66 (.text:ti_sysbios_hal_Timer_TimerProxy_setNextTick__E)
                  00832980    00000020     SRIOMulticore_fft_1_pe66.oe66 (.text:ti_sysbios_hal_Timer_TimerProxy_startup__E)
                  008329a0    00000020     SRIOMulticore_fft_1_pe66.oe66 (.text:ti_sysbios_heaps_HeapBuf_Module_startup__E)
                  008329c0    00000020     SRIOMulticore_fft_1_pe66.oe66 (.text:ti_sysbios_heaps_HeapMem_Module_GateProxy_enter__E)
                  008329e0    00000020     SRIOMulticore_fft_1_pe66.oe66 (.text:ti_sysbios_heaps_HeapMem_Module_GateProxy_leave__E)
                  00832a00    00000020     SRIOMulticore_fft_1_pe66.oe66 (.text:ti_sysbios_heaps_HeapMem_Module_GateProxy_query__E)
                  00832a20    00000020     sysbios.lib : BIOS.obj (.text:ti_sysbios_heaps_HeapMem_isBlocking__E)
                  00832a40    00000020     SRIOMulticore_fft_1_pe66.oe66 (.text:ti_sysbios_knl_Clock_Module_State_clockQ)
                  00832a60    00000020     SRIOMulticore_fft_1_pe66.oe66 (.text:ti_sysbios_knl_Clock_Module_startup__E)
                  00832a80    00000020     sysbios.lib : BIOS.obj (.text:ti_sysbios_knl_Queue_Instance_init__F)
                  00832aa0    00000020                 : BIOS.obj (.text:ti_sysbios_knl_Queue_empty__E)
                  00832ac0    00000020     SRIOMulticore_fft_1_pe66.oe66 (.text:ti_sysbios_knl_Swi_Module_startup__E)
                  00832ae0    00000020     sysbios.lib : BIOS.obj (.text:ti_sysbios_knl_Swi_disable__E)
                  00832b00    00000020     SRIOMulticore_fft_1_pe66.oe66 (.text:ti_sysbios_knl_Task_Module_startup__E)
                  00832b20    00000020     SRIOMulticore_fft_1_pe66.oe66 (.text:ti_sysbios_knl_Task_SupportProxy_Module__startupDone__S)
                  00832b40    00000020     SRIOMulticore_fft_1_pe66.oe66 (.text:ti_sysbios_knl_Task_SupportProxy_checkStack__E)
                  00832b60    00000020     SRIOMulticore_fft_1_pe66.oe66 (.text:ti_sysbios_knl_Task_SupportProxy_getStackAlignment__E)
                  00832b80    00000020     SRIOMulticore_fft_1_pe66.oe66 (.text:ti_sysbios_knl_Task_SupportProxy_start__E)
                  00832ba0    00000020     SRIOMulticore_fft_1_pe66.oe66 (.text:ti_sysbios_knl_Task_SupportProxy_swap__E)
                  00832bc0    00000020     sysbios.lib : BIOS.obj (.text:ti_sysbios_knl_Task_disable__E)
                  00832be0    00000020                 : BIOS.obj (.text:ti_sysbios_knl_Task_getPri__E)
                  00832c00    00000020                 : BIOS.obj (.text:ti_sysbios_knl_Task_self__E)
                  00832c20    00000020     SRIOMulticore_fft_1_pe66.oe66 (.text:ti_sysbios_timers_timer64_Timer_Module__startupDone__S)
                  00832c40    00000020     SRIOMulticore_fft_1_pe66.oe66 (.text:ti_sysbios_timers_timer64_Timer_Module_startup__E)
                  00832c60    00000020     SRIOMulticore_fft_1_pe66.oe66 (.text:ti_sysbios_timers_timer64_Timer_TimerSupportProxy_enable__E)
                  00832c80    00000020     sysbios.lib : BIOS.obj (.text:ti_sysbios_timers_timer64_Timer_setNextTick__E)
                  00832ca0    00000020     SRIOMulticore_fft_1_pe66.oe66 (.text:ti_sysbios_xdcruntime_GateThreadSupport_enter__E)
                  00832cc0    00000020     SRIOMulticore_fft_1_pe66.oe66 (.text:ti_sysbios_xdcruntime_GateThreadSupport_leave__E)
                  00832ce0    00000020     SRIOMulticore_fft_1_pe66.oe66 (.text:ti_sysbios_xdcruntime_GateThreadSupport_query__E)
                  00832d00    00000020     SRIOMulticore_fft_1_pe66.oe66 (.text:xdc_iargToPtr)
                  00832d20    00000020     SRIOMulticore_fft_1_pe66.oe66 (.text:xdc_runtime_Error_check__E)
                  00832d40    00000020     SRIOMulticore_fft_1_pe66.oe66 (.text:xdc_runtime_Error_init__E)
                  00832d60    00000020     SRIOMulticore_fft_1_pe66.oe66 (.text:xdc_runtime_Error_print__E)
                  00832d80    00000020     SRIOMulticore_fft_1_pe66.oe66 (.text:xdc_runtime_GateNull_enter__E)
                  00832da0    00000020     ti.targets.rts6000.ae66 : GateNull.oe66 (.text:xdc_runtime_GateNull_enter__F)
                  00832dc0    00000020     SRIOMulticore_fft_1_pe66.oe66 (.text:xdc_runtime_GateNull_leave__E)
                  00832de0    00000020     ti.targets.rts6000.ae66 : GateNull.oe66 (.text:xdc_runtime_GateNull_leave__F)
                  00832e00    00000020     SRIOMulticore_fft_1_pe66.oe66 (.text:xdc_runtime_GateNull_query__E)
                  00832e20    00000020     ti.targets.rts6000.ae66 : GateNull.oe66 (.text:xdc_runtime_GateNull_query__F)
                  00832e40    00000020     SRIOMulticore_fft_1_pe66.oe66 (.text:xdc_runtime_Gate_enterSystem__E)
                  00832e60    00000020     ti.targets.rts6000.ae66 : Gate.oe66 (.text:xdc_runtime_Gate_enterSystem__F)
                  00832e80    00000020     SRIOMulticore_fft_1_pe66.oe66 (.text:xdc_runtime_Gate_leaveSystem__E)
                  00832ea0    00000020     SRIOMulticore_fft_1_pe66.oe66 (.text:xdc_runtime_Memory_HeapProxy_alloc__E)
                  00832ec0    00000020     SRIOMulticore_fft_1_pe66.oe66 (.text:xdc_runtime_Memory_HeapProxy_free__E)
                  00832ee0    00000020     SRIOMulticore_fft_1_pe66.oe66 (.text:xdc_runtime_Memory_alloc__E)
                  00832f00    00000020     SRIOMulticore_fft_1_pe66.oe66 (.text:xdc_runtime_Memory_calloc__E)
                  00832f20    00000020     SRIOMulticore_fft_1_pe66.oe66 (.text:xdc_runtime_Memory_free__E)
                  00832f40    00000020     SRIOMulticore_fft_1_pe66.oe66 (.text:xdc_runtime_Memory_getMaxDefaultTypeAlign__E)
                  00832f60    00000020     ti.targets.rts6000.ae66 : Memory.oe66 (.text:xdc_runtime_Memory_getMaxDefaultTypeAlign__F)
                  00832f80    00000020     SRIOMulticore_fft_1_pe66.oe66 (.text:xdc_runtime_Registry_findById__E)
                  00832fa0    00000020     SRIOMulticore_fft_1_pe66.oe66 (.text:xdc_runtime_Startup_Module__startupDone__S)
                  00832fc0    00000020     SRIOMulticore_fft_1_pe66.oe66 (.text:xdc_runtime_Startup_exec__E)
                  00832fe0    00000020     SRIOMulticore_fft_1_pe66.oe66 (.text:xdc_runtime_Startup_reset__I)
                  00833000    00000020     SRIOMulticore_fft_1_pe66.oe66 (.text:xdc_runtime_Startup_rtsDone__E)
                  00833020    00000020     ti.targets.rts6000.ae66 : Startup.oe66 (.text:xdc_runtime_Startup_rtsDone__F)
                  00833040    00000020     SRIOMulticore_fft_1_pe66.oe66 (.text:xdc_runtime_SysStd_abort__E)
                  00833060    00000020     SRIOMulticore_fft_1_pe66.oe66 (.text:xdc_runtime_SysStd_exit__E)
                  00833080    00000020     ti.targets.rts6000.ae66 : SysStd.oe66 (.text:xdc_runtime_SysStd_exit__F)
                  008330a0    00000020     SRIOMulticore_fft_1_pe66.oe66 (.text:xdc_runtime_SysStd_putch__E)
                  008330c0    00000020     ti.targets.rts6000.ae66 : SysStd.oe66 (.text:xdc_runtime_SysStd_putch__F)
                  008330e0    00000020     SRIOMulticore_fft_1_pe66.oe66 (.text:xdc_runtime_SysStd_ready__E)
                  00833100    00000020     ti.targets.rts6000.ae66 : SysStd.oe66 (.text:xdc_runtime_SysStd_ready__F)
                  00833120    00000020     SRIOMulticore_fft_1_pe66.oe66 (.text:xdc_runtime_System_Module_GateProxy_enter__E)
                  00833140    00000020     SRIOMulticore_fft_1_pe66.oe66 (.text:xdc_runtime_System_Module_GateProxy_leave__E)
                  00833160    00000020     SRIOMulticore_fft_1_pe66.oe66 (.text:xdc_runtime_System_Module_startup__E)
                  00833180    00000020     ti.targets.rts6000.ae66 : System.oe66 (.text:xdc_runtime_System_Module_startup__F)
                  008331a0    00000020     SRIOMulticore_fft_1_pe66.oe66 (.text:xdc_runtime_System_SupportProxy_abort__E)
                  008331c0    00000020     SRIOMulticore_fft_1_pe66.oe66 (.text:xdc_runtime_System_SupportProxy_exit__E)
                  008331e0    00000020     SRIOMulticore_fft_1_pe66.oe66 (.text:xdc_runtime_System_SupportProxy_putch__E)
                  00833200    00000020     SRIOMulticore_fft_1_pe66.oe66 (.text:xdc_runtime_System_SupportProxy_ready__E)
                  00833220    00000020     SRIOMulticore_fft_1_pe66.oe66 (.text:xdc_runtime_System_abort__E)
                  00833240    00000020     SRIOMulticore_fft_1_pe66.oe66 (.text:xdc_runtime_System_atexit__E)
                  00833260    00000020     SRIOMulticore_fft_1_pe66.oe66 (.text:xdc_runtime_System_exit__E)
                  00833280    00000020     ti.targets.rts6000.ae66 : System.oe66 (.text:xdc_runtime_System_exit__F)
                  008332a0    00000020                             : System.oe66 (.text:xdc_runtime_System_lastFxn__I)
                  008332c0    00000020     SRIOMulticore_fft_1_pe66.oe66 (.text:xdc_runtime_System_vsprintf__E)
                  008332e0    00000020     ti.targets.rts6000.ae66 : System.oe66 (.text:xdc_runtime_System_vsprintf__F)
                  00833300    00000020     SRIOMulticore_fft_1_pe66.oe66 (.text:xdc_runtime_Text_cordText__E)
                  00833320    00000020     SRIOMulticore_fft_1_pe66.oe66 (.text:xdc_runtime_Text_putLab__E)
                  00833340    00000020     SRIOMulticore_fft_1_pe66.oe66 (.text:xdc_runtime_Text_putSite__E)
                  00833360    00000020     SRIOMulticore_fft_1_pe66.oe66 (.text:xdc_runtime_Text_ropeText__E)
                  00833380    00000020     SRIOMulticore_fft_1_pe66.oe66 (.text:xdc_runtime_knl_GateThread_Module__startupDone__S)
                  008333a0    00000020     SRIOMulticore_fft_1_pe66.oe66 (.text:xdc_runtime_knl_GateThread_Proxy_Object__delete__S)
                  008333c0    00000020     SRIOMulticore_fft_1_pe66.oe66 (.text:xdc_runtime_knl_GateThread_Proxy_enter__E)
                  008333e0    00000020     SRIOMulticore_fft_1_pe66.oe66 (.text:xdc_runtime_knl_GateThread_Proxy_leave__E)
                  00833400    00000020     SRIOMulticore_fft_1_pe66.oe66 (.text:xdc_runtime_knl_GateThread_Proxy_query__E)
                  00833420    00000020     SRIOMulticore_fft_1_pe66.oe66 (.text:xdc_runtime_knl_GateThread_enter__E)
                  00833440    00000020     ti.targets.rts6000.ae66 : GateThread.oe66 (.text:xdc_runtime_knl_GateThread_enter__F)
                  00833460    00000020     SRIOMulticore_fft_1_pe66.oe66 (.text:xdc_runtime_knl_GateThread_leave__E)
                  00833480    00000020     ti.targets.rts6000.ae66 : GateThread.oe66 (.text:xdc_runtime_knl_GateThread_leave__F)
                  008334a0    00000020     SRIOMulticore_fft_1_pe66.oe66 (.text:xdc_runtime_knl_GateThread_query__E)

systemHeap 
*          0    008334c0    00030000     UNINITIALIZED
                  008334c0    00030000     SRIOMulticore_fft_1_pe66.oe66 (systemHeap)

.const.1   0    008634c0    00000040     
                  008634c0    00000040     ti.targets.rts6000.ae66 : Text.oe66 (.const:.string)

.far       0    00863500    00005be8     UNINITIALIZED
                  00863500    00004000     fftRoutines.obj (.far)
                  00867500    00000da0     initialization.obj (.far)
                  008682a0    00000800     SRIOMulticore_fft_1_pe66.oe66 (.far:taskStackSection)
                  00868aa0    00000248     bioUtilityAndGlobals.obj (.far)
                  00868ce8    00000140     rts6600_elf.lib : defs.obj (.far)
                  00868e28    00000120     ti.drv.qmss.ae66 : qmss_drv.oe66 (.far)
                  00868f48    000000f0     multicoreLoopback_osal.obj (.far)
                  00869038    00000080     masterTask.obj (.far)
                  008690b8    00000024     SRIOMulticore_fft_1_pe66.oe66 (.far)
                  008690dc    00000004     --HOLE--
                  008690e0    00000008     rts6600_elf.lib : trgdrv.obj (.far)

.fardata.1 
*          0    008690e8    00000008     
                  008690e8    00000008     rts6600_elf.lib : _lock.obj (.fardata)

.const.2   0    008690f0    0000510a     
                  008690f0    000025b1     SRIOMulticore_fft_1_pe66.oe66 (.const:xdc_runtime_Text_charTab__A)
                  0086b6a1    00000003     --HOLE-- [fill = 0]
                  0086b6a4    00000004     ti.targets.rts6000.ae66 : Assert.oe66 (.const:.string)
                  0086b6a8    00000630     initialization.obj (.const:acc48_le)
                  0086bcd8    000004d8     srio_drv.obj (.const:.string)
                  0086c1b0    0000042c     sysbios.lib : BIOS.obj (.const:.string)
                  0086c5dc    00000004     SRIOMulticore_fft_1_pe66.oe66 (.const:ti_sdo_ipc_GateMP_A_invalidClose__C)
                  0086c5e0    00000400     SRIOMulticore_fft_1_pe66.oe66 (.const:ti_sysbios_family_c66_Cache_marvalues__C)
                  0086c9e0    00000228     initialization.obj (.const:.string)
                  0086cc08    00000178     SRIOMulticore_fft_1_pe66.oe66 (.const:xdc_runtime_Text_nodeTab__A)
                  0086cd80    000000d4     bioMain.obj (.const:.string)
                  0086ce54    000000d4     slaveTask.obj (.const:.string)
                  0086cf28    000000d0     SRIOMulticore_fft_1_pe66.oe66 (.const:.string)
                  0086cff8    0000008c     masterTask.obj (.const:.string)
                  0086d084    00000074     bioUtilityAndGlobals.obj (.const:.string)
                  0086d0f8    00000058     ti.targets.rts6000.ae66 : Error.oe66 (.const:.string)
                  0086d150    00000044     SRIOMulticore_fft_1_pe66.oe66 (.const:xdc_runtime_Startup_sfxnTab__A)
                  0086d194    00000038     requestProcessingData.obj (.const:.string)
                  0086d1cc    00000038     SRIOMulticore_fft_1_pe66.oe66 (.const:ti_sdo_ipc_notifyDrivers_NotifyDriverShm_Module__FXNS__C)
                  0086d204    00000038     SRIOMulticore_fft_1_pe66.oe66 (.const:ti_sysbios_knl_Task_Object__PARAMS__C)
                  0086d23c    00000004     SRIOMulticore_fft_1_pe66.oe66 (.const:ti_sdo_ipc_GateMP_A_invalidDelete__C)
                  0086d240    00000037     srio_drv.obj (.const:.string:gSrioDriverVersionStr)
                  0086d277    00000001     --HOLE-- [fill = 0]
                  0086d278    00000034     SRIOMulticore_fft_1_pe66.oe66 (.const:ti_sdo_ipc_GateMP_Object__PARAMS__C)
                  0086d2ac    00000034     SRIOMulticore_fft_1_pe66.oe66 (.const:ti_sdo_ipc_notifyDrivers_NotifyDriverShm_Object__PARAMS__C)
                  0086d2e0    00000030     SRIOMulticore_fft_1_pe66.oe66 (.const:ti_sdo_ipc_heaps_HeapMemMP_Object__PARAMS__C)
                  0086d310    00000030     SRIOMulticore_fft_1_pe66.oe66 (.const:ti_sysbios_family_c64p_Hwi_Object__PARAMS__C)
                  0086d340    0000002c     ti.targets.rts6000.ae66 : Startup.oe66 (.const:.string)
                  0086d36c    0000002c     SRIOMulticore_fft_1_pe66.oe66 (.const:ti_sdo_ipc_ListMP_Object__PARAMS__C)
                  0086d398    0000002c     SRIOMulticore_fft_1_pe66.oe66 (.const:ti_sdo_ipc_gates_GateHWSem_Module__FXNS__C)
                  0086d3c4    0000002c     SRIOMulticore_fft_1_pe66.oe66 (.const:ti_sdo_ipc_gates_GateMPSupportNull_Module__FXNS__C)
                  0086d3f0    0000002c     SRIOMulticore_fft_1_pe66.oe66 (.const:ti_sdo_ipc_gates_GatePeterson_Module__FXNS__C)
                  0086d41c    00000028     SRIOMulticore_fft_1_pe66.oe66 (.const:ti_sdo_ipc_heaps_HeapMemMP_Module__FXNS__C)
                  0086d444    00000028     SRIOMulticore_fft_1_pe66.oe66 (.const:ti_sdo_ipc_nsremote_NameServerRemoteNotify_Module__FXNS__C)
                  0086d46c    00000028     SRIOMulticore_fft_1_pe66.oe66 (.const:ti_sdo_ipc_transports_TransportShm_Module__FXNS__C)
                  0086d494    00000028     SRIOMulticore_fft_1_pe66.oe66 (.const:ti_sdo_ipc_transports_TransportShm_Object__PARAMS__C)
                  0086d4bc    00000028     SRIOMulticore_fft_1_pe66.oe66 (.const:ti_sysbios_heaps_HeapMem_Module__FXNS__C)
                  0086d4e4    00000028     SRIOMulticore_fft_1_pe66.oe66 (.const:ti_sysbios_knl_Swi_Object__PARAMS__C)
                  0086d50c    00000024     SRIOMulticore_fft_1_pe66.oe66 (.const:ti_sdo_ipc_gates_GateHWSem_Object__PARAMS__C)
                  0086d530    00000024     SRIOMulticore_fft_1_pe66.oe66 (.const:ti_sdo_ipc_gates_GateMPSupportNull_Object__PARAMS__C)
                  0086d554    00000024     SRIOMulticore_fft_1_pe66.oe66 (.const:ti_sdo_ipc_gates_GatePeterson_Object__PARAMS__C)
                  0086d578    00000024     SRIOMulticore_fft_1_pe66.oe66 (.const:ti_sysbios_gates_GateAll_Module__FXNS__C)
                  0086d59c    00000024     SRIOMulticore_fft_1_pe66.oe66 (.const:ti_sysbios_gates_GateHwi_Module__FXNS__C)
                  0086d5c0    00000024     SRIOMulticore_fft_1_pe66.oe66 (.const:ti_sysbios_gates_GateMutexPri_Module__FXNS__C)
                  0086d5e4    00000024     SRIOMulticore_fft_1_pe66.oe66 (.const:ti_sysbios_gates_GateMutex_Module__FXNS__C)
                  0086d608    00000024     SRIOMulticore_fft_1_pe66.oe66 (.const:ti_sysbios_gates_GateSwi_Module__FXNS__C)
                  0086d62c    00000024     SRIOMulticore_fft_1_pe66.oe66 (.const:ti_sysbios_knl_Clock_Object__PARAMS__C)
                  0086d650    00000024     SRIOMulticore_fft_1_pe66.oe66 (.const:ti_sysbios_knl_Semaphore_Object__PARAMS__C)
                  0086d674    00000024     SRIOMulticore_fft_1_pe66.oe66 (.const:xdc_runtime_GateNull_Module__FXNS__C)
                  0086d698    00000024     SRIOMulticore_fft_1_pe66.oe66 (.const:xdc_runtime_knl_GateThread_Module__FXNS__C)
                  0086d6bc    00000004     SRIOMulticore_fft_1_pe66.oe66 (.const:ti_sdo_ipc_GateMP_E_gateUnavailable__C)
                  0086d6c0    00000022     SRIOMulticore_fft_1_pe66.oe66 (.const:xdc_runtime_Startup_sfxnRts__A)
                  0086d6e2    00000002     --HOLE-- [fill = 0]
                  0086d6e4    00000020     ti.targets.rts6000.ae66 : Core-mem.oe66 (.const:.string)
                  0086d704    00000020     SRIOMulticore_fft_1_pe66.oe66 (.const:ti_sdo_ipc_GateMP_Object__DESC__C)
                  0086d724    00000020     SRIOMulticore_fft_1_pe66.oe66 (.const:ti_sdo_ipc_ListMP_Object__DESC__C)
                  0086d744    00000020     SRIOMulticore_fft_1_pe66.oe66 (.const:ti_sdo_ipc_Notify_Object__DESC__C)
                  0086d764    00000020     SRIOMulticore_fft_1_pe66.oe66 (.const:ti_sdo_ipc_gates_GateHWSem_Object__DESC__C)
                  0086d784    00000020     SRIOMulticore_fft_1_pe66.oe66 (.const:ti_sdo_ipc_gates_GateMPSupportNull_Object__DESC__C)
                  0086d7a4    00000020     SRIOMulticore_fft_1_pe66.oe66 (.const:ti_sdo_ipc_gates_GatePeterson_Object__DESC__C)
                  0086d7c4    00000020     SRIOMulticore_fft_1_pe66.oe66 (.const:ti_sdo_ipc_heaps_HeapMemMP_Object__DESC__C)
                  0086d7e4    00000020     SRIOMulticore_fft_1_pe66.oe66 (.const:ti_sdo_ipc_notifyDrivers_NotifyDriverShm_Object__DESC__C)
                  0086d804    00000020     SRIOMulticore_fft_1_pe66.oe66 (.const:ti_sdo_ipc_nsremote_NameServerRemoteNotify_Object__DESC__C)
                  0086d824    00000020     SRIOMulticore_fft_1_pe66.oe66 (.const:ti_sdo_ipc_nsremote_NameServerRemoteNotify_Object__PARAMS__C)
                  0086d844    00000020     SRIOMulticore_fft_1_pe66.oe66 (.const:ti_sdo_ipc_transports_TransportShm_Object__DESC__C)
                  0086d864    00000020     SRIOMulticore_fft_1_pe66.oe66 (.const:ti_sdo_utils_List_Object__DESC__C)
                  0086d884    00000020     SRIOMulticore_fft_1_pe66.oe66 (.const:ti_sysbios_family_c64p_Hwi_Object__DESC__C)
                  0086d8a4    00000020     SRIOMulticore_fft_1_pe66.oe66 (.const:ti_sysbios_gates_GateAll_Object__DESC__C)
                  0086d8c4    00000020     SRIOMulticore_fft_1_pe66.oe66 (.const:ti_sysbios_gates_GateHwi_Object__DESC__C)
                  0086d8e4    00000020     SRIOMulticore_fft_1_pe66.oe66 (.const:ti_sysbios_gates_GateMutexPri_Object__DESC__C)
                  0086d904    00000020     SRIOMulticore_fft_1_pe66.oe66 (.const:ti_sysbios_gates_GateMutex_Object__DESC__C)
                  0086d924    00000020     SRIOMulticore_fft_1_pe66.oe66 (.const:ti_sysbios_gates_GateSwi_Object__DESC__C)
                  0086d944    00000020     SRIOMulticore_fft_1_pe66.oe66 (.const:ti_sysbios_heaps_HeapMem_Object__DESC__C)
                  0086d964    00000020     SRIOMulticore_fft_1_pe66.oe66 (.const:ti_sysbios_heaps_HeapMem_Object__PARAMS__C)
                  0086d984    00000020     SRIOMulticore_fft_1_pe66.oe66 (.const:ti_sysbios_knl_Clock_Object__DESC__C)
                  0086d9a4    00000020     SRIOMulticore_fft_1_pe66.oe66 (.const:ti_sysbios_knl_Queue_Object__DESC__C)
                  0086d9c4    00000020     SRIOMulticore_fft_1_pe66.oe66 (.const:ti_sysbios_knl_Semaphore_Object__DESC__C)
                  0086d9e4    00000020     SRIOMulticore_fft_1_pe66.oe66 (.const:ti_sysbios_knl_Swi_Object__DESC__C)
                  0086da04    00000020     SRIOMulticore_fft_1_pe66.oe66 (.const:ti_sysbios_knl_Task_Object__DESC__C)
                  0086da24    00000020     SRIOMulticore_fft_1_pe66.oe66 (.const:ti_sysbios_xdcruntime_GateThreadSupport_Object__DESC__C)
                  0086da44    00000020     SRIOMulticore_fft_1_pe66.oe66 (.const:xdc_runtime_GateNull_Object__DESC__C)
                  0086da64    00000020     SRIOMulticore_fft_1_pe66.oe66 (.const:xdc_runtime_knl_GateThread_Object__DESC__C)
                  0086da84    00000004     SRIOMulticore_fft_1_pe66.oe66 (.const:ti_sdo_ipc_GateMP_E_localGate__C)
                  0086da88    00000018     device_srio_loopback.obj (.const:$P$T0$1)
                  0086daa0    00000018     SRIOMulticore_fft_1_pe66.oe66 (.const:ti_sdo_ipc_Notify_Object__PARAMS__C)
                  0086dab8    00000018     SRIOMulticore_fft_1_pe66.oe66 (.const:ti_sdo_utils_List_Object__PARAMS__C)
                  0086dad0    00000018     SRIOMulticore_fft_1_pe66.oe66 (.const:ti_sysbios_gates_GateAll_Object__PARAMS__C)
                  0086dae8    00000018     SRIOMulticore_fft_1_pe66.oe66 (.const:ti_sysbios_gates_GateHwi_Object__PARAMS__C)
                  0086db00    00000018     SRIOMulticore_fft_1_pe66.oe66 (.const:ti_sysbios_gates_GateMutexPri_Object__PARAMS__C)
                  0086db18    00000018     SRIOMulticore_fft_1_pe66.oe66 (.const:ti_sysbios_gates_GateMutex_Object__PARAMS__C)
                  0086db30    00000018     SRIOMulticore_fft_1_pe66.oe66 (.const:ti_sysbios_gates_GateSwi_Object__PARAMS__C)
                  0086db48    00000018     SRIOMulticore_fft_1_pe66.oe66 (.const:ti_sysbios_knl_Queue_Object__PARAMS__C)
                  0086db60    00000018     SRIOMulticore_fft_1_pe66.oe66 (.const:ti_sysbios_knl_Task_hooks__A)
                  0086db78    00000018     SRIOMulticore_fft_1_pe66.oe66 (.const:ti_sysbios_xdcruntime_GateThreadSupport_Object__PARAMS__C)
                  0086db90    00000018     SRIOMulticore_fft_1_pe66.oe66 (.const:xdc_runtime_GateNull_Object__PARAMS__C)
                  0086dba8    00000018     SRIOMulticore_fft_1_pe66.oe66 (.const:xdc_runtime_knl_GateThread_Object__PARAMS__C)
                  0086dbc0    00000011     ti.targets.rts6000.ae66 : System.oe66 (.const:digtohex)
                  0086dbd1    00000003     --HOLE-- [fill = 0]
                  0086dbd4    00000004     SRIOMulticore_fft_1_pe66.oe66 (.const:ti_sdo_ipc_GateMP_LM_create__C)
                  0086dbd8    00000010     SRIOMulticore_fft_1_pe66.oe66 (.const:ti_sdo_ipc_family_c647x_MultiProcSetup_procMap__A)
                  0086dbe8    00000010     SRIOMulticore_fft_1_pe66.oe66 (.const:ti_sysbios_family_c64p_EventCombiner_EVTMASK__C)
                  0086dbf8    00000010     SRIOMulticore_fft_1_pe66.oe66 (.const:xdc_runtime_Startup_firstFxns__A)
                  0086dc08    0000000c     SRIOMulticore_fft_1_pe66.oe66 (.const:ti_sysbios_family_c66_Cache_initSize__C)
                  0086dc14    00000008     ti.targets.rts6000.ae66 : System.oe66 (.const:.string)
                  0086dc1c    00000008     SRIOMulticore_fft_1_pe66.oe66 (.const:ti_sysbios_knl_Idle_funcList__C)
                  0086dc24    00000008     SRIOMulticore_fft_1_pe66.oe66 (.const:ti_sysbios_knl_Task_hooks__C)
                  0086dc2c    00000008     SRIOMulticore_fft_1_pe66.oe66 (.const:xdc_runtime_Startup_firstFxns__C)
                  0086dc34    00000008     SRIOMulticore_fft_1_pe66.oe66 (.const:xdc_runtime_Startup_lastFxns__C)
                  0086dc3c    00000004     SRIOMulticore_fft_1_pe66.oe66 (.const:ti_sdo_ipc_GateMP_LM_delete__C)
                  0086dc40    00000004     SRIOMulticore_fft_1_pe66.oe66 (.const:ti_sdo_ipc_GateMP_LM_enter__C)
                  0086dc44    00000004     SRIOMulticore_fft_1_pe66.oe66 (.const:ti_sdo_ipc_GateMP_LM_leave__C)
                  0086dc48    00000004     SRIOMulticore_fft_1_pe66.oe66 (.const:ti_sdo_ipc_GateMP_LM_open__C)
                  0086dc4c    00000004     SRIOMulticore_fft_1_pe66.oe66 (.const:ti_sdo_ipc_GateMP_Module__diagsEnabled__C)
                  0086dc50    00000004     SRIOMulticore_fft_1_pe66.oe66 (.const:ti_sdo_ipc_GateMP_Module__diagsIncluded__C)
                  0086dc54    00000004     SRIOMulticore_fft_1_pe66.oe66 (.const:ti_sdo_ipc_GateMP_Module__diagsMask__C)
                  0086dc58    00000004     SRIOMulticore_fft_1_pe66.oe66 (.const:ti_sdo_ipc_GateMP_Module__loggerFxn2__C)
                  0086dc5c    00000004     SRIOMulticore_fft_1_pe66.oe66 (.const:ti_sdo_ipc_GateMP_Module__loggerFxn4__C)
                  0086dc60    00000004     SRIOMulticore_fft_1_pe66.oe66 (.const:ti_sdo_ipc_GateMP_Module__loggerObj__C)
                  0086dc64    00000004     SRIOMulticore_fft_1_pe66.oe66 (.const:ti_sdo_ipc_Ipc_A_addrNotCacheAligned__C)
                  0086dc68    00000004     SRIOMulticore_fft_1_pe66.oe66 (.const:ti_sdo_ipc_Ipc_A_addrNotInSharedRegion__C)
                  0086dc6c    00000004     SRIOMulticore_fft_1_pe66.oe66 (.const:ti_sdo_ipc_Ipc_A_internal__C)
                  0086dc70    00000004     SRIOMulticore_fft_1_pe66.oe66 (.const:ti_sdo_ipc_Ipc_A_invArgument__C)
                  0086dc74    00000004     SRIOMulticore_fft_1_pe66.oe66 (.const:ti_sdo_ipc_Ipc_A_invParam__C)
                  0086dc78    00000004     SRIOMulticore_fft_1_pe66.oe66 (.const:ti_sdo_ipc_Ipc_A_nullArgument__C)
                  0086dc7c    00000004     SRIOMulticore_fft_1_pe66.oe66 (.const:ti_sdo_ipc_Ipc_A_nullPointer__C)
                  0086dc80    00000004     SRIOMulticore_fft_1_pe66.oe66 (.const:ti_sdo_ipc_Ipc_E_internal__C)
                  0086dc84    00000004     SRIOMulticore_fft_1_pe66.oe66 (.const:ti_sdo_ipc_Ipc_E_nameFailed__C)
                  0086dc88    00000004     SRIOMulticore_fft_1_pe66.oe66 (.const:ti_sdo_ipc_Ipc_E_versionMismatch__C)
                  0086dc8c    00000004     SRIOMulticore_fft_1_pe66.oe66 (.const:ti_sdo_ipc_Ipc_Module__diagsEnabled__C)
                  0086dc90    00000004     SRIOMulticore_fft_1_pe66.oe66 (.const:ti_sdo_ipc_Ipc_Module__diagsIncluded__C)
                  0086dc94    00000004     SRIOMulticore_fft_1_pe66.oe66 (.const:ti_sdo_ipc_Ipc_Module__diagsMask__C)
                  0086dc98    00000004     SRIOMulticore_fft_1_pe66.oe66 (.const:ti_sdo_ipc_Ipc_numUserFxns__C)
                  0086dc9c    00000004     SRIOMulticore_fft_1_pe66.oe66 (.const:ti_sdo_ipc_Ipc_procSync__C)
                  0086dca0    00000004     SRIOMulticore_fft_1_pe66.oe66 (.const:ti_sdo_ipc_Ipc_userFxns__C)
                  0086dca4    00000004     SRIOMulticore_fft_1_pe66.oe66 (.const:ti_sdo_ipc_ListMP_Module__diagsEnabled__C)
                  0086dca8    00000004     SRIOMulticore_fft_1_pe66.oe66 (.const:ti_sdo_ipc_ListMP_Module__diagsIncluded__C)
                  0086dcac    00000004     SRIOMulticore_fft_1_pe66.oe66 (.const:ti_sdo_ipc_ListMP_Module__diagsMask__C)
                  0086dcb0    00000004     SRIOMulticore_fft_1_pe66.oe66 (.const:ti_sdo_ipc_MessageQ_A_invalidMsg__C)
                  0086dcb4    00000004     SRIOMulticore_fft_1_pe66.oe66 (.const:ti_sdo_ipc_MessageQ_A_invalidObj__C)
                  0086dcb8    00000004     SRIOMulticore_fft_1_pe66.oe66 (.const:ti_sdo_ipc_MessageQ_A_invalidQueueId__C)
                  0086dcbc    00000004     SRIOMulticore_fft_1_pe66.oe66 (.const:ti_sdo_ipc_MessageQ_A_procIdInvalid__C)
                  0086dcc0    00000004     SRIOMulticore_fft_1_pe66.oe66 (.const:ti_sdo_ipc_MessageQ_A_unregisteredTransport__C)
                  0086dcc4    00000004     SRIOMulticore_fft_1_pe66.oe66 (.const:ti_sdo_ipc_MessageQ_Instance_State_highList__O)
                  0086dcc8    00000004     SRIOMulticore_fft_1_pe66.oe66 (.const:ti_sdo_ipc_MessageQ_Instance_State_normalList__O)
                  0086dccc    00000004     SRIOMulticore_fft_1_pe66.oe66 (.const:ti_sdo_ipc_MessageQ_LM_putLocal__C)
                  0086dcd0    00000004     SRIOMulticore_fft_1_pe66.oe66 (.const:ti_sdo_ipc_MessageQ_Module__diagsEnabled__C)
                  0086dcd4    00000004     SRIOMulticore_fft_1_pe66.oe66 (.const:ti_sdo_ipc_MessageQ_Module__diagsIncluded__C)
                  0086dcd8    00000004     SRIOMulticore_fft_1_pe66.oe66 (.const:ti_sdo_ipc_MessageQ_Module__diagsMask__C)
                  0086dcdc    00000004     SRIOMulticore_fft_1_pe66.oe66 (.const:ti_sdo_ipc_MessageQ_Module__loggerFxn4__C)
                  0086dce0    00000004     SRIOMulticore_fft_1_pe66.oe66 (.const:ti_sdo_ipc_MessageQ_Module__loggerObj__C)
                  0086dce4    00000004     SRIOMulticore_fft_1_pe66.oe66 (.const:ti_sdo_ipc_MessageQ_Object__count__C)
                  0086dce8    00000004     SRIOMulticore_fft_1_pe66.oe66 (.const:ti_sdo_ipc_MessageQ_Object__table__C)
                  0086dcec    00000004     SRIOMulticore_fft_1_pe66.oe66 (.const:ti_sdo_ipc_Notify_A_alreadyRegistered__C)
                  0086dcf0    00000004     SRIOMulticore_fft_1_pe66.oe66 (.const:ti_sdo_ipc_Notify_A_internal__C)
                  0086dcf4    00000004     SRIOMulticore_fft_1_pe66.oe66 (.const:ti_sdo_ipc_Notify_A_invArgument__C)
                  0086dcf8    00000004     SRIOMulticore_fft_1_pe66.oe66 (.const:ti_sdo_ipc_Notify_A_notRegistered__C)
                  0086dcfc    00000004     SRIOMulticore_fft_1_pe66.oe66 (.const:ti_sdo_ipc_Notify_A_reservedEvent__C)
                  0086dd00    00000004     SRIOMulticore_fft_1_pe66.oe66 (.const:ti_sdo_ipc_Notify_Module__diagsEnabled__C)
                  0086dd04    00000004     SRIOMulticore_fft_1_pe66.oe66 (.const:ti_sdo_ipc_Notify_Module__diagsIncluded__C)
                  0086dd08    00000004     SRIOMulticore_fft_1_pe66.oe66 (.const:ti_sdo_ipc_Notify_Module__diagsMask__C)
                  0086dd0c    00000004     SRIOMulticore_fft_1_pe66.oe66 (.const:ti_sdo_ipc_Notify_Module__gateObj__C)
                  0086dd10    00000004     SRIOMulticore_fft_1_pe66.oe66 (.const:ti_sdo_ipc_Notify_Object__heap__C)
                  0086dd14    00000004     SRIOMulticore_fft_1_pe66.oe66 (.const:ti_sdo_ipc_Notify_numEvents__C)
                  0086dd18    00000004     SRIOMulticore_fft_1_pe66.oe66 (.const:ti_sdo_ipc_Notify_sendEventPollCount__C)
                  0086dd1c    00000004     SRIOMulticore_fft_1_pe66.oe66 (.const:ti_sdo_ipc_SharedRegion_A_addrOutOfRange__C)
                  0086dd20    00000004     SRIOMulticore_fft_1_pe66.oe66 (.const:ti_sdo_ipc_SharedRegion_A_idTooLarge__C)
                  0086dd24    00000004     SRIOMulticore_fft_1_pe66.oe66 (.const:ti_sdo_ipc_SharedRegion_A_noHeap__C)
                  0086dd28    00000004     SRIOMulticore_fft_1_pe66.oe66 (.const:ti_sdo_ipc_SharedRegion_A_region0Invalid__C)
                  0086dd2c    00000004     SRIOMulticore_fft_1_pe66.oe66 (.const:ti_sdo_ipc_SharedRegion_A_regionInvalid__C)
                  0086dd30    00000004     SRIOMulticore_fft_1_pe66.oe66 (.const:ti_sdo_ipc_SharedRegion_A_reserveTooMuch__C)
                  0086dd34    00000004     SRIOMulticore_fft_1_pe66.oe66 (.const:ti_sdo_ipc_SharedRegion_INVALIDSRPTR__C)
                  0086dd38    00000004     SRIOMulticore_fft_1_pe66.oe66 (.const:ti_sdo_ipc_SharedRegion_Module__diagsEnabled__C)
                  0086dd3c    00000004     SRIOMulticore_fft_1_pe66.oe66 (.const:ti_sdo_ipc_SharedRegion_Module__diagsIncluded__C)
                  0086dd40    00000004     SRIOMulticore_fft_1_pe66.oe66 (.const:ti_sdo_ipc_SharedRegion_Module__diagsMask__C)
                  0086dd44    00000004     SRIOMulticore_fft_1_pe66.oe66 (.const:ti_sdo_ipc_SharedRegion_cacheLineSize__C)
                  0086dd48    00000004     SRIOMulticore_fft_1_pe66.oe66 (.const:ti_sdo_ipc_SharedRegion_numOffsetBits__C)
                  0086dd4c    00000004     SRIOMulticore_fft_1_pe66.oe66 (.const:ti_sdo_ipc_SharedRegion_offsetMask__C)
                  0086dd50    00000004     SRIOMulticore_fft_1_pe66.oe66 (.const:ti_sdo_ipc_family_c647x_Interrupt_INTERDSPINT__C)
                  0086dd54    00000004     SRIOMulticore_fft_1_pe66.oe66 (.const:ti_sdo_ipc_family_c647x_Interrupt_IPCAR0__C)
                  0086dd58    00000004     SRIOMulticore_fft_1_pe66.oe66 (.const:ti_sdo_ipc_family_c647x_Interrupt_IPCGR0__C)
                  0086dd5c    00000004     SRIOMulticore_fft_1_pe66.oe66 (.const:ti_sdo_ipc_family_c647x_Interrupt_KICK0__C)
                  0086dd60    00000004     SRIOMulticore_fft_1_pe66.oe66 (.const:ti_sdo_ipc_family_c647x_Interrupt_KICK1__C)
                  0086dd64    00000004     SRIOMulticore_fft_1_pe66.oe66 (.const:ti_sdo_ipc_family_c647x_MultiProcSetup_A_invalidProcessor__C)
                  0086dd68    00000004     SRIOMulticore_fft_1_pe66.oe66 (.const:ti_sdo_ipc_family_c647x_MultiProcSetup_Module__diagsEnabled__C)
                  0086dd6c    00000004     SRIOMulticore_fft_1_pe66.oe66 (.const:ti_sdo_ipc_family_c647x_MultiProcSetup_Module__diagsIncluded__C)
                  0086dd70    00000004     SRIOMulticore_fft_1_pe66.oe66 (.const:ti_sdo_ipc_family_c647x_MultiProcSetup_Module__diagsMask__C)
                  0086dd74    00000004     SRIOMulticore_fft_1_pe66.oe66 (.const:ti_sdo_ipc_family_c647x_MultiProcSetup_procMap__C)
                  0086dd78    00000004     SRIOMulticore_fft_1_pe66.oe66 (.const:ti_sdo_ipc_family_c647x_NotifySetup_dspIntVectId__C)
                  0086dd7c    00000004     SRIOMulticore_fft_1_pe66.oe66 (.const:ti_sdo_ipc_gates_GateHWSem_A_invSemNum__C)
                  0086dd80    00000004     SRIOMulticore_fft_1_pe66.oe66 (.const:ti_sdo_ipc_gates_GateHWSem_Module__diagsEnabled__C)
                  0086dd84    00000004     SRIOMulticore_fft_1_pe66.oe66 (.const:ti_sdo_ipc_gates_GateHWSem_Module__diagsIncluded__C)
                  0086dd88    00000004     SRIOMulticore_fft_1_pe66.oe66 (.const:ti_sdo_ipc_gates_GateHWSem_Module__diagsMask__C)
                  0086dd8c    00000004     SRIOMulticore_fft_1_pe66.oe66 (.const:ti_sdo_ipc_gates_GateHWSem_baseAddr__C)
                  0086dd90    00000004     SRIOMulticore_fft_1_pe66.oe66 (.const:ti_sdo_ipc_gates_GateHWSem_numSems__C)
                  0086dd94    00000004     SRIOMulticore_fft_1_pe66.oe66 (.const:ti_sdo_ipc_gates_GateHWSem_reservedMaskArr__C)
                  0086dd98    00000004     SRIOMulticore_fft_1_pe66.oe66 (.const:ti_sdo_ipc_gates_GateHWSem_reservedMaskArr__A)
                  0086dd9c    00000004     SRIOMulticore_fft_1_pe66.oe66 (.const:ti_sdo_ipc_gates_GateMPSupportNull_A_invalidAction__C)
                  0086dda0    00000004     SRIOMulticore_fft_1_pe66.oe66 (.const:ti_sdo_ipc_gates_GateMPSupportNull_Module__diagsEnabled__C)
                  0086dda4    00000004     SRIOMulticore_fft_1_pe66.oe66 (.const:ti_sdo_ipc_gates_GateMPSupportNull_Module__diagsIncluded__C)
                  0086dda8    00000004     SRIOMulticore_fft_1_pe66.oe66 (.const:ti_sdo_ipc_gates_GateMPSupportNull_Module__diagsMask__C)
                  0086ddac    00000004     SRIOMulticore_fft_1_pe66.oe66 (.const:ti_sdo_ipc_gates_GateMPSupportNull_action__C)
                  0086ddb0    00000004     SRIOMulticore_fft_1_pe66.oe66 (.const:ti_sdo_ipc_gates_GatePeterson_E_gateRemotelyOpened__C)
                  0086ddb4    00000004     SRIOMulticore_fft_1_pe66.oe66 (.const:ti_sdo_ipc_gates_GatePeterson_Module__diagsEnabled__C)
                  0086ddb8    00000004     SRIOMulticore_fft_1_pe66.oe66 (.const:ti_sdo_ipc_gates_GatePeterson_Module__diagsIncluded__C)
                  0086ddbc    00000004     SRIOMulticore_fft_1_pe66.oe66 (.const:ti_sdo_ipc_gates_GatePeterson_Module__diagsMask__C)
                  0086ddc0    00000004     SRIOMulticore_fft_1_pe66.oe66 (.const:ti_sdo_ipc_gates_GatePeterson_numInstances__C)
                  0086ddc4    00000004     SRIOMulticore_fft_1_pe66.oe66 (.const:ti_sdo_ipc_heaps_HeapMemMP_A_align__C)
                  0086ddc8    00000004     SRIOMulticore_fft_1_pe66.oe66 (.const:ti_sdo_ipc_heaps_HeapMemMP_A_heapSize__C)
                  0086ddcc    00000004     SRIOMulticore_fft_1_pe66.oe66 (.const:ti_sdo_ipc_heaps_HeapMemMP_A_invalidFree__C)
                  0086ddd0    00000004     SRIOMulticore_fft_1_pe66.oe66 (.const:ti_sdo_ipc_heaps_HeapMemMP_A_zeroBlock__C)
                  0086ddd4    00000004     SRIOMulticore_fft_1_pe66.oe66 (.const:ti_sdo_ipc_heaps_HeapMemMP_E_memory__C)
                  0086ddd8    00000004     SRIOMulticore_fft_1_pe66.oe66 (.const:ti_sdo_ipc_heaps_HeapMemMP_Module__diagsEnabled__C)
                  0086dddc    00000004     SRIOMulticore_fft_1_pe66.oe66 (.const:ti_sdo_ipc_heaps_HeapMemMP_Module__diagsIncluded__C)
                  0086dde0    00000004     SRIOMulticore_fft_1_pe66.oe66 (.const:ti_sdo_ipc_heaps_HeapMemMP_Module__diagsMask__C)
                  0086dde4    00000004     SRIOMulticore_fft_1_pe66.oe66 (.const:ti_sdo_ipc_interfaces_IGateMPSupport_Interface__BASE__C)
                  0086dde8    00000004     SRIOMulticore_fft_1_pe66.oe66 (.const:ti_sdo_ipc_interfaces_IMessageQTransport_Interface__BASE__C)
                  0086ddec    00000004     SRIOMulticore_fft_1_pe66.oe66 (.const:ti_sdo_ipc_interfaces_INotifyDriver_Interface__BASE__C)
                  0086ddf0    00000004     SRIOMulticore_fft_1_pe66.oe66 (.const:ti_sdo_ipc_notifyDrivers_NotifyDriverShm_Module__diagsEnabled__C)
                  0086ddf4    00000004     SRIOMulticore_fft_1_pe66.oe66 (.const:ti_sdo_ipc_notifyDrivers_NotifyDriverShm_Module__diagsIncluded__C)
                  0086ddf8    00000004     SRIOMulticore_fft_1_pe66.oe66 (.const:ti_sdo_ipc_notifyDrivers_NotifyDriverShm_Module__diagsMask__C)
                  0086ddfc    00000004     SRIOMulticore_fft_1_pe66.oe66 (.const:ti_sdo_ipc_notifyDrivers_NotifyDriverShm_Object__heap__C)
                  0086de00    00000004     SRIOMulticore_fft_1_pe66.oe66 (.const:ti_sdo_ipc_nsremote_NameServerRemoteNotify_A_invalidValueLen__C)
                  0086de04    00000004     SRIOMulticore_fft_1_pe66.oe66 (.const:ti_sdo_ipc_nsremote_NameServerRemoteNotify_Instance_State_semMultiBlock__O)
                  0086de08    00000004     SRIOMulticore_fft_1_pe66.oe66 (.const:ti_sdo_ipc_nsremote_NameServerRemoteNotify_Instance_State_semRemoteWait__O)
                  0086de0c    00000004     SRIOMulticore_fft_1_pe66.oe66 (.const:ti_sdo_ipc_nsremote_NameServerRemoteNotify_Instance_State_swiObj__O)
                  0086de10    00000004     SRIOMulticore_fft_1_pe66.oe66 (.const:ti_sdo_ipc_nsremote_NameServerRemoteNotify_Module__diagsEnabled__C)
                  0086de14    00000004     SRIOMulticore_fft_1_pe66.oe66 (.const:ti_sdo_ipc_nsremote_NameServerRemoteNotify_Module__diagsIncluded__C)
                  0086de18    00000004     SRIOMulticore_fft_1_pe66.oe66 (.const:ti_sdo_ipc_nsremote_NameServerRemoteNotify_Module__diagsMask__C)
                  0086de1c    00000004     SRIOMulticore_fft_1_pe66.oe66 (.const:ti_sdo_ipc_nsremote_NameServerRemoteNotify_notifyEventId__C)
                  0086de20    00000004     SRIOMulticore_fft_1_pe66.oe66 (.const:ti_sdo_ipc_nsremote_NameServerRemoteNotify_timeout__C)
                  0086de24    00000004     SRIOMulticore_fft_1_pe66.oe66 (.const:ti_sdo_ipc_transports_TransportShmSetup_priority__C)
                  0086de28    00000004     SRIOMulticore_fft_1_pe66.oe66 (.const:ti_sdo_ipc_transports_TransportShm_Instance_State_swiObj__O)
                  0086de2c    00000004     SRIOMulticore_fft_1_pe66.oe66 (.const:ti_sdo_ipc_transports_TransportShm_Module__diagsEnabled__C)
                  0086de30    00000004     SRIOMulticore_fft_1_pe66.oe66 (.const:ti_sdo_ipc_transports_TransportShm_Module__diagsIncluded__C)
                  0086de34    00000004     SRIOMulticore_fft_1_pe66.oe66 (.const:ti_sdo_ipc_transports_TransportShm_Module__diagsMask__C)
                  0086de38    00000004     SRIOMulticore_fft_1_pe66.oe66 (.const:ti_sdo_utils_INameServerRemote_Interface__BASE__C)
                  0086de3c    00000004     SRIOMulticore_fft_1_pe66.oe66 (.const:ti_sdo_utils_List_Object__count__C)
                  0086de40    00000004     SRIOMulticore_fft_1_pe66.oe66 (.const:ti_sdo_utils_List_Object__table__C)
                  0086de44    00000004     SRIOMulticore_fft_1_pe66.oe66 (.const:ti_sdo_utils_MultiProc_A_invalidMultiProcId__C)
                  0086de48    00000004     SRIOMulticore_fft_1_pe66.oe66 (.const:ti_sdo_utils_MultiProc_Module__diagsEnabled__C)
                  0086de4c    00000004     SRIOMulticore_fft_1_pe66.oe66 (.const:ti_sdo_utils_MultiProc_Module__diagsIncluded__C)
                  0086de50    00000004     SRIOMulticore_fft_1_pe66.oe66 (.const:ti_sdo_utils_MultiProc_Module__diagsMask__C)
                  0086de54    00000004     SRIOMulticore_fft_1_pe66.oe66 (.const:ti_sdo_utils_NameServer_A_invArgument__C)
                  0086de58    00000004     SRIOMulticore_fft_1_pe66.oe66 (.const:ti_sdo_utils_NameServer_A_invalidLen__C)
                  0086de5c    00000004     SRIOMulticore_fft_1_pe66.oe66 (.const:ti_sdo_utils_NameServer_E_entryExists__C)
                  0086de60    00000004     SRIOMulticore_fft_1_pe66.oe66 (.const:ti_sdo_utils_NameServer_E_maxReached__C)
                  0086de64    00000004     SRIOMulticore_fft_1_pe66.oe66 (.const:ti_sdo_utils_NameServer_Instance_State_freeList__O)
                  0086de68    00000004     SRIOMulticore_fft_1_pe66.oe66 (.const:ti_sdo_utils_NameServer_Instance_State_nameList__O)
                  0086de6c    00000004     SRIOMulticore_fft_1_pe66.oe66 (.const:ti_sdo_utils_NameServer_Module__diagsEnabled__C)
                  0086de70    00000004     SRIOMulticore_fft_1_pe66.oe66 (.const:ti_sdo_utils_NameServer_Module__diagsIncluded__C)
                  0086de74    00000004     SRIOMulticore_fft_1_pe66.oe66 (.const:ti_sdo_utils_NameServer_Module__diagsMask__C)
                  0086de78    00000004     SRIOMulticore_fft_1_pe66.oe66 (.const:ti_sdo_utils_NameServer_Object__count__C)
                  0086de7c    00000004     SRIOMulticore_fft_1_pe66.oe66 (.const:ti_sdo_utils_NameServer_Object__table__C)
                  0086de80    00000004     SRIOMulticore_fft_1_pe66.oe66 (.const:ti_sysbios_BIOS_Module__diagsEnabled__C)
                  0086de84    00000004     SRIOMulticore_fft_1_pe66.oe66 (.const:ti_sysbios_BIOS_Module__diagsIncluded__C)
                  0086de88    00000004     SRIOMulticore_fft_1_pe66.oe66 (.const:ti_sysbios_BIOS_Module__diagsMask__C)
                  0086de8c    00000004     SRIOMulticore_fft_1_pe66.oe66 (.const:ti_sysbios_BIOS_installedErrorHook__C)
                  0086de90    00000004     SRIOMulticore_fft_1_pe66.oe66 (.const:ti_sysbios_family_c62_TaskSupport_stackAlignment__C)
                  0086de94    00000004     SRIOMulticore_fft_1_pe66.oe66 (.const:ti_sysbios_family_c64p_EventCombiner_E_unpluggedEvent__C)
                  0086de98    00000004     SRIOMulticore_fft_1_pe66.oe66 (.const:ti_sysbios_family_c64p_Exception_E_exceptionMin__C)
                  0086de9c    00000004     SRIOMulticore_fft_1_pe66.oe66 (.const:ti_sysbios_family_c64p_Exception_exceptionHook__C)
                  0086dea0    00000004     SRIOMulticore_fft_1_pe66.oe66 (.const:ti_sysbios_family_c64p_Exception_externalHook__C)
                  0086dea4    00000004     SRIOMulticore_fft_1_pe66.oe66 (.const:ti_sysbios_family_c64p_Exception_internalHook__C)
                  0086dea8    00000004     SRIOMulticore_fft_1_pe66.oe66 (.const:ti_sysbios_family_c64p_Exception_nmiHook__C)
                  0086deac    00000004     SRIOMulticore_fft_1_pe66.oe66 (.const:ti_sysbios_family_c64p_Hwi_E_alreadyDefined__C)
                  0086deb0    00000004     SRIOMulticore_fft_1_pe66.oe66 (.const:ti_sysbios_family_c64p_Hwi_E_handleNotFound__C)
                  0086deb4    00000004     SRIOMulticore_fft_1_pe66.oe66 (.const:ti_sysbios_family_c64p_Hwi_LD_end__C)
                  0086deb8    00000004     SRIOMulticore_fft_1_pe66.oe66 (.const:ti_sysbios_family_c64p_Hwi_LM_begin__C)
                  0086debc    00000004     SRIOMulticore_fft_1_pe66.oe66 (.const:ti_sysbios_family_c64p_Hwi_Module__diagsEnabled__C)
                  0086dec0    00000004     SRIOMulticore_fft_1_pe66.oe66 (.const:ti_sysbios_family_c64p_Hwi_Module__diagsIncluded__C)
                  0086dec4    00000004     SRIOMulticore_fft_1_pe66.oe66 (.const:ti_sysbios_family_c64p_Hwi_Module__diagsMask__C)
                  0086dec8    00000004     SRIOMulticore_fft_1_pe66.oe66 (.const:ti_sysbios_family_c64p_Hwi_Module__loggerFxn1__C)
                  0086decc    00000004     SRIOMulticore_fft_1_pe66.oe66 (.const:ti_sysbios_family_c64p_Hwi_Module__loggerFxn8__C)
                  0086ded0    00000004     SRIOMulticore_fft_1_pe66.oe66 (.const:ti_sysbios_family_c64p_Hwi_Module__loggerObj__C)
                  0086ded4    00000004     SRIOMulticore_fft_1_pe66.oe66 (.const:ti_sysbios_family_c66_Cache_atomicBlockSize__C)
                  0086ded8    00000004     SRIOMulticore_fft_1_pe66.oe66 (.const:ti_sysbios_gates_GateMutexPri_A_badContext__C)
                  0086dedc    00000004     SRIOMulticore_fft_1_pe66.oe66 (.const:ti_sysbios_gates_GateMutexPri_Instance_State_pendQ__O)
                  0086dee0    00000004     SRIOMulticore_fft_1_pe66.oe66 (.const:ti_sysbios_gates_GateMutexPri_Module__diagsEnabled__C)
                  0086dee4    00000004     SRIOMulticore_fft_1_pe66.oe66 (.const:ti_sysbios_gates_GateMutexPri_Module__diagsIncluded__C)
                  0086dee8    00000004     SRIOMulticore_fft_1_pe66.oe66 (.const:ti_sysbios_gates_GateMutexPri_Module__diagsMask__C)
                  0086deec    00000004     SRIOMulticore_fft_1_pe66.oe66 (.const:ti_sysbios_gates_GateMutex_A_badContext__C)
                  0086def0    00000004     SRIOMulticore_fft_1_pe66.oe66 (.const:ti_sysbios_gates_GateMutex_Instance_State_sem__O)
                  0086def4    00000004     SRIOMulticore_fft_1_pe66.oe66 (.const:ti_sysbios_gates_GateMutex_Module__diagsEnabled__C)
                  0086def8    00000004     SRIOMulticore_fft_1_pe66.oe66 (.const:ti_sysbios_gates_GateMutex_Module__diagsIncluded__C)
                  0086defc    00000004     SRIOMulticore_fft_1_pe66.oe66 (.const:ti_sysbios_gates_GateMutex_Module__diagsMask__C)
                  0086df00    00000004     SRIOMulticore_fft_1_pe66.oe66 (.const:ti_sysbios_gates_GateSwi_A_badContext__C)
                  0086df04    00000004     SRIOMulticore_fft_1_pe66.oe66 (.const:ti_sysbios_gates_GateSwi_Module__diagsEnabled__C)
                  0086df08    00000004     SRIOMulticore_fft_1_pe66.oe66 (.const:ti_sysbios_gates_GateSwi_Module__diagsIncluded__C)
                  0086df0c    00000004     SRIOMulticore_fft_1_pe66.oe66 (.const:ti_sysbios_gates_GateSwi_Module__diagsMask__C)
                  0086df10    00000004     SRIOMulticore_fft_1_pe66.oe66 (.const:ti_sysbios_hal_Hwi_E_stackOverflow__C)
                  0086df14    00000004     SRIOMulticore_fft_1_pe66.oe66 (.const:ti_sysbios_heaps_HeapBuf_Instance_State_freeList__O)
                  0086df18    00000004     SRIOMulticore_fft_1_pe66.oe66 (.const:ti_sysbios_heaps_HeapBuf_Object__count__C)
                  0086df1c    00000004     SRIOMulticore_fft_1_pe66.oe66 (.const:ti_sysbios_heaps_HeapBuf_Object__table__C)
                  0086df20    00000004     SRIOMulticore_fft_1_pe66.oe66 (.const:ti_sysbios_heaps_HeapBuf_numConstructedHeaps__C)
                  0086df24    00000004     SRIOMulticore_fft_1_pe66.oe66 (.const:ti_sysbios_heaps_HeapMem_A_align__C)
                  0086df28    00000004     SRIOMulticore_fft_1_pe66.oe66 (.const:ti_sysbios_heaps_HeapMem_A_heapSize__C)
                  0086df2c    00000004     SRIOMulticore_fft_1_pe66.oe66 (.const:ti_sysbios_heaps_HeapMem_A_invalidFree__C)
                  0086df30    00000004     SRIOMulticore_fft_1_pe66.oe66 (.const:ti_sysbios_heaps_HeapMem_A_zeroBlock__C)
                  0086df34    00000004     SRIOMulticore_fft_1_pe66.oe66 (.const:ti_sysbios_heaps_HeapMem_E_memory__C)
                  0086df38    00000004     SRIOMulticore_fft_1_pe66.oe66 (.const:ti_sysbios_heaps_HeapMem_Module__diagsEnabled__C)
                  0086df3c    00000004     SRIOMulticore_fft_1_pe66.oe66 (.const:ti_sysbios_heaps_HeapMem_Module__diagsIncluded__C)
                  0086df40    00000004     SRIOMulticore_fft_1_pe66.oe66 (.const:ti_sysbios_heaps_HeapMem_Module__diagsMask__C)
                  0086df44    00000004     SRIOMulticore_fft_1_pe66.oe66 (.const:ti_sysbios_heaps_HeapMem_Module__gateObj__C)
                  0086df48    00000004     SRIOMulticore_fft_1_pe66.oe66 (.const:ti_sysbios_heaps_HeapMem_Object__count__C)
                  0086df4c    00000004     SRIOMulticore_fft_1_pe66.oe66 (.const:ti_sysbios_heaps_HeapMem_Object__table__C)
                  0086df50    00000004     SRIOMulticore_fft_1_pe66.oe66 (.const:ti_sysbios_heaps_HeapMem_reqAlignMask__C)
                  0086df54    00000004     SRIOMulticore_fft_1_pe66.oe66 (.const:ti_sysbios_heaps_HeapMem_reqAlign__C)
                  0086df58    00000004     SRIOMulticore_fft_1_pe66.oe66 (.const:ti_sysbios_knl_Clock_A_badThreadType__C)
                  0086df5c    00000004     SRIOMulticore_fft_1_pe66.oe66 (.const:ti_sysbios_knl_Clock_LM_begin__C)
                  0086df60    00000004     SRIOMulticore_fft_1_pe66.oe66 (.const:ti_sysbios_knl_Clock_LM_tick__C)
                  0086df64    00000004     SRIOMulticore_fft_1_pe66.oe66 (.const:ti_sysbios_knl_Clock_LW_delayed__C)
                  0086df68    00000004     SRIOMulticore_fft_1_pe66.oe66 (.const:ti_sysbios_knl_Clock_Module_State_clockQ__O)
                  0086df6c    00000004     SRIOMulticore_fft_1_pe66.oe66 (.const:ti_sysbios_knl_Clock_Module__diagsEnabled__C)
                  0086df70    00000004     SRIOMulticore_fft_1_pe66.oe66 (.const:ti_sysbios_knl_Clock_Module__diagsIncluded__C)
                  0086df74    00000004     SRIOMulticore_fft_1_pe66.oe66 (.const:ti_sysbios_knl_Clock_Module__diagsMask__C)
                  0086df78    00000004     SRIOMulticore_fft_1_pe66.oe66 (.const:ti_sysbios_knl_Clock_Module__loggerFxn1__C)
                  0086df7c    00000004     SRIOMulticore_fft_1_pe66.oe66 (.const:ti_sysbios_knl_Clock_Module__loggerFxn2__C)
                  0086df80    00000004     SRIOMulticore_fft_1_pe66.oe66 (.const:ti_sysbios_knl_Clock_Module__loggerObj__C)
                  0086df84    00000004     SRIOMulticore_fft_1_pe66.oe66 (.const:ti_sysbios_knl_Clock_tickMode__C)
                  0086df88    00000004     SRIOMulticore_fft_1_pe66.oe66 (.const:ti_sysbios_knl_Clock_tickSource__C)
                  0086df8c    00000004     SRIOMulticore_fft_1_pe66.oe66 (.const:ti_sysbios_knl_Queue_Object__count__C)
                  0086df90    00000004     SRIOMulticore_fft_1_pe66.oe66 (.const:ti_sysbios_knl_Idle_funcList__A)
                  0086df94    00000004     SRIOMulticore_fft_1_pe66.oe66 (.const:ti_sysbios_knl_Queue_Object__table__C)
                  0086df98    00000004     SRIOMulticore_fft_1_pe66.oe66 (.const:ti_sysbios_knl_Semaphore_A_badContext__C)
                  0086df9c    00000004     SRIOMulticore_fft_1_pe66.oe66 (.const:ti_sysbios_knl_Semaphore_A_noEvents__C)
                  0086dfa0    00000004     SRIOMulticore_fft_1_pe66.oe66 (.const:ti_sysbios_knl_Semaphore_A_overflow__C)
                  0086dfa4    00000004     SRIOMulticore_fft_1_pe66.oe66 (.const:ti_sysbios_knl_Semaphore_Instance_State_pendQ__O)
                  0086dfa8    00000004     SRIOMulticore_fft_1_pe66.oe66 (.const:ti_sysbios_knl_Semaphore_LM_pend__C)
                  0086dfac    00000004     SRIOMulticore_fft_1_pe66.oe66 (.const:ti_sysbios_knl_Semaphore_LM_post__C)
                  0086dfb0    00000004     SRIOMulticore_fft_1_pe66.oe66 (.const:ti_sysbios_knl_Semaphore_Module__diagsEnabled__C)
                  0086dfb4    00000004     SRIOMulticore_fft_1_pe66.oe66 (.const:ti_sysbios_knl_Semaphore_Module__diagsIncluded__C)
                  0086dfb8    00000004     SRIOMulticore_fft_1_pe66.oe66 (.const:ti_sysbios_knl_Semaphore_Module__diagsMask__C)
                  0086dfbc    00000004     SRIOMulticore_fft_1_pe66.oe66 (.const:ti_sysbios_knl_Semaphore_Module__loggerFxn2__C)
                  0086dfc0    00000004     SRIOMulticore_fft_1_pe66.oe66 (.const:ti_sysbios_knl_Semaphore_Module__loggerFxn4__C)
                  0086dfc4    00000004     SRIOMulticore_fft_1_pe66.oe66 (.const:ti_sysbios_knl_Semaphore_Module__loggerObj__C)
                  0086dfc8    00000004     SRIOMulticore_fft_1_pe66.oe66 (.const:ti_sysbios_knl_Swi_A_badPriority__C)
                  0086dfcc    00000004     SRIOMulticore_fft_1_pe66.oe66 (.const:ti_sysbios_knl_Swi_LD_end__C)
                  0086dfd0    00000004     SRIOMulticore_fft_1_pe66.oe66 (.const:ti_sysbios_knl_Swi_LM_begin__C)
                  0086dfd4    00000004     SRIOMulticore_fft_1_pe66.oe66 (.const:ti_sysbios_knl_Swi_LM_post__C)
                  0086dfd8    00000004     SRIOMulticore_fft_1_pe66.oe66 (.const:ti_sysbios_knl_Swi_Module__diagsEnabled__C)
                  0086dfdc    00000004     SRIOMulticore_fft_1_pe66.oe66 (.const:ti_sysbios_knl_Swi_Module__diagsIncluded__C)
                  0086dfe0    00000004     SRIOMulticore_fft_1_pe66.oe66 (.const:ti_sysbios_knl_Swi_Module__diagsMask__C)
                  0086dfe4    00000004     SRIOMulticore_fft_1_pe66.oe66 (.const:ti_sysbios_knl_Swi_Module__loggerFxn1__C)
                  0086dfe8    00000004     SRIOMulticore_fft_1_pe66.oe66 (.const:ti_sysbios_knl_Swi_Module__loggerFxn4__C)
                  0086dfec    00000004     SRIOMulticore_fft_1_pe66.oe66 (.const:ti_sysbios_knl_Swi_Module__loggerObj__C)
                  0086dff0    00000004     SRIOMulticore_fft_1_pe66.oe66 (.const:ti_sysbios_knl_Swi_Object__count__C)
                  0086dff4    00000004     SRIOMulticore_fft_1_pe66.oe66 (.const:ti_sysbios_knl_Swi_Object__table__C)
                  0086dff8    00000004     SRIOMulticore_fft_1_pe66.oe66 (.const:ti_sysbios_knl_Task_A_badPriority__C)
                  0086dffc    00000004     SRIOMulticore_fft_1_pe66.oe66 (.const:ti_sysbios_knl_Task_A_badTaskState__C)
                  0086e000    00000004     SRIOMulticore_fft_1_pe66.oe66 (.const:ti_sysbios_knl_Task_A_badThreadType__C)
                  0086e004    00000004     SRIOMulticore_fft_1_pe66.oe66 (.const:ti_sysbios_knl_Task_A_noPendElem__C)
                  0086e008    00000004     SRIOMulticore_fft_1_pe66.oe66 (.const:ti_sysbios_knl_Task_E_spOutOfBounds__C)
                  0086e00c    00000004     SRIOMulticore_fft_1_pe66.oe66 (.const:ti_sysbios_knl_Task_E_stackOverflow__C)
                  0086e010    00000004     SRIOMulticore_fft_1_pe66.oe66 (.const:ti_sysbios_knl_Task_LD_block__C)
                  0086e014    00000004     SRIOMulticore_fft_1_pe66.oe66 (.const:ti_sysbios_knl_Task_LD_exit__C)
                  0086e018    00000004     SRIOMulticore_fft_1_pe66.oe66 (.const:ti_sysbios_knl_Task_LD_ready__C)
                  0086e01c    00000004     SRIOMulticore_fft_1_pe66.oe66 (.const:ti_sysbios_knl_Task_LM_setPri__C)
                  0086e020    00000004     SRIOMulticore_fft_1_pe66.oe66 (.const:ti_sysbios_knl_Task_LM_switch__C)
                  0086e024    00000004     SRIOMulticore_fft_1_pe66.oe66 (.const:ti_sysbios_knl_Task_LM_yield__C)
                  0086e028    00000004     SRIOMulticore_fft_1_pe66.oe66 (.const:ti_sysbios_knl_Task_Module_State_inactiveQ__O)
                  0086e02c    00000004     SRIOMulticore_fft_1_pe66.oe66 (.const:ti_sysbios_knl_Task_Module_State_terminatedQ__O)
                  0086e030    00000004     SRIOMulticore_fft_1_pe66.oe66 (.const:ti_sysbios_knl_Task_Module__diagsEnabled__C)
                  0086e034    00000004     SRIOMulticore_fft_1_pe66.oe66 (.const:ti_sysbios_knl_Task_Module__diagsIncluded__C)
                  0086e038    00000004     SRIOMulticore_fft_1_pe66.oe66 (.const:ti_sysbios_knl_Task_Module__diagsMask__C)
                  0086e03c    00000004     SRIOMulticore_fft_1_pe66.oe66 (.const:ti_sysbios_knl_Task_Module__loggerFxn2__C)
                  0086e040    00000004     SRIOMulticore_fft_1_pe66.oe66 (.const:ti_sysbios_knl_Task_Module__loggerFxn4__C)
                  0086e044    00000004     SRIOMulticore_fft_1_pe66.oe66 (.const:ti_sysbios_knl_Task_Module__loggerObj__C)
                  0086e048    00000004     SRIOMulticore_fft_1_pe66.oe66 (.const:ti_sysbios_knl_Task_Object__count__C)
                  0086e04c    00000004     SRIOMulticore_fft_1_pe66.oe66 (.const:ti_sysbios_knl_Task_Object__heap__C)
                  0086e050    00000004     SRIOMulticore_fft_1_pe66.oe66 (.const:ti_sysbios_knl_Task_Object__table__C)
                  0086e054    00000004     SRIOMulticore_fft_1_pe66.oe66 (.const:ti_sysbios_knl_Task_allBlockedFunc__C)
                  0086e058    00000004     SRIOMulticore_fft_1_pe66.oe66 (.const:ti_sysbios_knl_Task_defaultStackHeap__C)
                  0086e05c    00000004     SRIOMulticore_fft_1_pe66.oe66 (.const:ti_sysbios_knl_Task_defaultStackSize__C)
                  0086e060    00000004     SRIOMulticore_fft_1_pe66.oe66 (.const:ti_sysbios_knl_Task_numConstructedTasks__C)
                  0086e064    00000004     SRIOMulticore_fft_1_pe66.oe66 (.const:ti_sysbios_knl_Task_numPriorities__C)
                  0086e068    00000004     SRIOMulticore_fft_1_pe66.oe66 (.const:ti_sysbios_timers_timer64_Timer_A_notAvailable__C)
                  0086e06c    00000004     SRIOMulticore_fft_1_pe66.oe66 (.const:ti_sysbios_timers_timer64_Timer_E_cannotSupport__C)
                  0086e070    00000004     SRIOMulticore_fft_1_pe66.oe66 (.const:ti_sysbios_timers_timer64_Timer_Module__diagsEnabled__C)
                  0086e074    00000004     SRIOMulticore_fft_1_pe66.oe66 (.const:ti_sysbios_timers_timer64_Timer_Module__diagsIncluded__C)
                  0086e078    00000004     SRIOMulticore_fft_1_pe66.oe66 (.const:ti_sysbios_timers_timer64_Timer_Module__diagsMask__C)
                  0086e07c    00000004     SRIOMulticore_fft_1_pe66.oe66 (.const:ti_sysbios_timers_timer64_Timer_anyMask__C)
                  0086e080    00000004     SRIOMulticore_fft_1_pe66.oe66 (.const:ti_sysbios_timers_timer64_Timer_freqDivisor__C)
                  0086e084    00000004     SRIOMulticore_fft_1_pe66.oe66 (.const:ti_sysbios_timers_timer64_Timer_numLocalTimers__C)
                  0086e088    00000004     SRIOMulticore_fft_1_pe66.oe66 (.const:ti_sysbios_timers_timer64_Timer_numTimerDevices__C)
                  0086e08c    00000004     SRIOMulticore_fft_1_pe66.oe66 (.const:ti_sysbios_xdcruntime_GateThreadSupport_Instance_State_gate__O)
                  0086e090    00000004     SRIOMulticore_fft_1_pe66.oe66 (.const:xdc_runtime_Assert_E_assertFailed__C)
                  0086e094    00000004     SRIOMulticore_fft_1_pe66.oe66 (.const:xdc_runtime_Core_A_initializedParams__C)
                  0086e098    00000004     SRIOMulticore_fft_1_pe66.oe66 (.const:xdc_runtime_Core_Module__diagsEnabled__C)
                  0086e09c    00000004     SRIOMulticore_fft_1_pe66.oe66 (.const:xdc_runtime_Core_Module__diagsIncluded__C)
                  0086e0a0    00000004     SRIOMulticore_fft_1_pe66.oe66 (.const:xdc_runtime_Core_Module__diagsMask__C)
                  0086e0a4    00000004     SRIOMulticore_fft_1_pe66.oe66 (.const:xdc_runtime_Error_E_generic__C)
                  0086e0a8    00000004     SRIOMulticore_fft_1_pe66.oe66 (.const:xdc_runtime_Error_E_memory__C)
                  0086e0ac    00000004     SRIOMulticore_fft_1_pe66.oe66 (.const:xdc_runtime_Error_Module__diagsEnabled__C)
                  0086e0b0    00000004     SRIOMulticore_fft_1_pe66.oe66 (.const:xdc_runtime_Error_Module__diagsIncluded__C)
                  0086e0b4    00000004     SRIOMulticore_fft_1_pe66.oe66 (.const:xdc_runtime_Error_Module__diagsMask__C)
                  0086e0b8    00000004     SRIOMulticore_fft_1_pe66.oe66 (.const:xdc_runtime_Error_Module__loggerFxn8__C)
                  0086e0bc    00000004     SRIOMulticore_fft_1_pe66.oe66 (.const:xdc_runtime_Error_Module__loggerObj__C)
                  0086e0c0    00000004     SRIOMulticore_fft_1_pe66.oe66 (.const:xdc_runtime_Error_policy__C)
                  0086e0c4    00000004     SRIOMulticore_fft_1_pe66.oe66 (.const:xdc_runtime_Error_raiseHook__C)
                  0086e0c8    00000004     SRIOMulticore_fft_1_pe66.oe66 (.const:xdc_runtime_IGateProvider_Interface__BASE__C)
                  0086e0cc    00000004     SRIOMulticore_fft_1_pe66.oe66 (.const:xdc_runtime_IHeap_Interface__BASE__C)
                  0086e0d0    00000004     SRIOMulticore_fft_1_pe66.oe66 (.const:xdc_runtime_IModule_Interface__BASE__C)
                  0086e0d4    00000004     SRIOMulticore_fft_1_pe66.oe66 (.const:xdc_runtime_Log_L_error__C)
                  0086e0d8    00000004     SRIOMulticore_fft_1_pe66.oe66 (.const:xdc_runtime_Memory_defaultHeapInstance__C)
                  0086e0dc    00000004     SRIOMulticore_fft_1_pe66.oe66 (.const:xdc_runtime_Startup_execImpl__C)
                  0086e0e0    00000004     SRIOMulticore_fft_1_pe66.oe66 (.const:xdc_runtime_Startup_lastFxns__A)
                  0086e0e4    00000004     SRIOMulticore_fft_1_pe66.oe66 (.const:xdc_runtime_Startup_maxPasses__C)
                  0086e0e8    00000004     SRIOMulticore_fft_1_pe66.oe66 (.const:xdc_runtime_Startup_sfxnRts__C)
                  0086e0ec    00000004     SRIOMulticore_fft_1_pe66.oe66 (.const:xdc_runtime_Startup_sfxnTab__C)
                  0086e0f0    00000004     SRIOMulticore_fft_1_pe66.oe66 (.const:xdc_runtime_Startup_startModsFxn__C)
                  0086e0f4    00000004     SRIOMulticore_fft_1_pe66.oe66 (.const:xdc_runtime_System_Module__gateObj__C)
                  0086e0f8    00000004     SRIOMulticore_fft_1_pe66.oe66 (.const:xdc_runtime_System_extendFxn__C)
                  0086e0fc    00000004     SRIOMulticore_fft_1_pe66.oe66 (.const:xdc_runtime_System_maxAtexitHandlers__C)
                  0086e100    00000004     SRIOMulticore_fft_1_pe66.oe66 (.const:xdc_runtime_Text_charTab__C)
                  0086e104    00000004     SRIOMulticore_fft_1_pe66.oe66 (.const:xdc_runtime_Text_nameEmpty__C)
                  0086e108    00000004     SRIOMulticore_fft_1_pe66.oe66 (.const:xdc_runtime_Text_nameStatic__C)
                  0086e10c    00000004     SRIOMulticore_fft_1_pe66.oe66 (.const:xdc_runtime_Text_nameUnknown__C)
                  0086e110    00000004     SRIOMulticore_fft_1_pe66.oe66 (.const:xdc_runtime_Text_nodeTab__C)
                  0086e114    00000004     SRIOMulticore_fft_1_pe66.oe66 (.const:xdc_runtime_Text_visitRopeFxn__C)
                  0086e118    00000002     SRIOMulticore_fft_1_pe66.oe66 (.const:ti_sdo_ipc_GateMP_Module__id__C)
                  0086e11a    00000002     --HOLE-- [fill = 0]
                  0086e11c    00000002     SRIOMulticore_fft_1_pe66.oe66 (.const:ti_sdo_ipc_GateMP_Module__loggerDefined__C)
                  0086e11e    00000002     --HOLE-- [fill = 0]
                  0086e120    00000002     SRIOMulticore_fft_1_pe66.oe66 (.const:ti_sdo_ipc_Ipc_Module__id__C)
                  0086e122    00000002     --HOLE-- [fill = 0]
                  0086e124    00000002     SRIOMulticore_fft_1_pe66.oe66 (.const:ti_sdo_ipc_Ipc_generateSlaveDataForHost__C)
                  0086e126    00000002     --HOLE-- [fill = 0]
                  0086e128    00000002     SRIOMulticore_fft_1_pe66.oe66 (.const:ti_sdo_ipc_ListMP_Module__id__C)
                  0086e12a    00000002     --HOLE-- [fill = 0]
                  0086e12c    00000002     SRIOMulticore_fft_1_pe66.oe66 (.const:ti_sdo_ipc_MessageQ_Module__id__C)
                  0086e12e    00000002     --HOLE-- [fill = 0]
                  0086e130    00000002     SRIOMulticore_fft_1_pe66.oe66 (.const:ti_sdo_ipc_MessageQ_Module__loggerDefined__C)
                  0086e132    00000002     --HOLE-- [fill = 0]
                  0086e134    00000002     SRIOMulticore_fft_1_pe66.oe66 (.const:ti_sdo_ipc_Notify_Module__id__C)
                  0086e136    00000002     --HOLE-- [fill = 0]
                  0086e138    00000002     SRIOMulticore_fft_1_pe66.oe66 (.const:ti_sdo_ipc_Notify_numLines__C)
                  0086e13a    00000002     --HOLE-- [fill = 0]
                  0086e13c    00000002     SRIOMulticore_fft_1_pe66.oe66 (.const:ti_sdo_ipc_Notify_reservedEvents__C)
                  0086e13e    00000002     --HOLE-- [fill = 0]
                  0086e140    00000002     SRIOMulticore_fft_1_pe66.oe66 (.const:ti_sdo_ipc_SharedRegion_Module__id__C)
                  0086e142    00000002     --HOLE-- [fill = 0]
                  0086e144    00000002     SRIOMulticore_fft_1_pe66.oe66 (.const:ti_sdo_ipc_SharedRegion_numEntries__C)
                  0086e146    00000002     --HOLE-- [fill = 0]
                  0086e148    00000002     SRIOMulticore_fft_1_pe66.oe66 (.const:ti_sdo_ipc_SharedRegion_translate__C)
                  0086e14a    00000002     --HOLE-- [fill = 0]
                  0086e14c    00000002     SRIOMulticore_fft_1_pe66.oe66 (.const:ti_sdo_ipc_family_c647x_Interrupt_enableKick__C)
                  0086e14e    00000002     --HOLE-- [fill = 0]
                  0086e150    00000002     SRIOMulticore_fft_1_pe66.oe66 (.const:ti_sdo_ipc_family_c647x_MultiProcSetup_Module__id__C)
                  0086e152    00000002     --HOLE-- [fill = 0]
                  0086e154    00000002     SRIOMulticore_fft_1_pe66.oe66 (.const:ti_sdo_ipc_gates_GateHWSem_Module__id__C)
                  0086e156    00000002     --HOLE-- [fill = 0]
                  0086e158    00000002     SRIOMulticore_fft_1_pe66.oe66 (.const:ti_sdo_ipc_gates_GateMPSupportNull_Module__id__C)
                  0086e15a    00000002     --HOLE-- [fill = 0]
                  0086e15c    00000002     SRIOMulticore_fft_1_pe66.oe66 (.const:ti_sdo_ipc_gates_GatePeterson_Module__id__C)
                  0086e15e    00000002     --HOLE-- [fill = 0]
                  0086e160    00000002     SRIOMulticore_fft_1_pe66.oe66 (.const:ti_sdo_ipc_heaps_HeapMemMP_Module__id__C)
                  0086e162    00000002     --HOLE-- [fill = 0]
                  0086e164    00000002     SRIOMulticore_fft_1_pe66.oe66 (.const:ti_sdo_ipc_notifyDrivers_NotifyDriverShm_Module__id__C)
                  0086e166    00000002     --HOLE-- [fill = 0]
                  0086e168    00000002     SRIOMulticore_fft_1_pe66.oe66 (.const:ti_sdo_ipc_nsremote_NameServerRemoteNotify_Module__id__C)
                  0086e16a    00000002     --HOLE-- [fill = 0]
                  0086e16c    00000002     SRIOMulticore_fft_1_pe66.oe66 (.const:ti_sdo_ipc_transports_TransportShm_Module__id__C)
                  0086e16e    00000002     --HOLE-- [fill = 0]
                  0086e170    00000002     SRIOMulticore_fft_1_pe66.oe66 (.const:ti_sdo_ipc_transports_TransportShm_notifyEventId__C)
                  0086e172    00000002     --HOLE-- [fill = 0]
                  0086e174    00000002     SRIOMulticore_fft_1_pe66.oe66 (.const:ti_sdo_utils_MultiProc_Module__id__C)
                  0086e176    00000002     --HOLE-- [fill = 0]
                  0086e178    00000002     SRIOMulticore_fft_1_pe66.oe66 (.const:ti_sdo_utils_MultiProc_numProcessors__C)
                  0086e17a    00000002     --HOLE-- [fill = 0]
                  0086e17c    00000002     SRIOMulticore_fft_1_pe66.oe66 (.const:ti_sdo_utils_MultiProc_numProcsInCluster__C)
                  0086e17e    00000002     --HOLE-- [fill = 0]
                  0086e180    00000002     SRIOMulticore_fft_1_pe66.oe66 (.const:ti_sdo_utils_NameServer_Module__id__C)
                  0086e182    00000002     --HOLE-- [fill = 0]
                  0086e184    00000002     SRIOMulticore_fft_1_pe66.oe66 (.const:ti_sysbios_BIOS_Module__id__C)
                  0086e186    00000002     --HOLE-- [fill = 0]
                  0086e188    00000002     SRIOMulticore_fft_1_pe66.oe66 (.const:ti_sysbios_family_c64p_EventCombiner_Module__id__C)
                  0086e18a    00000002     --HOLE-- [fill = 0]
                  0086e18c    00000002     SRIOMulticore_fft_1_pe66.oe66 (.const:ti_sysbios_family_c64p_Exception_Module__id__C)
                  0086e18e    00000002     --HOLE-- [fill = 0]
                  0086e190    00000002     SRIOMulticore_fft_1_pe66.oe66 (.const:ti_sysbios_family_c64p_Hwi_Module__id__C)
                  0086e192    00000002     --HOLE-- [fill = 0]
                  0086e194    00000002     SRIOMulticore_fft_1_pe66.oe66 (.const:ti_sysbios_family_c64p_Hwi_Module__loggerDefined__C)
                  0086e196    00000002     --HOLE-- [fill = 0]
                  0086e198    00000002     SRIOMulticore_fft_1_pe66.oe66 (.const:ti_sysbios_gates_GateMutexPri_Module__id__C)
                  0086e19a    00000002     --HOLE-- [fill = 0]
                  0086e19c    00000002     SRIOMulticore_fft_1_pe66.oe66 (.const:ti_sysbios_gates_GateMutex_Module__id__C)
                  0086e19e    00000002     --HOLE-- [fill = 0]
                  0086e1a0    00000002     SRIOMulticore_fft_1_pe66.oe66 (.const:ti_sysbios_gates_GateSwi_Module__id__C)
                  0086e1a2    00000002     --HOLE-- [fill = 0]
                  0086e1a4    00000002     SRIOMulticore_fft_1_pe66.oe66 (.const:ti_sysbios_hal_Hwi_Module__id__C)
                  0086e1a6    00000002     --HOLE-- [fill = 0]
                  0086e1a8    00000002     SRIOMulticore_fft_1_pe66.oe66 (.const:ti_sysbios_heaps_HeapMem_Module__id__C)
                  0086e1aa    00000002     --HOLE-- [fill = 0]
                  0086e1ac    00000002     SRIOMulticore_fft_1_pe66.oe66 (.const:ti_sysbios_knl_Clock_Module__id__C)
                  0086e1ae    00000002     --HOLE-- [fill = 0]
                  0086e1b0    00000002     SRIOMulticore_fft_1_pe66.oe66 (.const:ti_sysbios_knl_Clock_Module__loggerDefined__C)
                  0086e1b2    00000002     --HOLE-- [fill = 0]
                  0086e1b4    00000002     SRIOMulticore_fft_1_pe66.oe66 (.const:ti_sysbios_knl_Semaphore_Module__id__C)
                  0086e1b6    00000002     --HOLE-- [fill = 0]
                  0086e1b8    00000002     SRIOMulticore_fft_1_pe66.oe66 (.const:ti_sysbios_knl_Semaphore_Module__loggerDefined__C)
                  0086e1ba    00000002     --HOLE-- [fill = 0]
                  0086e1bc    00000002     SRIOMulticore_fft_1_pe66.oe66 (.const:ti_sysbios_knl_Swi_Module__id__C)
                  0086e1be    00000002     --HOLE-- [fill = 0]
                  0086e1c0    00000002     SRIOMulticore_fft_1_pe66.oe66 (.const:ti_sysbios_knl_Swi_Module__loggerDefined__C)
                  0086e1c2    00000002     --HOLE-- [fill = 0]
                  0086e1c4    00000002     SRIOMulticore_fft_1_pe66.oe66 (.const:ti_sysbios_knl_Task_Module__id__C)
                  0086e1c6    00000002     --HOLE-- [fill = 0]
                  0086e1c8    00000002     SRIOMulticore_fft_1_pe66.oe66 (.const:ti_sysbios_knl_Task_Module__loggerDefined__C)
                  0086e1ca    00000002     --HOLE-- [fill = 0]
                  0086e1cc    00000002     SRIOMulticore_fft_1_pe66.oe66 (.const:ti_sysbios_knl_Task_deleteTerminatedTasks__C)
                  0086e1ce    00000002     --HOLE-- [fill = 0]
                  0086e1d0    00000002     SRIOMulticore_fft_1_pe66.oe66 (.const:ti_sysbios_knl_Task_initStackFlag__C)
                  0086e1d2    00000002     --HOLE-- [fill = 0]
                  0086e1d4    00000002     SRIOMulticore_fft_1_pe66.oe66 (.const:ti_sysbios_timers_timer64_Timer_Module__id__C)
                  0086e1d6    00000002     --HOLE-- [fill = 0]
                  0086e1d8    00000002     SRIOMulticore_fft_1_pe66.oe66 (.const:ti_sysbios_timers_timer64_Timer_startupNeeded__C)
                  0086e1da    00000002     --HOLE-- [fill = 0]
                  0086e1dc    00000002     SRIOMulticore_fft_1_pe66.oe66 (.const:xdc_runtime_Core_Module__id__C)
                  0086e1de    00000002     --HOLE-- [fill = 0]
                  0086e1e0    00000002     SRIOMulticore_fft_1_pe66.oe66 (.const:xdc_runtime_Error_Module__loggerDefined__C)
                  0086e1e2    00000002     --HOLE-- [fill = 0]
                  0086e1e4    00000002     SRIOMulticore_fft_1_pe66.oe66 (.const:xdc_runtime_Error_maxDepth__C)
                  0086e1e6    00000002     --HOLE-- [fill = 0]
                  0086e1e8    00000002     SRIOMulticore_fft_1_pe66.oe66 (.const:xdc_runtime_Memory_Module__id__C)
                  0086e1ea    00000002     --HOLE-- [fill = 0]
                  0086e1ec    00000002     SRIOMulticore_fft_1_pe66.oe66 (.const:xdc_runtime_Text_charCnt__C)
                  0086e1ee    00000002     --HOLE-- [fill = 0]
                  0086e1f0    00000002     SRIOMulticore_fft_1_pe66.oe66 (.const:xdc_runtime_Text_isLoaded__C)
                  0086e1f2    00000002     --HOLE-- [fill = 0]
                  0086e1f4    00000002     SRIOMulticore_fft_1_pe66.oe66 (.const:xdc_runtime_Text_registryModsLastId__C)
                  0086e1f6    00000002     --HOLE-- [fill = 0]
                  0086e1f8    00000002     SRIOMulticore_fft_1_pe66.oe66 (.const:xdc_runtime_Text_unnamedModsLastId__C)

.fardata.2 
*          0    0086e200    00001e9a     
                  0086e200    00000800     SRIOMulticore_fft_1_pe66.oe66 (.fardata:ti_sdo_ipc_GateMP_Module_State_0_remoteCustom1Gates__A)
                  0086ea00    00000720     SRIOMulticore_fft_1_pe66.oe66 (.fardata)
                  0086f120    000001e0     rts6600_elf.lib : defs.obj (.fardata:_ftable)
                  0086f300    00000180     SRIOMulticore_fft_1_pe66.oe66 (.fardata:ti_sysbios_timers_timer64_Timer_Module_State_0_device__A)
                  0086f480    00000120     initialization.obj (.fardata:qmssGblCfgParams)
                  0086f5a0    000000e0     SRIOMulticore_fft_1_pe66.oe66 (.fardata:ti_sdo_utils_NameServer_Object__table__V)
                  0086f680    000000a0     rts6600_elf.lib : lowlev.obj (.fardata:_stream)
                  0086f720    000000a0     SRIOMulticore_fft_1_pe66.oe66 (.fardata:ti_sdo_ipc_Ipc_Module_State_0_procEntry__A)
                  0086f7c0    00000090     SRIOMulticore_fft_1_pe66.oe66 (.fardata:ti_sdo_ipc_SharedRegion_Module_State_0_regions__A)
                  0086f850    00000080     SRIOMulticore_fft_1_pe66.oe66 (.fardata:ti_sdo_ipc_GateMP_Module_State_0_remoteSystemGates__A)
                  0086f8d0    00000080     SRIOMulticore_fft_1_pe66.oe66 (.fardata:ti_sysbios_knl_Swi_Module_State_0_readyQ__A)
                  0086f950    00000080     SRIOMulticore_fft_1_pe66.oe66 (.fardata:ti_sysbios_knl_Task_Module_State_0_readyQ__A)
                  0086f9d0    00000080     SRIOMulticore_fft_1_pe66.oe66 (.fardata:ti_sysbios_timers_timer64_Timer_Module_State_0_gctrl__A)
                  0086fa50    00000080     SRIOMulticore_fft_1_pe66.oe66 (.fardata:ti_sysbios_timers_timer64_Timer_Module_State_0_handles__A)
                  0086fad0    00000080     SRIOMulticore_fft_1_pe66.oe66 (.fardata:ti_sysbios_timers_timer64_Timer_Module_State_0_intFreqs__A)
                  0086fb50    00000078     rts6600_elf.lib : lowlev.obj (.fardata:_device)
                  0086fbc8    00000078     initialization.obj (.fardata:cppiGblCfgParams)
                  0086fc40    00000078     SRIOMulticore_fft_1_pe66.oe66 (.fardata:ti_sysbios_family_c64p_Hwi_Object__table__V)
                  0086fcb8    0000004c     SRIOMulticore_fft_1_pe66.oe66 (.fardata:ti_sysbios_timers_timer64_Timer_Object__table__V)
                  0086fd04    00000004     rts6600_elf.lib : defs.obj (.fardata)
                  0086fd08    00000044     SRIOMulticore_fft_1_pe66.oe66 (.fardata:ti_sysbios_knl_Task_Object__table__V)
                  0086fd4c    00000004     rts6600_elf.lib : dtor_list.obj (.fardata)
                  0086fd50    00000040                     : cos.obj (.fardata:R$1)
                  0086fd90    00000040                     : sin.obj (.fardata:R$1)
                  0086fdd0    00000040                     : atan.obj (.fardata:arctan_consts$1)
                  0086fe10    00000040     SRIOMulticore_fft_1_pe66.oe66 (.fardata:ti_sdo_ipc_MessageQ_Module_State_0_transports__A)
                  0086fe50    00000040     SRIOMulticore_fft_1_pe66.oe66 (.fardata:ti_sdo_ipc_family_c647x_Interrupt_Module_State_0_fxnTable__A)
                  0086fe90    00000040     SRIOMulticore_fft_1_pe66.oe66 (.fardata:ti_sysbios_gates_GateMutex_Object__table__V)
                  0086fed0    00000030     SRIOMulticore_fft_1_pe66.oe66 (.fardata:ti_sysbios_knl_Swi_Object__table__V)
                  0086ff00    00000020     rts6600_elf.lib : atan.obj (.fardata:A$2)
                  0086ff20    00000020     ti.drv.qmss.ae66 : qmss_drv.oe66 (.fardata:Qmss_highEoiVector)
                  0086ff40    00000020     SRIOMulticore_fft_1_pe66.oe66 (.fardata:ti_sdo_ipc_MessageQ_Module_State_0_heaps__A)
                  0086ff60    00000020     SRIOMulticore_fft_1_pe66.oe66 (.fardata:ti_sdo_ipc_Notify_Module_State_0_notifyHandles__A)
                  0086ff80    00000020     SRIOMulticore_fft_1_pe66.oe66 (.fardata:ti_sdo_ipc_transports_TransportShmSetup_Module_State_0_handles__A)
                  0086ffa0    00000020     SRIOMulticore_fft_1_pe66.oe66 (.fardata:xdc_runtime_System_Module_State_0_atexitHandlers__A)
                  0086ffc0    00000018     SRIOMulticore_fft_1_pe66.oe66 (.fardata:ti_sysbios_gates_GateMutexPri_Object__table__V)
                  0086ffd8    00000014     SRIOMulticore_fft_1_pe66.oe66 (.fardata:ti_sysbios_heaps_HeapMem_Object__table__V)
                  0086ffec    00000004     rts6600_elf.lib : rand.obj (.fardata)
                  0086fff0    00000010     ti.drv.qmss.ae66 : qmss_drv.oe66 (.fardata:Qmss_lowEoiVector)
                  00870000    00000010     SRIOMulticore_fft_1_pe66.oe66 (.fardata:ti_sysbios_gates_GateAll_Object__table__V)
                  00870010    0000000c     rts6600_elf.lib : exit.obj (.fardata)
                  0087001c    00000004     ti.drv.cppi.ae66 : cppi_drv.oe66 (.fardata)
                  00870020    0000000c     SRIOMulticore_fft_1_pe66.oe66 (.fardata:ti_sysbios_gates_GateSwi_Object__table__V)
                  0087002c    00000004     --HOLE--
                  00870030    00000008     SRIOMulticore_fft_1_pe66.oe66 (.fardata:ti_sysbios_hal_Hwi_Object__table__V)
                  00870038    00000008     SRIOMulticore_fft_1_pe66.oe66 (.fardata:ti_sysbios_hal_Timer_Object__table__V)
                  00870040    00000004     SRIOMulticore_fft_1_pe66.oe66 (.fardata:ti_sdo_ipc_GateMP_Module_State_0_remoteCustom2Gates__A)
                  00870044    00000004     --HOLE--
                  00870048    00000004     SRIOMulticore_fft_1_pe66.oe66 (.fardata:ti_sdo_ipc_Notify_Module_State_0_notifyHandles_0__A)
                  0087004c    00000004     --HOLE--
                  00870050    00000004     SRIOMulticore_fft_1_pe66.oe66 (.fardata:ti_sdo_ipc_Notify_Module_State_0_notifyHandles_1__A)
                  00870054    00000004     --HOLE--
                  00870058    00000004     SRIOMulticore_fft_1_pe66.oe66 (.fardata:ti_sdo_ipc_Notify_Module_State_0_notifyHandles_2__A)
                  0087005c    00000004     --HOLE--
                  00870060    00000004     SRIOMulticore_fft_1_pe66.oe66 (.fardata:ti_sdo_ipc_Notify_Module_State_0_notifyHandles_3__A)
                  00870064    00000004     --HOLE--
                  00870068    00000004     SRIOMulticore_fft_1_pe66.oe66 (.fardata:ti_sdo_ipc_Notify_Module_State_0_notifyHandles_4__A)
                  0087006c    00000004     --HOLE--
                  00870070    00000004     SRIOMulticore_fft_1_pe66.oe66 (.fardata:ti_sdo_ipc_Notify_Module_State_0_notifyHandles_5__A)
                  00870074    00000004     --HOLE--
                  00870078    00000004     SRIOMulticore_fft_1_pe66.oe66 (.fardata:ti_sdo_ipc_Notify_Module_State_0_notifyHandles_6__A)
                  0087007c    00000004     --HOLE--
                  00870080    00000004     SRIOMulticore_fft_1_pe66.oe66 (.fardata:ti_sdo_ipc_Notify_Module_State_0_notifyHandles_7__A)
                  00870084    00000004     --HOLE--
                  00870088    00000004     SRIOMulticore_fft_1_pe66.oe66 (.fardata:ti_sysbios_gates_GateHwi_Object__table__V)
                  0087008c    00000004     --HOLE--
                  00870090    00000004     SRIOMulticore_fft_1_pe66.oe66 (.fardata:xdc_runtime_GateNull_Object__table__V)
                  00870094    00000004     --HOLE--
                  00870098    00000002     ti.drv.qmss.ae66 : qmss_drv.oe66 (.fardata:Qmss_cdmaEoiVector)

.stack     0    008700a0    00001000     UNINITIALIZED
                  008700a0    00000008     boot.ae66 : boot.oe66 (.stack)
                  008700a8    00000ff8     --HOLE--

.cio       0    008710a0    00000120     UNINITIALIZED
                  008710a0    00000120     rts6600_elf.lib : trgmsg.obj (.cio)

.bss       0    008711c0    00000058     UNINITIALIZED
                  008711c0    00000054     bioUtilityAndGlobals.obj (.bss)
                  00871214    00000004     SRIOMulticore_fft_1_pe66.oe66 (.bss)

.neardata 
*          0    00871218    00000029     
                  00871218    00000010     initialization.obj (.neardata)
                  00871228    0000000c     multicoreLoopback_osal.obj (.neardata)
                  00871234    00000008     bioUtilityAndGlobals.obj (.neardata)
                  0087123c    00000002     masterTask.obj (.neardata)
                  0087123e    00000002     --HOLE-- [fill = 0]
                  00871240    00000001     ti.drv.qmss.ae66 : qmss_drv.oe66 (.neardata)

.rodata    0    00871244    00000040     
                  00871244    00000040     bioUtilityAndGlobals.obj (.rodata)

.switch    0    00871284    00000080     
                  00871284    00000070     ti.csl.ae66 : csl_chip.oe66 (.switch:CSL_chipReadReg)
                  008712f4    00000010     ipc.lib : Ipc.obj (.switch:ti_sdo_ipc_GateMP_Instance_finalize__F)

.vecs      0    00871400    00000200     
                  00871400    00000200     SRIOMulticore_fft_1_pe66.oe66 (.vecs)

.cinit     0    00871600    00000f4c     
                  00871600    00000e2a     (.cinit..fardata.2.load) [load image, compression = rle]
                  0087242a    00000002     --HOLE-- [fill = 0]
                  0087242c    00000046     (.cinit..rodata.load) [load image, compression = rle]
                  00872472    00000002     --HOLE-- [fill = 0]
                  00872474    00000018     (.cinit..neardata.load) [load image, compression = rle]
                  0087248c    0000000e     (.cinit..fardata.1.load) [load image, compression = rle]
                  0087249a    00000002     --HOLE-- [fill = 0]
                  0087249c    0000000c     (__TI_handler_table)
                  008724a8    0000000b     (.cinit..srioSharedMem.load) [load image, compression = rle]
                  008724b3    00000001     --HOLE-- [fill = 0]
                  008724b4    00000008     (.cinit..bss.load) [load image, compression = zero_init]
                  008724bc    00000008     (.cinit..cppi.load) [load image, compression = zero_init]
                  008724c4    00000008     (.cinit..far.load) [load image, compression = zero_init]
                  008724cc    00000008     (.cinit..fftInput.load) [load image, compression = zero_init]
                  008724d4    00000008     (.cinit..qmss.load) [load image, compression = zero_init]
                  008724dc    00000008     (.cinit..twiddleFactor.load) [load image, compression = zero_init]
                  008724e4    00000008     (.cinit.systemHeap.load) [load image, compression = zero_init]
                  008724ec    00000060     (__TI_cinit_table)

.qmss      0    0c000000    00002400     UNINITIALIZED
                  0c000000    00002400     ti.drv.qmss.ae66 : qmss_drv.oe66 (.qmss)

.srioSharedMem 
*          0    0c002400    00000184     
                  0c002400    00000100     srio_drv.obj (.srioSharedMem) [fill = 0]
                  0c002500    00000084     initialization.obj (.srioSharedMem)

.cppi      0    0c002600    00000200     UNINITIALIZED
                  0c002600    00000200     ti.drv.cppi.ae66 : cppi_drv.oe66 (.cppi)

ti.sdo.ipc.SharedRegion_0 
*          0    0c020000    00200000     NOLOAD SECTION
                  0c020000    00200000     --HOLE--

.fftInput 
*          0    80000000    00011000     UNINITIALIZED
                  80000000    00009000     fftRoutines.obj (.fftInput)
                  80009000    00008000     masterTask.obj (.fftInput)

.twiddleFactor 
*          0    80011000    00001f80     UNINITIALIZED
                  80011000    00001f80     bioUtilityAndGlobals.obj (.twiddleFactor)


LINKER GENERATED COPY TABLES

__TI_cinit_table @ 008724ec records: 12, size/record: 8, table size: 96
	.fardata.2: load addr=00871600, load size=00000e2a bytes, run addr=0086e200, run size=00001e9a bytes, compression=rle
	.rodata: load addr=0087242c, load size=00000046 bytes, run addr=00871244, run size=00000040 bytes, compression=rle
	.neardata: load addr=00872474, load size=00000018 bytes, run addr=00871218, run size=00000029 bytes, compression=rle
	.fardata.1: load addr=0087248c, load size=0000000e bytes, run addr=008690e8, run size=00000008 bytes, compression=rle
	.srioSharedMem: load addr=008724a8, load size=0000000b bytes, run addr=0c002400, run size=00000184 bytes, compression=rle
	.bss: load addr=008724b4, load size=00000008 bytes, run addr=008711c0, run size=00000058 bytes, compression=zero_init
	.cppi: load addr=008724bc, load size=00000008 bytes, run addr=0c002600, run size=00000200 bytes, compression=zero_init
	.far: load addr=008724c4, load size=00000008 bytes, run addr=00863500, run size=00005be8 bytes, compression=zero_init
	.fftInput: load addr=008724cc, load size=00000008 bytes, run addr=80000000, run size=00011000 bytes, compression=zero_init
	.qmss: load addr=008724d4, load size=00000008 bytes, run addr=0c000000, run size=00002400 bytes, compression=zero_init
	.twiddleFactor: load addr=008724dc, load size=00000008 bytes, run addr=80011000, run size=00001f80 bytes, compression=zero_init
	systemHeap: load addr=008724e4, load size=00000008 bytes, run addr=008334c0, run size=00030000 bytes, compression=zero_init


LINKER GENERATED HANDLER TABLE

__TI_handler_table @ 0087249c records: 3, size/record: 4, table size: 12
	index: 0, handler: __TI_zero_init
	index: 1, handler: __TI_decompress_rle24
	index: 2, handler: __TI_decompress_none


GLOBAL SYMBOLS: SORTED ALPHABETICALLY BY Name 

address    name
--------   ----
008317c0   C$$EXIT
0082f438   C$$IO$$
008315a0   CSL_SRIO_Open
00826f20   CSL_chipReadReg
0082c1a0   Cppi_channelEnable
0080fb00   Cppi_configureRxFlow
008315c0   Cppi_getFlowId
008315e0   Cppi_init
008230e0   Cppi_initCfg
00818dc0   Cppi_initDescriptor
0081fdc0   Cppi_open
00816d00   Cppi_rxChannelOpen
0082cf60   Cppi_setCpdmaLoopback
00815680   Cppi_txChannelOpen
00871244   DEVICE_ID1_16BIT
00871248   DEVICE_ID1_8BIT
0087124c   DEVICE_ID2_16BIT
00871250   DEVICE_ID2_8BIT
00871254   DEVICE_ID3_16BIT
00871258   DEVICE_ID3_8BIT
0087125c   DEVICE_ID4_16BIT
00871260   DEVICE_ID4_8BIT
00871264   DEVICE_ID5_16BIT
00871268   DEVICE_ID5_8BIT
0087126c   DEVICE_ID6_16BIT
00871270   DEVICE_ID6_8BIT
00871274   DEVICE_ID7_16BIT
00871278   DEVICE_ID7_8BIT
0087127c   DEVICE_ID8_16BIT
00871280   DEVICE_ID8_8BIT
00812b20   DSP_fft16x16
0082e660   GateMP_Params_init
00827060   GateMP_close
00821160   GateMP_enter
00821360   GateMP_leave
0081b100   GateMP_openByAddr
0081a740   GateMP_sharedMemReq
0082c240   HOSTclose
00828880   HOSTlseek
00829c80   HOSTopen
0082a9a0   HOSTread
00823ee0   HOSTrename
0082c2e0   HOSTtime
0082aa60   HOSTunlink
0082ab20   HOSTwrite
0082e6c0   HeapMemMP_Params_init
0082abe0   HeapMemMP_create
008232a0   HeapMemMP_openByAddr
0081a060   HeapMemMP_sharedMemReq
00819e94   IdFromCore
008092c0   Ipc_attach
00871214   Ipc_sr0MemorySetup
0081d380   Ipc_start
0082aca0   ListMP_create
008119e0   ListMP_getHead
00821560   ListMP_openByAddr
00817140   ListMP_putTail
0081f1e0   ListMP_sharedMemReq
0080c020   MessageQ_put
00824f20   MultiProc_setLocalId
0080f460   NameServer_add
008250a0   NameServer_getHandle
0081d620   NameServer_getLocal
008271a0   Notify_attach
00825220   Notify_intLineRegistered
00811400   Notify_registerEventSingle
008107c0   Notify_sendEvent
00811fa0   Notify_unregisterEventSingle
0080e550   Osal_cppiBeginMemAccess
0080e528   Osal_cppiCsEnter
0080e544   Osal_cppiCsExit
0080e588   Osal_cppiEndMemAccess
0080e504   Osal_cppiFree
0080e4e0   Osal_cppiMalloc
0080e174   Osal_dataBufferInitMemory
0080e5f8   Osal_qmssBeginMemAccess
0080e5b8   Osal_qmssCsEnter
0080e5d4   Osal_qmssCsExit
0080e630   Osal_qmssEndMemAccess
0080e5e4   Osal_qmssMtCsEnter
0080e5e8   Osal_qmssMtCsExit
0080e4b0   Osal_srioBeginDescriptorAccess
0080e448   Osal_srioBeginMemAccess
0080e398   Osal_srioCreateSem
0080e2ec   Osal_srioDataBufferFree
0080e228   Osal_srioDataBufferMalloc
0080e3ac   Osal_srioDeleteSem
0080e4c4   Osal_srioEndDescriptorAccess
0080e480   Osal_srioEndMemAccess
0080e3d8   Osal_srioEnterMultipleCoreCriticalSection
0080e404   Osal_srioEnterSingleCoreCriticalSection
0080e3f4   Osal_srioExitMultipleCoreCriticalSection
0080e428   Osal_srioExitSingleCoreCriticalSection
0080e148   Osal_srioFree
0080e384   Osal_srioLog
0080e114   Osal_srioMalloc
0080e3b8   Osal_srioPendSem
0080e3cc   Osal_srioPostSem
0082f6e0   Qmss_ackInterrupt
00870098   Qmss_cdmaEoiVector
0082f720   Qmss_getMemRegDescSize
0082cfe0   Qmss_getMemRegQueueHandle
00826420   Qmss_getMemoryRegionCfg
00831600   Qmss_getQueueHandle
00831620   Qmss_getQueueNumber
0086ff20   Qmss_highEoiVector
0081aa80   Qmss_init
0080c860   Qmss_insertMemoryRegion
0086fff0   Qmss_lowEoiVector
00821960   Qmss_programAccumulator
0082c380   Qmss_queueClose
0082d060   Qmss_queueOpen
0082ad60   Qmss_setEoiVector
0082ae20   Qmss_setQueueThreshold
00831640   Qmss_start
0082c420   Qmss_startCfg
00824080   SharedRegion_getCacheLineSize
0081ba00   SharedRegion_getEntry
00824220   SharedRegion_getHeap
0081bce0   SharedRegion_getPtr
0081db60   SharedRegion_getSRPtr
008243c0   SharedRegion_isCacheEnabled
0080e680   SrioDevice_init
008037f0   Srio_allocTransmitBuffer
008018b0   Srio_dioCompletionIsr
00803f94   Srio_freeRxDrvBuffer
00803834   Srio_freeTransmitBuffer
008040d8   Srio_getSockOpt
00804584   Srio_getVersion
00804590   Srio_getVersionStr
00801b90   Srio_init
0082f760   Srio_listAdd
0082e720   Srio_listCat
00831660   Srio_listGetHead
00831680   Srio_listGetNext
0082f7a0   Srio_listRemove
0082e780   Srio_listRemoveNode
00801260   Srio_processReceivedBD
00801748   Srio_rxCompletionIsr
00803fe0   Srio_setSockOpt
008030c4   Srio_sockBind
008041e4   Srio_sockClose
00802acc   Srio_sockOpen
00803eb0   Srio_sockRecv
00803868   Srio_sockSend
00802870   Srio_start
0086fd08   TSK_idle
00800000   __ASM__
008710a0   __CIOBUF_
00800070   __ISA__
00800088   __PLAT__
008000b0   __TARG__
008724ec   __TI_CINIT_Base
0087254c   __TI_CINIT_Limit
0087249c   __TI_Handler_Table_Base
008724a8   __TI_Handler_Table_Limit
UNDEFED    __TI_INITARRAY_Base
UNDEFED    __TI_INITARRAY_Limit
008710a0   __TI_STACK_END
00001000   __TI_STACK_SIZE
008711c0   __TI_STATIC_BASE
00000001   __TI_args_main
00831840   __TI_decompress_none
00831860   __TI_decompress_rle24
00870018   __TI_enable_exit_profile_output
ffffffff   __TI_pprof_out_hndl
ffffffff   __TI_prof_data_size
ffffffff   __TI_prof_data_start
00829e40   __TI_zero_init
008000d8   __TRDR__
ffffffff   __binit__
00812560   __c6xabi_divd
0081dde0   __c6xabi_divf
0082b060   __c6xabi_divu
00820000   __c6xabi_divull
0082e7e0   __c6xabi_frcmpyd_div
0082d0e0   __c6xabi_llshl
0082e840   __c6xabi_llshru
0082c4c0   __c6xabi_nround
0082b120   __c6xabi_remi
0082c560   __c6xabi_remu
0082f7e0   __c6xabi_strasgi_64plus
008316a0   __c6xabi_trunc
ffffffff   __c_args__
008316c0   __cxa_atexit
0082afa0   __cxa_finalize
008316e0   __cxa_ia64_exit
0082b060   __divu
0082b120   __remi
0082c560   __remu
0082f7e0   __strasgi_64plus
00831700   __xdc__init
0086f11c   __xdc__init__addr
0082f820   _args_main
00000000   _argsize
008272e0   _auto_init_elf
0082c600   _c_int00
0082c6a0   _cleanup
00870010   _cleanup_ptr
008280a0   _closefile
0082b1e0   _doflush
00870014   _dtors_ptr
0086fd04   _ft_end
0086f120   _ftable
008690e8   _lock
00831720   _nop
00831740   _register_lock
00831760   _register_unlock
008700a0   _stack
0082e8a0   _subcull
00868ce8   _tmpnams
008690ec   _unlock
00828980   _wrt_ok
008317c0   abort
0086b6a8   acc48_le
008711e8   allocatedLen
00823620   atan
008317e0   atexit
00868b20   bindInfo
ffffffff   binit
00868180   buffer9
00871224   bufferCounter
00868aa0   cfg
00829d60   close
00869038   controlVector
00868b48   coreDeviceID
008711f0   coreLoop
00871218   coreNum
00819e28   coreNumberFromId
0081cb40   cos
0086fbc8   cppiGblCfgParams
0087001c   cppiLObj
0c002600   cppiObject
00821f60   cppi_internal_heap_add
0082d1e0   cppi_internal_heap_cache_begin
0082c7e0   cppi_internal_heap_malloc
0082e900   cppi_list_add
0082e960   cppi_list_cache_invalidate
0082c880   cppi_list_cat
00831800   cppi_list_get_head
00831820   cppi_list_get_next
0082d260   cppi_list_remove
00819eb8   disableCaches
00807548   enable_srio
0082b2a0   exit
00829f20   fflush
80009000   fftBuffer
008711f8   firstSendStart
0082f8e0   floor
008206c0   fputc
0082f920   free
0081c2a0   freeBuffer
00871230   free_counter
00868b38   from
008281c0   fseek
00868f48   gDataBufferMemMgr
00871228   gDataBufferMemMgrMaxSize
00868220   gHiPriAccumList
0c002400   gSRIODriverMCB
0086d240   gSrioDriverVersionStr
0081c054   gen_twiddle_fft16x16
0081ce00   generateShortInput
00816148   getNextfreeBuffer
008711e4   hDrvBuffer
008711c0   hSrioDriver
00867500   host_region
008711d4   idx
008160e0   initializeBufferControl
00807c78   initializeMain
008711c4   isAllocated
0c002500   isSRIOInitialized
0c002580   isSRIOSocketsCreated
008711fc   iterationCounter
00819f30   l2_global_address
0087123c   lastOne
0082c9c0   lseek
00818970   main
0082d2e0   malloc
0087122c   malloc_counter
008076d8   masterTaskInitialization
0082ca60   memcpy
0082a000   memset
008711ec   messageSource
00871234   messageValue
0082cb00   modf
008188b4   multicoreTestTask
00868b58   myBuffer
00819f60   myStartupFxn
00871204   myStatus
008711d8   num_bytes
00871220   pp1
008161ec   prepareData
00819ec8   printMessages
00819f74   printStartEnd
00871238   processingCounter
008711dc   ptr_rxDataPayload
008318a0   putc
008318c0   putchar
0c002000   qmssGObj
0086f480   qmssGblCfgParams
00868100   qmssInitConfig
00868e28   qmssLObj
00871240   qmssLObjIsValid
0c000000   queueFree
00819d90   ranDelay
0082d360   rand
008711f4   randomValue
0082d3e0   readmsg
00871208   recvFromCore
0082e2e0   remove
0081c318   requestProcessingData
0087121c   runFlag
00819d34   saveTime
008711e0   sendToCore
0081d030   seperateRealImg
00822160   setvbuf
0081e2e0   sin
00807994   slaveTaskInitialization
0082e9c0   srand
008711c8   srioSocket
00818944   startSlaveUtil
00807588   system_init
00816258   test_multicoreMaster
008189e0   test_multicoreUser
008186b0   threadInitialization
0086c5dc   ti_sdo_ipc_GateMP_A_invalidClose__C
0086d23c   ti_sdo_ipc_GateMP_A_invalidDelete__C
0086d6bc   ti_sdo_ipc_GateMP_E_gateUnavailable__C
0086da84   ti_sdo_ipc_GateMP_E_localGate__C
0080b7c0   ti_sdo_ipc_GateMP_Instance_finalize__F
00806100   ti_sdo_ipc_GateMP_Instance_init__F
0086dbd4   ti_sdo_ipc_GateMP_LM_create__C
0086dc3c   ti_sdo_ipc_GateMP_LM_delete__C
0086dc40   ti_sdo_ipc_GateMP_LM_enter__C
0086dc44   ti_sdo_ipc_GateMP_LM_leave__C
0086dc48   ti_sdo_ipc_GateMP_LM_open__C
0086e200   ti_sdo_ipc_GateMP_Module_State_0_remoteCustom1Gates__A
00870040   ti_sdo_ipc_GateMP_Module_State_0_remoteCustom2Gates__A
0086f850   ti_sdo_ipc_GateMP_Module_State_0_remoteSystemGates__A
0086dc4c   ti_sdo_ipc_GateMP_Module__diagsEnabled__C
0086dc50   ti_sdo_ipc_GateMP_Module__diagsIncluded__C
0086dc54   ti_sdo_ipc_GateMP_Module__diagsMask__C
0086e118   ti_sdo_ipc_GateMP_Module__id__C
0086e11c   ti_sdo_ipc_GateMP_Module__loggerDefined__C
0086dc58   ti_sdo_ipc_GateMP_Module__loggerFxn2__C
0086dc5c   ti_sdo_ipc_GateMP_Module__loggerFxn4__C
0086dc60   ti_sdo_ipc_GateMP_Module__loggerObj__C
0086ea00   ti_sdo_ipc_GateMP_Module__root__V
0086ea08   ti_sdo_ipc_GateMP_Module__state__V
0086d704   ti_sdo_ipc_GateMP_Object__DESC__C
0086d278   ti_sdo_ipc_GateMP_Object__PARAMS__C
0082b360   ti_sdo_ipc_GateMP_Object__create__S
0082f9a0   ti_sdo_ipc_GateMP_Object__delete__S
0082f9e0   ti_sdo_ipc_GateMP_Params__init__S
0082fa20   ti_sdo_ipc_GateMP_RemoteCustom1Proxy_Object__create__S
008318e0   ti_sdo_ipc_GateMP_RemoteCustom1Proxy_Object__delete__S
00831900   ti_sdo_ipc_GateMP_RemoteCustom1Proxy_Params__init__S
00831920   ti_sdo_ipc_GateMP_RemoteCustom1Proxy_Proxy__abstract__S
00831940   ti_sdo_ipc_GateMP_RemoteCustom1Proxy_Proxy__delegate__S
00831960   ti_sdo_ipc_GateMP_RemoteCustom1Proxy_getReservedMask__E
00831980   ti_sdo_ipc_GateMP_RemoteCustom1Proxy_sharedMemReq__E
0082fa60   ti_sdo_ipc_GateMP_RemoteCustom2Proxy_Object__create__S
008319a0   ti_sdo_ipc_GateMP_RemoteCustom2Proxy_Object__delete__S
008319c0   ti_sdo_ipc_GateMP_RemoteCustom2Proxy_Params__init__S
008319e0   ti_sdo_ipc_GateMP_RemoteCustom2Proxy_Proxy__abstract__S
00831a00   ti_sdo_ipc_GateMP_RemoteCustom2Proxy_Proxy__delegate__S
00831a20   ti_sdo_ipc_GateMP_RemoteCustom2Proxy_getReservedMask__E
00831a40   ti_sdo_ipc_GateMP_RemoteCustom2Proxy_sharedMemReq__E
0082faa0   ti_sdo_ipc_GateMP_RemoteSystemProxy_Object__create__S
00831a60   ti_sdo_ipc_GateMP_RemoteSystemProxy_Object__delete__S
00831a80   ti_sdo_ipc_GateMP_RemoteSystemProxy_Params__init__S
00831aa0   ti_sdo_ipc_GateMP_RemoteSystemProxy_Proxy__abstract__S
00831ac0   ti_sdo_ipc_GateMP_RemoteSystemProxy_Proxy__delegate__S
00831ae0   ti_sdo_ipc_GateMP_RemoteSystemProxy_getReservedMask__E
00831b00   ti_sdo_ipc_GateMP_RemoteSystemProxy_sharedMemReq__E
00831b20   ti_sdo_ipc_GateMP_attach__E
00822960   ti_sdo_ipc_GateMP_attach__F
00826580   ti_sdo_ipc_GateMP_createLocal__F
00822b40   ti_sdo_ipc_GateMP_getFreeResource__I
00831b40   ti_sdo_ipc_GateMP_getRegion0ReservedSize__E
0082b420   ti_sdo_ipc_GateMP_getRegion0ReservedSize__F
00831b60   ti_sdo_ipc_GateMP_getSharedAddr__E
00831b80   ti_sdo_ipc_GateMP_getSharedAddr__F
00824560   ti_sdo_ipc_GateMP_openRegion0Reserved__F
00816440   ti_sdo_ipc_GateMP_setRegion0Reserved__F
00831ba0   ti_sdo_ipc_GateMP_start__E
00828b80   ti_sdo_ipc_GateMP_start__F
0086dc64   ti_sdo_ipc_Ipc_A_addrNotCacheAligned__C
0086dc68   ti_sdo_ipc_Ipc_A_addrNotInSharedRegion__C
0086dc6c   ti_sdo_ipc_Ipc_A_internal__C
0086dc70   ti_sdo_ipc_Ipc_A_invArgument__C
0086dc74   ti_sdo_ipc_Ipc_A_invParam__C
0086dc78   ti_sdo_ipc_Ipc_A_nullArgument__C
0086dc7c   ti_sdo_ipc_Ipc_A_nullPointer__C
0086dc80   ti_sdo_ipc_Ipc_E_internal__C
0086dc84   ti_sdo_ipc_Ipc_E_nameFailed__C
0086dc88   ti_sdo_ipc_Ipc_E_versionMismatch__C
0086f720   ti_sdo_ipc_Ipc_Module_State_0_procEntry__A
0086dc8c   ti_sdo_ipc_Ipc_Module__diagsEnabled__C
0086dc90   ti_sdo_ipc_Ipc_Module__diagsIncluded__C
0086dc94   ti_sdo_ipc_Ipc_Module__diagsMask__C
0086e120   ti_sdo_ipc_Ipc_Module__id__C
0086ea50   ti_sdo_ipc_Ipc_Module__state__V
0086e124   ti_sdo_ipc_Ipc_generateSlaveDataForHost__C
0086dc98   ti_sdo_ipc_Ipc_numUserFxns__C
008168a0   ti_sdo_ipc_Ipc_procSyncFinish__I
00814760   ti_sdo_ipc_Ipc_procSyncStart__I
0086dc9c   ti_sdo_ipc_Ipc_procSync__C
0086dca0   ti_sdo_ipc_Ipc_userFxns__C
0081f440   ti_sdo_ipc_ListMP_Instance_finalize__F
0080af20   ti_sdo_ipc_ListMP_Instance_init__F
0086dca4   ti_sdo_ipc_ListMP_Module__diagsEnabled__C
0086dca8   ti_sdo_ipc_ListMP_Module__diagsIncluded__C
0086dcac   ti_sdo_ipc_ListMP_Module__diagsMask__C
0086e128   ti_sdo_ipc_ListMP_Module__id__C
0086ea5c   ti_sdo_ipc_ListMP_Module__root__V
0086ea64   ti_sdo_ipc_ListMP_Module__state__V
0086d724   ti_sdo_ipc_ListMP_Object__DESC__C
0086d36c   ti_sdo_ipc_ListMP_Object__PARAMS__C
0082b4e0   ti_sdo_ipc_ListMP_Object__create__S
0082fae0   ti_sdo_ipc_ListMP_Object__delete__S
0082fb20   ti_sdo_ipc_ListMP_Params__init__S
0086dcb0   ti_sdo_ipc_MessageQ_A_invalidMsg__C
0086dcb4   ti_sdo_ipc_MessageQ_A_invalidObj__C
0086dcb8   ti_sdo_ipc_MessageQ_A_invalidQueueId__C
0086dcbc   ti_sdo_ipc_MessageQ_A_procIdInvalid__C
0086dcc0   ti_sdo_ipc_MessageQ_A_unregisteredTransport__C
0086dcc4   ti_sdo_ipc_MessageQ_Instance_State_highList__O
0086dcc8   ti_sdo_ipc_MessageQ_Instance_State_normalList__O
0086dccc   ti_sdo_ipc_MessageQ_LM_putLocal__C
0086ff40   ti_sdo_ipc_MessageQ_Module_State_0_heaps__A
0086fe10   ti_sdo_ipc_MessageQ_Module_State_0_transports__A
0086dcd0   ti_sdo_ipc_MessageQ_Module__diagsEnabled__C
0086dcd4   ti_sdo_ipc_MessageQ_Module__diagsIncluded__C
0086dcd8   ti_sdo_ipc_MessageQ_Module__diagsMask__C
0086e12c   ti_sdo_ipc_MessageQ_Module__id__C
0086e130   ti_sdo_ipc_MessageQ_Module__loggerDefined__C
0086dcdc   ti_sdo_ipc_MessageQ_Module__loggerFxn4__C
0086dce0   ti_sdo_ipc_MessageQ_Module__loggerObj__C
0086ea68   ti_sdo_ipc_MessageQ_Module__root__V
0086ea70   ti_sdo_ipc_MessageQ_Module__state__V
00831bc0   ti_sdo_ipc_MessageQ_Module_startup__E
00828400   ti_sdo_ipc_MessageQ_Module_startup__F
0086dce4   ti_sdo_ipc_MessageQ_Object__count__C
0082ea20   ti_sdo_ipc_MessageQ_Object__get__S
0086dce8   ti_sdo_ipc_MessageQ_Object__table__C
00831be0   ti_sdo_ipc_MessageQ_SetupTransportProxy_attach__E
00831c00   ti_sdo_ipc_MessageQ_SetupTransportProxy_isRegistered__E
00831c20   ti_sdo_ipc_MessageQ_SetupTransportProxy_sharedMemReq__E
0082fb60   ti_sdo_ipc_MessageQ_registerTransport__E
008256a0   ti_sdo_ipc_MessageQ_registerTransport__F
00831c40   ti_sdo_ipc_MessageQ_unregisterTransport__E
008266e0   ti_sdo_ipc_MessageQ_unregisterTransport__F
0086dcec   ti_sdo_ipc_Notify_A_alreadyRegistered__C
0086dcf0   ti_sdo_ipc_Notify_A_internal__C
0086dcf4   ti_sdo_ipc_Notify_A_invArgument__C
0086dcf8   ti_sdo_ipc_Notify_A_notRegistered__C
0086dcfc   ti_sdo_ipc_Notify_A_reservedEvent__C
00828c80   ti_sdo_ipc_Notify_Instance_finalize__F
00817e00   ti_sdo_ipc_Notify_Instance_init__F
00831c60   ti_sdo_ipc_Notify_Module_GateProxy_enter__E
00831c80   ti_sdo_ipc_Notify_Module_GateProxy_leave__E
00870048   ti_sdo_ipc_Notify_Module_State_0_notifyHandles_0__A
00870050   ti_sdo_ipc_Notify_Module_State_0_notifyHandles_1__A
00870058   ti_sdo_ipc_Notify_Module_State_0_notifyHandles_2__A
00870060   ti_sdo_ipc_Notify_Module_State_0_notifyHandles_3__A
00870068   ti_sdo_ipc_Notify_Module_State_0_notifyHandles_4__A
00870070   ti_sdo_ipc_Notify_Module_State_0_notifyHandles_5__A
00870078   ti_sdo_ipc_Notify_Module_State_0_notifyHandles_6__A
00870080   ti_sdo_ipc_Notify_Module_State_0_notifyHandles_7__A
0086ff60   ti_sdo_ipc_Notify_Module_State_0_notifyHandles__A
0086dd00   ti_sdo_ipc_Notify_Module__diagsEnabled__C
0086dd04   ti_sdo_ipc_Notify_Module__diagsIncluded__C
0086dd08   ti_sdo_ipc_Notify_Module__diagsMask__C
0086dd0c   ti_sdo_ipc_Notify_Module__gateObj__C
0086e134   ti_sdo_ipc_Notify_Module__id__C
0086ea8c   ti_sdo_ipc_Notify_Module__root__V
0086ea94   ti_sdo_ipc_Notify_Module__state__V
00831ca0   ti_sdo_ipc_Notify_Module_startup__E
00825820   ti_sdo_ipc_Notify_Module_startup__F
0086d744   ti_sdo_ipc_Notify_Object__DESC__C
0086daa0   ti_sdo_ipc_Notify_Object__PARAMS__C
0082a0e0   ti_sdo_ipc_Notify_Object__create__S
0086dd10   ti_sdo_ipc_Notify_Object__heap__C
00831cc0   ti_sdo_ipc_Notify_SetupProxy_attach__E
00831ce0   ti_sdo_ipc_Notify_SetupProxy_numIntLines__E
00831d00   ti_sdo_ipc_Notify_SetupProxy_sharedMemReq__E
00831d20   ti_sdo_ipc_Notify_exec__E
00827560   ti_sdo_ipc_Notify_exec__F
0086dd14   ti_sdo_ipc_Notify_numEvents__C
0086e138   ti_sdo_ipc_Notify_numLines__C
0086e13c   ti_sdo_ipc_Notify_reservedEvents__C
0086dd18   ti_sdo_ipc_Notify_sendEventPollCount__C
0086dd1c   ti_sdo_ipc_SharedRegion_A_addrOutOfRange__C
0086dd20   ti_sdo_ipc_SharedRegion_A_idTooLarge__C
0086dd24   ti_sdo_ipc_SharedRegion_A_noHeap__C
0086dd28   ti_sdo_ipc_SharedRegion_A_region0Invalid__C
0086dd2c   ti_sdo_ipc_SharedRegion_A_regionInvalid__C
0086dd30   ti_sdo_ipc_SharedRegion_A_reserveTooMuch__C
0086dd34   ti_sdo_ipc_SharedRegion_INVALIDSRPTR__C
0086f7c0   ti_sdo_ipc_SharedRegion_Module_State_0_regions__A
0086dd38   ti_sdo_ipc_SharedRegion_Module__diagsEnabled__C
0086dd3c   ti_sdo_ipc_SharedRegion_Module__diagsIncluded__C
0086dd40   ti_sdo_ipc_SharedRegion_Module__diagsMask__C
0086e140   ti_sdo_ipc_SharedRegion_Module__id__C
0086ea9c   ti_sdo_ipc_SharedRegion_Module__state__V
00831d40   ti_sdo_ipc_SharedRegion_attach__E
00828d80   ti_sdo_ipc_SharedRegion_attach__F
0086dd44   ti_sdo_ipc_SharedRegion_cacheLineSize__C
00831d60   ti_sdo_ipc_SharedRegion_clearReservedMemory__E
00828e80   ti_sdo_ipc_SharedRegion_clearReservedMemory__F
0086e144   ti_sdo_ipc_SharedRegion_numEntries__C
0086dd48   ti_sdo_ipc_SharedRegion_numOffsetBits__C
0086dd4c   ti_sdo_ipc_SharedRegion_offsetMask__C
00831d80   ti_sdo_ipc_SharedRegion_reserveMemory__E
00819180   ti_sdo_ipc_SharedRegion_reserveMemory__F
00831da0   ti_sdo_ipc_SharedRegion_start__E
008130e0   ti_sdo_ipc_SharedRegion_start__F
0086e148   ti_sdo_ipc_SharedRegion_translate__C
0086dd50   ti_sdo_ipc_family_c647x_Interrupt_INTERDSPINT__C
0086dd54   ti_sdo_ipc_family_c647x_Interrupt_IPCAR0__C
0086dd58   ti_sdo_ipc_family_c647x_Interrupt_IPCGR0__C
0086dd5c   ti_sdo_ipc_family_c647x_Interrupt_KICK0__C
0086dd60   ti_sdo_ipc_family_c647x_Interrupt_KICK1__C
0086fe50   ti_sdo_ipc_family_c647x_Interrupt_Module_State_0_fxnTable__A
0086eaa0   ti_sdo_ipc_family_c647x_Interrupt_Module__state__V
00831dc0   ti_sdo_ipc_family_c647x_Interrupt_Module_startup__E
00828f80   ti_sdo_ipc_family_c647x_Interrupt_Module_startup__F
0086e14c   ti_sdo_ipc_family_c647x_Interrupt_enableKick__C
0082fba0   ti_sdo_ipc_family_c647x_Interrupt_intClear__E
00831de0   ti_sdo_ipc_family_c647x_Interrupt_intDisable__E
00831e00   ti_sdo_ipc_family_c647x_Interrupt_intEnable__E
00828520   ti_sdo_ipc_family_c647x_Interrupt_intRegister__E
0082fbe0   ti_sdo_ipc_family_c647x_Interrupt_intSend__E
0082b5a0   ti_sdo_ipc_family_c647x_Interrupt_intShmStub__I
0082cba0   ti_sdo_ipc_family_c647x_Interrupt_intUnregister__E
0086dd64   ti_sdo_ipc_family_c647x_MultiProcSetup_A_invalidProcessor__C
0086dd68   ti_sdo_ipc_family_c647x_MultiProcSetup_Module__diagsEnabled__C
0086dd6c   ti_sdo_ipc_family_c647x_MultiProcSetup_Module__diagsIncluded__C
0086dd70   ti_sdo_ipc_family_c647x_MultiProcSetup_Module__diagsMask__C
0086e150   ti_sdo_ipc_family_c647x_MultiProcSetup_Module__id__C
00822360   ti_sdo_ipc_family_c647x_MultiProcSetup_init__I
0086dbd8   ti_sdo_ipc_family_c647x_MultiProcSetup_procMap__A
0086dd74   ti_sdo_ipc_family_c647x_MultiProcSetup_procMap__C
0082a1c0   ti_sdo_ipc_family_c647x_NotifySetup_attach__E
0086dd78   ti_sdo_ipc_family_c647x_NotifySetup_dspIntVectId__C
00831e20   ti_sdo_ipc_family_c647x_NotifySetup_numIntLines__E
0082ea80   ti_sdo_ipc_family_c647x_NotifySetup_sharedMemReq__E
0086dd7c   ti_sdo_ipc_gates_GateHWSem_A_invSemNum__C
0082fc20   ti_sdo_ipc_gates_GateHWSem_Handle__label__S
00826840   ti_sdo_ipc_gates_GateHWSem_Instance_init__F
0086d398   ti_sdo_ipc_gates_GateHWSem_Module__FXNS__C
0086dd80   ti_sdo_ipc_gates_GateHWSem_Module__diagsEnabled__C
0086dd84   ti_sdo_ipc_gates_GateHWSem_Module__diagsIncluded__C
0086dd88   ti_sdo_ipc_gates_GateHWSem_Module__diagsMask__C
0086e154   ti_sdo_ipc_gates_GateHWSem_Module__id__C
0086eaa8   ti_sdo_ipc_gates_GateHWSem_Module__root__V
00831e40   ti_sdo_ipc_gates_GateHWSem_Module_startup__E
00829080   ti_sdo_ipc_gates_GateHWSem_Module_startup__F
0086d764   ti_sdo_ipc_gates_GateHWSem_Object__DESC__C
0086d50c   ti_sdo_ipc_gates_GateHWSem_Object__PARAMS__C
0082d460   ti_sdo_ipc_gates_GateHWSem_Object__create__S
0082fc60   ti_sdo_ipc_gates_GateHWSem_Object__delete__S
0082fca0   ti_sdo_ipc_gates_GateHWSem_Params__init__S
0086dd8c   ti_sdo_ipc_gates_GateHWSem_baseAddr__C
0082a2a0   ti_sdo_ipc_gates_GateHWSem_enter__E
00831e60   ti_sdo_ipc_gates_GateHWSem_getReservedMask__E
0082eae0   ti_sdo_ipc_gates_GateHWSem_leave__E
0086dd90   ti_sdo_ipc_gates_GateHWSem_numSems__C
00831e80   ti_sdo_ipc_gates_GateHWSem_query__E
00831ea0   ti_sdo_ipc_gates_GateHWSem_query__F
0086dd98   ti_sdo_ipc_gates_GateHWSem_reservedMaskArr__A
0086dd94   ti_sdo_ipc_gates_GateHWSem_reservedMaskArr__C
00831ec0   ti_sdo_ipc_gates_GateHWSem_sharedMemReq__E
0086dd9c   ti_sdo_ipc_gates_GateMPSupportNull_A_invalidAction__C
0082fce0   ti_sdo_ipc_gates_GateMPSupportNull_Handle__label__S
00831ee0   ti_sdo_ipc_gates_GateMPSupportNull_Instance_init__F
0086d3c4   ti_sdo_ipc_gates_GateMPSupportNull_Module__FXNS__C
0086dda0   ti_sdo_ipc_gates_GateMPSupportNull_Module__diagsEnabled__C
0086dda4   ti_sdo_ipc_gates_GateMPSupportNull_Module__diagsIncluded__C
0086dda8   ti_sdo_ipc_gates_GateMPSupportNull_Module__diagsMask__C
0086e158   ti_sdo_ipc_gates_GateMPSupportNull_Module__id__C
0086eab0   ti_sdo_ipc_gates_GateMPSupportNull_Module__root__V
0086d784   ti_sdo_ipc_gates_GateMPSupportNull_Object__DESC__C
0086d530   ti_sdo_ipc_gates_GateMPSupportNull_Object__PARAMS__C
0082d4e0   ti_sdo_ipc_gates_GateMPSupportNull_Object__create__S
0082fd20   ti_sdo_ipc_gates_GateMPSupportNull_Object__delete__S
0082fd60   ti_sdo_ipc_gates_GateMPSupportNull_Params__init__S
0086ddac   ti_sdo_ipc_gates_GateMPSupportNull_action__C
00829180   ti_sdo_ipc_gates_GateMPSupportNull_enter__E
00831f00   ti_sdo_ipc_gates_GateMPSupportNull_getReservedMask__E
00829280   ti_sdo_ipc_gates_GateMPSupportNull_leave__E
00831f20   ti_sdo_ipc_gates_GateMPSupportNull_query__E
00831f40   ti_sdo_ipc_gates_GateMPSupportNull_query__F
00831f60   ti_sdo_ipc_gates_GateMPSupportNull_sharedMemReq__E
0086ddb0   ti_sdo_ipc_gates_GatePeterson_E_gateRemotelyOpened__C
0082fda0   ti_sdo_ipc_gates_GatePeterson_Handle__label__S
0082eb40   ti_sdo_ipc_gates_GatePeterson_Instance_finalize__F
00815b40   ti_sdo_ipc_gates_GatePeterson_Instance_init__F
0086d3f0   ti_sdo_ipc_gates_GatePeterson_Module__FXNS__C
0086ddb4   ti_sdo_ipc_gates_GatePeterson_Module__diagsEnabled__C
0086ddb8   ti_sdo_ipc_gates_GatePeterson_Module__diagsIncluded__C
0086ddbc   ti_sdo_ipc_gates_GatePeterson_Module__diagsMask__C
0086e15c   ti_sdo_ipc_gates_GatePeterson_Module__id__C
0086eab8   ti_sdo_ipc_gates_GatePeterson_Module__root__V
0086d7a4   ti_sdo_ipc_gates_GatePeterson_Object__DESC__C
0086d554   ti_sdo_ipc_gates_GatePeterson_Object__PARAMS__C
0082b660   ti_sdo_ipc_gates_GatePeterson_Object__create__S
0082fde0   ti_sdo_ipc_gates_GatePeterson_Object__delete__S
0082fe20   ti_sdo_ipc_gates_GatePeterson_Params__init__S
008259a0   ti_sdo_ipc_gates_GatePeterson_enter__E
00831f80   ti_sdo_ipc_gates_GatePeterson_getReservedMask__E
0082cc40   ti_sdo_ipc_gates_GatePeterson_leave__E
0086ddc0   ti_sdo_ipc_gates_GatePeterson_numInstances__C
00831fa0   ti_sdo_ipc_gates_GatePeterson_query__E
00831fc0   ti_sdo_ipc_gates_GatePeterson_query__F
0082eba0   ti_sdo_ipc_gates_GatePeterson_sharedMemReq__E
0086ddc4   ti_sdo_ipc_heaps_HeapMemMP_A_align__C
0086ddc8   ti_sdo_ipc_heaps_HeapMemMP_A_heapSize__C
0086ddcc   ti_sdo_ipc_heaps_HeapMemMP_A_invalidFree__C
0086ddd0   ti_sdo_ipc_heaps_HeapMemMP_A_zeroBlock__C
0086ddd4   ti_sdo_ipc_heaps_HeapMemMP_E_memory__C
0082fe60   ti_sdo_ipc_heaps_HeapMemMP_Handle__label__S
0081f6a0   ti_sdo_ipc_heaps_HeapMemMP_Instance_finalize__F
0080d040   ti_sdo_ipc_heaps_HeapMemMP_Instance_init__F
0086d41c   ti_sdo_ipc_heaps_HeapMemMP_Module__FXNS__C
0086ddd8   ti_sdo_ipc_heaps_HeapMemMP_Module__diagsEnabled__C
0086dddc   ti_sdo_ipc_heaps_HeapMemMP_Module__diagsIncluded__C
0086dde0   ti_sdo_ipc_heaps_HeapMemMP_Module__diagsMask__C
0086e160   ti_sdo_ipc_heaps_HeapMemMP_Module__id__C
0086eac0   ti_sdo_ipc_heaps_HeapMemMP_Module__root__V
0086eac8   ti_sdo_ipc_heaps_HeapMemMP_Module__state__V
0086d7c4   ti_sdo_ipc_heaps_HeapMemMP_Object__DESC__C
0086d2e0   ti_sdo_ipc_heaps_HeapMemMP_Object__PARAMS__C
0082b720   ti_sdo_ipc_heaps_HeapMemMP_Object__create__S
0082fea0   ti_sdo_ipc_heaps_HeapMemMP_Object__delete__S
0082fee0   ti_sdo_ipc_heaps_HeapMemMP_Params__init__S
00807e80   ti_sdo_ipc_heaps_HeapMemMP_alloc__E
008088e0   ti_sdo_ipc_heaps_HeapMemMP_free__E
00817580   ti_sdo_ipc_heaps_HeapMemMP_getStats__E
00831fe0   ti_sdo_ipc_heaps_HeapMemMP_isBlocking__E
00832000   ti_sdo_ipc_heaps_HeapMemMP_isBlocking__F
008179c0   ti_sdo_ipc_heaps_HeapMemMP_postInit__I
0086dde4   ti_sdo_ipc_interfaces_IGateMPSupport_Interface__BASE__C
0086dde8   ti_sdo_ipc_interfaces_IMessageQTransport_Interface__BASE__C
0086ddec   ti_sdo_ipc_interfaces_INotifyDriver_Interface__BASE__C
0082ff20   ti_sdo_ipc_notifyDrivers_NotifyDriverShm_Handle__label__S
0082cce0   ti_sdo_ipc_notifyDrivers_NotifyDriverShm_Instance_finalize__F
008151a0   ti_sdo_ipc_notifyDrivers_NotifyDriverShm_Instance_init__F
00832020   ti_sdo_ipc_notifyDrivers_NotifyDriverShm_InterruptProxy_intClear__E
00832040   ti_sdo_ipc_notifyDrivers_NotifyDriverShm_InterruptProxy_intDisable__E
00832060   ti_sdo_ipc_notifyDrivers_NotifyDriverShm_InterruptProxy_intEnable__E
0082ff60   ti_sdo_ipc_notifyDrivers_NotifyDriverShm_InterruptProxy_intRegister__E
00832080   ti_sdo_ipc_notifyDrivers_NotifyDriverShm_InterruptProxy_intSend__E
008320a0   ti_sdo_ipc_notifyDrivers_NotifyDriverShm_InterruptProxy_intUnregister__E
0086d1cc   ti_sdo_ipc_notifyDrivers_NotifyDriverShm_Module__FXNS__C
0086ddf0   ti_sdo_ipc_notifyDrivers_NotifyDriverShm_Module__diagsEnabled__C
0086ddf4   ti_sdo_ipc_notifyDrivers_NotifyDriverShm_Module__diagsIncluded__C
0086ddf8   ti_sdo_ipc_notifyDrivers_NotifyDriverShm_Module__diagsMask__C
0086e164   ti_sdo_ipc_notifyDrivers_NotifyDriverShm_Module__id__C
0086eacc   ti_sdo_ipc_notifyDrivers_NotifyDriverShm_Module__root__V
0086d7e4   ti_sdo_ipc_notifyDrivers_NotifyDriverShm_Object__DESC__C
0086d2ac   ti_sdo_ipc_notifyDrivers_NotifyDriverShm_Object__PARAMS__C
0082b7e0   ti_sdo_ipc_notifyDrivers_NotifyDriverShm_Object__create__S
0082ffa0   ti_sdo_ipc_notifyDrivers_NotifyDriverShm_Object__delete__S
0086ddfc   ti_sdo_ipc_notifyDrivers_NotifyDriverShm_Object__heap__C
0082ffe0   ti_sdo_ipc_notifyDrivers_NotifyDriverShm_Params__init__S
0081f900   ti_sdo_ipc_notifyDrivers_NotifyDriverShm_disableEvent__E
00830020   ti_sdo_ipc_notifyDrivers_NotifyDriverShm_disable__E
00824700   ti_sdo_ipc_notifyDrivers_NotifyDriverShm_enableEvent__E
00830060   ti_sdo_ipc_notifyDrivers_NotifyDriverShm_enable__E
0081d0c0   ti_sdo_ipc_notifyDrivers_NotifyDriverShm_isr__I
008237e0   ti_sdo_ipc_notifyDrivers_NotifyDriverShm_registerEvent__E
00822560   ti_sdo_ipc_notifyDrivers_NotifyDriverShm_sendEvent__E
0082ec00   ti_sdo_ipc_notifyDrivers_NotifyDriverShm_setNotifyHandle__E
008320c0   ti_sdo_ipc_notifyDrivers_NotifyDriverShm_sharedMemReq__E
0081e560   ti_sdo_ipc_notifyDrivers_NotifyDriverShm_sharedMemReq__F
008248a0   ti_sdo_ipc_notifyDrivers_NotifyDriverShm_unregisterEvent__E
0086de00   ti_sdo_ipc_nsremote_NameServerRemoteNotify_A_invalidValueLen__C
008300a0   ti_sdo_ipc_nsremote_NameServerRemoteNotify_Handle__label__S
0086de04   ti_sdo_ipc_nsremote_NameServerRemoteNotify_Instance_State_semMultiBlock__O
0086de08   ti_sdo_ipc_nsremote_NameServerRemoteNotify_Instance_State_semRemoteWait__O
0086de0c   ti_sdo_ipc_nsremote_NameServerRemoteNotify_Instance_State_swiObj__O
00828640   ti_sdo_ipc_nsremote_NameServerRemoteNotify_Instance_finalize__F
0080eda0   ti_sdo_ipc_nsremote_NameServerRemoteNotify_Instance_init__F
0086d444   ti_sdo_ipc_nsremote_NameServerRemoteNotify_Module__FXNS__C
0086de10   ti_sdo_ipc_nsremote_NameServerRemoteNotify_Module__diagsEnabled__C
0086de14   ti_sdo_ipc_nsremote_NameServerRemoteNotify_Module__diagsIncluded__C
0086de18   ti_sdo_ipc_nsremote_NameServerRemoteNotify_Module__diagsMask__C
0086e168   ti_sdo_ipc_nsremote_NameServerRemoteNotify_Module__id__C
0086ead4   ti_sdo_ipc_nsremote_NameServerRemoteNotify_Module__root__V
0086d804   ti_sdo_ipc_nsremote_NameServerRemoteNotify_Object__DESC__C
0086d824   ti_sdo_ipc_nsremote_NameServerRemoteNotify_Object__PARAMS__C
0082b8a0   ti_sdo_ipc_nsremote_NameServerRemoteNotify_Object__create__S
008300e0   ti_sdo_ipc_nsremote_NameServerRemoteNotify_Object__delete__S
00830120   ti_sdo_ipc_nsremote_NameServerRemoteNotify_Object__first__S
00830160   ti_sdo_ipc_nsremote_NameServerRemoteNotify_Object__next__S
008301a0   ti_sdo_ipc_nsremote_NameServerRemoteNotify_Params__init__S
00824a40   ti_sdo_ipc_nsremote_NameServerRemoteNotify_attach__E
008320e0   ti_sdo_ipc_nsremote_NameServerRemoteNotify_cbFxn__I
0082d560   ti_sdo_ipc_nsremote_NameServerRemoteNotify_detach__E
008301e0   ti_sdo_ipc_nsremote_NameServerRemoteNotify_get__E
00813c60   ti_sdo_ipc_nsremote_NameServerRemoteNotify_get__F
0086de1c   ti_sdo_ipc_nsremote_NameServerRemoteNotify_notifyEventId__C
00830220   ti_sdo_ipc_nsremote_NameServerRemoteNotify_sharedMemReq__E
0081adc0   ti_sdo_ipc_nsremote_NameServerRemoteNotify_swiFxn__I
0086de20   ti_sdo_ipc_nsremote_NameServerRemoteNotify_timeout__C
0086ff80   ti_sdo_ipc_transports_TransportShmSetup_Module_State_0_handles__A
0086eae4   ti_sdo_ipc_transports_TransportShmSetup_Module__state__V
00829380   ti_sdo_ipc_transports_TransportShmSetup_attach__E
00832100   ti_sdo_ipc_transports_TransportShmSetup_isRegistered__E
0086de24   ti_sdo_ipc_transports_TransportShmSetup_priority__C
0082ec60   ti_sdo_ipc_transports_TransportShmSetup_sharedMemReq__E
00830260   ti_sdo_ipc_transports_TransportShm_Handle__label__S
0086de28   ti_sdo_ipc_transports_TransportShm_Instance_State_swiObj__O
00822760   ti_sdo_ipc_transports_TransportShm_Instance_finalize__F
0080a600   ti_sdo_ipc_transports_TransportShm_Instance_init__F
0086d46c   ti_sdo_ipc_transports_TransportShm_Module__FXNS__C
0086de2c   ti_sdo_ipc_transports_TransportShm_Module__diagsEnabled__C
0086de30   ti_sdo_ipc_transports_TransportShm_Module__diagsIncluded__C
0086de34   ti_sdo_ipc_transports_TransportShm_Module__diagsMask__C
0086e16c   ti_sdo_ipc_transports_TransportShm_Module__id__C
0086eadc   ti_sdo_ipc_transports_TransportShm_Module__root__V
0086d844   ti_sdo_ipc_transports_TransportShm_Object__DESC__C
0086d494   ti_sdo_ipc_transports_TransportShm_Object__PARAMS__C
0082b960   ti_sdo_ipc_transports_TransportShm_Object__create__S
008302a0   ti_sdo_ipc_transports_TransportShm_Object__delete__S
008302e0   ti_sdo_ipc_transports_TransportShm_Params__init__S
00832120   ti_sdo_ipc_transports_TransportShm_control__E
00832140   ti_sdo_ipc_transports_TransportShm_getStatus__E
0086e170   ti_sdo_ipc_transports_TransportShm_notifyEventId__C
00832160   ti_sdo_ipc_transports_TransportShm_notifyFxn__I
00832180   ti_sdo_ipc_transports_TransportShm_openByAddr__E
0081b400   ti_sdo_ipc_transports_TransportShm_openByAddr__F
008141e0   ti_sdo_ipc_transports_TransportShm_put__E
008321a0   ti_sdo_ipc_transports_TransportShm_setErrFxn__E
008321c0   ti_sdo_ipc_transports_TransportShm_setErrFxn__F
008321e0   ti_sdo_ipc_transports_TransportShm_sharedMemReq__E
008269a0   ti_sdo_ipc_transports_TransportShm_sharedMemReq__F
0082d5e0   ti_sdo_ipc_transports_TransportShm_swiFxn__I
0086de38   ti_sdo_utils_INameServerRemote_Interface__BASE__C
00832200   ti_sdo_utils_List_Instance_init__F
0086eae8   ti_sdo_utils_List_Module__root__V
0086d864   ti_sdo_utils_List_Object__DESC__C
0086dab8   ti_sdo_utils_List_Object__PARAMS__C
0086de3c   ti_sdo_utils_List_Object__count__C
0082d660   ti_sdo_utils_List_Object__create__S
00830320   ti_sdo_utils_List_Object__destruct__S
0082ecc0   ti_sdo_utils_List_Object__get__S
0086de40   ti_sdo_utils_List_Object__table__C
0086de44   ti_sdo_utils_MultiProc_A_invalidMultiProcId__C
0086de48   ti_sdo_utils_MultiProc_Module__diagsEnabled__C
0086de4c   ti_sdo_utils_MultiProc_Module__diagsIncluded__C
0086de50   ti_sdo_utils_MultiProc_Module__diagsMask__C
0086e174   ti_sdo_utils_MultiProc_Module__id__C
0086eaf0   ti_sdo_utils_MultiProc_Module__state__V
00832220   ti_sdo_utils_MultiProc_getClusterId__E
00832240   ti_sdo_utils_MultiProc_getClusterId__F
0086e178   ti_sdo_utils_MultiProc_numProcessors__C
0086e17c   ti_sdo_utils_MultiProc_numProcsInCluster__C
0086eb04   ti_sdo_utils_NameServerRemoteNull_Module__root__V
0086de54   ti_sdo_utils_NameServer_A_invArgument__C
0086de58   ti_sdo_utils_NameServer_A_invalidLen__C
0086de5c   ti_sdo_utils_NameServer_E_entryExists__C
0086de60   ti_sdo_utils_NameServer_E_maxReached__C
0086de64   ti_sdo_utils_NameServer_Instance_State_freeList__O
0086de68   ti_sdo_utils_NameServer_Instance_State_nameList__O
008690b8   ti_sdo_utils_NameServer_Module_State_0_nsRemoteHandle__A
0086de6c   ti_sdo_utils_NameServer_Module__diagsEnabled__C
0086de70   ti_sdo_utils_NameServer_Module__diagsIncluded__C
0086de74   ti_sdo_utils_NameServer_Module__diagsMask__C
0086e180   ti_sdo_utils_NameServer_Module__id__C
0086eaf4   ti_sdo_utils_NameServer_Module__root__V
00830360   ti_sdo_utils_NameServer_Module__startupDone__F
00832260   ti_sdo_utils_NameServer_Module__startupDone__S
0086eafc   ti_sdo_utils_NameServer_Module__state__V
00832280   ti_sdo_utils_NameServer_Module_startup__E
00825b20   ti_sdo_utils_NameServer_Module_startup__F
0086de78   ti_sdo_utils_NameServer_Object__count__C
008303a0   ti_sdo_utils_NameServer_Object__first__S
0082ed20   ti_sdo_utils_NameServer_Object__get__S
008303e0   ti_sdo_utils_NameServer_Object__next__S
0086de7c   ti_sdo_utils_NameServer_Object__table__C
0086f5a0   ti_sdo_utils_NameServer_Object__table__V
008322a0   ti_sdo_utils_NameServer_SetupProxy_attach__E
008322c0   ti_sdo_utils_NameServer_SetupProxy_sharedMemReq__E
00826b00   ti_sdo_utils_NameServer_isRegistered__E
00826c60   ti_sdo_utils_NameServer_registerRemoteDriver__E
00826dc0   ti_sdo_utils_NameServer_unregisterRemoteDriver__E
0086de80   ti_sysbios_BIOS_Module__diagsEnabled__C
0086de84   ti_sysbios_BIOS_Module__diagsIncluded__C
0086de88   ti_sysbios_BIOS_Module__diagsMask__C
0086e184   ti_sysbios_BIOS_Module__id__C
0086eb0c   ti_sysbios_BIOS_Module__state__V
008322e0   ti_sysbios_BIOS_RtsGateProxy_enter__E
00832300   ti_sysbios_BIOS_RtsGateProxy_leave__E
0082ba20   ti_sysbios_BIOS_errorRaiseHook__I
0082ed80   ti_sysbios_BIOS_exitFunc__I
00832320   ti_sysbios_BIOS_getThreadType__E
0086de8c   ti_sysbios_BIOS_installedErrorHook__C
0082ede0   ti_sysbios_BIOS_registerRTSLock__I
00832340   ti_sysbios_BIOS_setThreadType__E
00830420   ti_sysbios_BIOS_startFunc__I
00830460   ti_sysbios_BIOS_start__E
00832360   ti_sysbios_family_c62_TaskSupport_Module__startupDone__S
0082f860   ti_sysbios_family_c62_TaskSupport_buildTaskStack
00832380   ti_sysbios_family_c62_TaskSupport_checkStack__E
008323a0   ti_sysbios_family_c62_TaskSupport_getStackAlignment__E
00831780   ti_sysbios_family_c62_TaskSupport_glue
0086de90   ti_sysbios_family_c62_TaskSupport_stackAlignment__C
0082d6e0   ti_sysbios_family_c62_TaskSupport_start__E
0082d160   ti_sysbios_family_c62_TaskSupport_swap__E
0086dbe8   ti_sysbios_family_c64p_EventCombiner_EVTMASK__C
0086de94   ti_sysbios_family_c64p_EventCombiner_E_unpluggedEvent__C
0086e188   ti_sysbios_family_c64p_EventCombiner_Module__id__C
0086eb28   ti_sysbios_family_c64p_EventCombiner_Module__state__V
008323c0   ti_sysbios_family_c64p_EventCombiner_Module_startup__E
0082ee40   ti_sysbios_family_c64p_EventCombiner_Module_startup__F
008304a0   ti_sysbios_family_c64p_EventCombiner_dispatchPlug__E
0082eea0   ti_sysbios_family_c64p_EventCombiner_dispatchPlug__F
008323e0   ti_sysbios_family_c64p_EventCombiner_dispatch__E
00829480   ti_sysbios_family_c64p_EventCombiner_dispatch__F
00832400   ti_sysbios_family_c64p_EventCombiner_enableEvent__E
008304e0   ti_sysbios_family_c64p_EventCombiner_enableEvent__F
00832420   ti_sysbios_family_c64p_EventCombiner_unused__E
0082ef00   ti_sysbios_family_c64p_EventCombiner_unused__F
0086de98   ti_sysbios_family_c64p_Exception_E_exceptionMin__C
0086e18c   ti_sysbios_family_c64p_Exception_Module__id__C
0086ef28   ti_sysbios_family_c64p_Exception_Module__state__V
00832440   ti_sysbios_family_c64p_Exception_Module_startup__E
0082d760   ti_sysbios_family_c64p_Exception_Module_startup__F
00825520   ti_sysbios_family_c64p_Exception_dispatch__E
0086de9c   ti_sysbios_family_c64p_Exception_exceptionHook__C
0086dea0   ti_sysbios_family_c64p_Exception_externalHook__C
0080d7c0   ti_sysbios_family_c64p_Exception_handler__I
00820240   ti_sysbios_family_c64p_Exception_internalHandler__I
0086dea4   ti_sysbios_family_c64p_Exception_internalHook__C
0086dea8   ti_sysbios_family_c64p_Exception_nmiHook__C
00871400   ti_sysbios_family_c64p_Hwi0
00871420   ti_sysbios_family_c64p_Hwi1
00871540   ti_sysbios_family_c64p_Hwi10
00871560   ti_sysbios_family_c64p_Hwi11
00871580   ti_sysbios_family_c64p_Hwi12
008715a0   ti_sysbios_family_c64p_Hwi13
008715c0   ti_sysbios_family_c64p_Hwi14
008715e0   ti_sysbios_family_c64p_Hwi15
00871440   ti_sysbios_family_c64p_Hwi2
00871460   ti_sysbios_family_c64p_Hwi3
00871480   ti_sysbios_family_c64p_Hwi4
008714a0   ti_sysbios_family_c64p_Hwi5
008714c0   ti_sysbios_family_c64p_Hwi6
008714e0   ti_sysbios_family_c64p_Hwi7
00871500   ti_sysbios_family_c64p_Hwi8
00871520   ti_sysbios_family_c64p_Hwi9
0086deac   ti_sysbios_family_c64p_Hwi_E_alreadyDefined__C
0086deb0   ti_sysbios_family_c64p_Hwi_E_handleNotFound__C
0082a380   ti_sysbios_family_c64p_Hwi_Instance_finalize__F
0082a460   ti_sysbios_family_c64p_Hwi_Instance_init__F
0086deb4   ti_sysbios_family_c64p_Hwi_LD_end__C
0086deb8   ti_sysbios_family_c64p_Hwi_LM_begin__C
0086debc   ti_sysbios_family_c64p_Hwi_Module__diagsEnabled__C
0086dec0   ti_sysbios_family_c64p_Hwi_Module__diagsIncluded__C
0086dec4   ti_sysbios_family_c64p_Hwi_Module__diagsMask__C
0086e190   ti_sysbios_family_c64p_Hwi_Module__id__C
0086e194   ti_sysbios_family_c64p_Hwi_Module__loggerDefined__C
0086dec8   ti_sysbios_family_c64p_Hwi_Module__loggerFxn1__C
0086decc   ti_sysbios_family_c64p_Hwi_Module__loggerFxn8__C
0086ded0   ti_sysbios_family_c64p_Hwi_Module__loggerObj__C
0086ef54   ti_sysbios_family_c64p_Hwi_Module__root__V
00830520   ti_sysbios_family_c64p_Hwi_Module__startupDone__F
00832460   ti_sysbios_family_c64p_Hwi_Module__startupDone__S
0086ef5c   ti_sysbios_family_c64p_Hwi_Module__state__V
00832480   ti_sysbios_family_c64p_Hwi_Module_startup__E
008276a0   ti_sysbios_family_c64p_Hwi_Module_startup__F
0086d884   ti_sysbios_family_c64p_Hwi_Object__DESC__C
0086d310   ti_sysbios_family_c64p_Hwi_Object__PARAMS__C
0082a540   ti_sysbios_family_c64p_Hwi_Object__create__S
00830560   ti_sysbios_family_c64p_Hwi_Object__delete__S
0086fc40   ti_sysbios_family_c64p_Hwi_Object__table__V
008305a0   ti_sysbios_family_c64p_Hwi_Params__init__S
008324a0   ti_sysbios_family_c64p_Hwi_clearInterrupt__E
008305e0   ti_sysbios_family_c64p_Hwi_disableInterrupt__E
00821b60   ti_sysbios_family_c64p_Hwi_dispatchAlways
0081b700   ti_sysbios_family_c64p_Hwi_dispatchC__I
00830620   ti_sysbios_family_c64p_Hwi_enableInterrupt__E
0082d7e0   ti_sysbios_family_c64p_Hwi_eventMap__E
008324c0   ti_sysbios_family_c64p_Hwi_getHandle__E
0082c740   ti_sysbios_family_c64p_Hwi_plug__E
008208e0   ti_sysbios_family_c64p_Hwi_reconfig__E
008324e0   ti_sysbios_family_c64p_Hwi_startup__E
00832500   ti_sysbios_family_c64p_Hwi_switchFromBootStack__E
00832520   ti_sysbios_family_c64p_Hwi_unPluggedInterrupt__I
00832540   ti_sysbios_family_c64p_tci6488_TimerSupport_enable__E
00832560   ti_sysbios_family_c66_Cache_Module_startup__E
008277e0   ti_sysbios_family_c66_Cache_Module_startup__F
0086ded4   ti_sysbios_family_c66_Cache_atomicBlockSize__C
0086dc08   ti_sysbios_family_c66_Cache_initSize__C
0082d860   ti_sysbios_family_c66_Cache_invL1pAll__E
00832580   ti_sysbios_family_c66_Cache_inv__E
0086c5e0   ti_sysbios_family_c66_Cache_marvalues__C
008325a0   ti_sysbios_family_c66_Cache_wbInv__E
0082f8a0   ti_sysbios_family_xxx_Hwi_switchToIsrStack
008317a0   ti_sysbios_family_xxx_Hwi_switchToTaskStack
00830660   ti_sysbios_gates_GateAll_Handle__label__S
008325c0   ti_sysbios_gates_GateAll_Instance_init__F
0086d578   ti_sysbios_gates_GateAll_Module__FXNS__C
0086efc4   ti_sysbios_gates_GateAll_Module__root__V
0086d8a4   ti_sysbios_gates_GateAll_Object__DESC__C
0086dad0   ti_sysbios_gates_GateAll_Object__PARAMS__C
0082d8e0   ti_sysbios_gates_GateAll_Object__create__S
008306a0   ti_sysbios_gates_GateAll_Object__delete__S
00870000   ti_sysbios_gates_GateAll_Object__table__V
0082ef60   ti_sysbios_gates_GateAll_enter__E
0082bae0   ti_sysbios_gates_GateAll_leave__E
008325e0   ti_sysbios_gates_GateAll_query__E
00832600   ti_sysbios_gates_GateAll_query__F
008306e0   ti_sysbios_gates_GateHwi_Handle__label__S
00832620   ti_sysbios_gates_GateHwi_Instance_init__F
0086d59c   ti_sysbios_gates_GateHwi_Module__FXNS__C
0086efcc   ti_sysbios_gates_GateHwi_Module__root__V
0086d8c4   ti_sysbios_gates_GateHwi_Object__DESC__C
0086dae8   ti_sysbios_gates_GateHwi_Object__PARAMS__C
0082d960   ti_sysbios_gates_GateHwi_Object__create__S
00830720   ti_sysbios_gates_GateHwi_Object__delete__S
00870088   ti_sysbios_gates_GateHwi_Object__table__V
00832640   ti_sysbios_gates_GateHwi_enter__E
00832660   ti_sysbios_gates_GateHwi_leave__E
00832680   ti_sysbios_gates_GateHwi_query__E
008326a0   ti_sysbios_gates_GateHwi_query__F
0086ded8   ti_sysbios_gates_GateMutexPri_A_badContext__C
00830760   ti_sysbios_gates_GateMutexPri_Handle__label__S
0086dedc   ti_sysbios_gates_GateMutexPri_Instance_State_pendQ__O
008307a0   ti_sysbios_gates_GateMutexPri_Instance_finalize__F
008307e0   ti_sysbios_gates_GateMutexPri_Instance_init__F
0086d5c0   ti_sysbios_gates_GateMutexPri_Module__FXNS__C
0086dee0   ti_sysbios_gates_GateMutexPri_Module__diagsEnabled__C
0086dee4   ti_sysbios_gates_GateMutexPri_Module__diagsIncluded__C
0086dee8   ti_sysbios_gates_GateMutexPri_Module__diagsMask__C
0086e198   ti_sysbios_gates_GateMutexPri_Module__id__C
0086efdc   ti_sysbios_gates_GateMutexPri_Module__root__V
0086d8e4   ti_sysbios_gates_GateMutexPri_Object__DESC__C
0086db00   ti_sysbios_gates_GateMutexPri_Object__PARAMS__C
0082d9e0   ti_sysbios_gates_GateMutexPri_Object__create__S
00830820   ti_sysbios_gates_GateMutexPri_Object__delete__S
00830860   ti_sysbios_gates_GateMutexPri_Object__destruct__S
0086ffc0   ti_sysbios_gates_GateMutexPri_Object__table__V
0081c580   ti_sysbios_gates_GateMutexPri_enter__E
00829580   ti_sysbios_gates_GateMutexPri_leave__E
008326c0   ti_sysbios_gates_GateMutexPri_query__E
008326e0   ti_sysbios_gates_GateMutexPri_query__F
0086deec   ti_sysbios_gates_GateMutex_A_badContext__C
008308a0   ti_sysbios_gates_GateMutex_Handle__label__S
0086def0   ti_sysbios_gates_GateMutex_Instance_State_sem__O
008308e0   ti_sysbios_gates_GateMutex_Instance_finalize__F
0082efc0   ti_sysbios_gates_GateMutex_Instance_init__F
0086d5e4   ti_sysbios_gates_GateMutex_Module__FXNS__C
0086def4   ti_sysbios_gates_GateMutex_Module__diagsEnabled__C
0086def8   ti_sysbios_gates_GateMutex_Module__diagsIncluded__C
0086defc   ti_sysbios_gates_GateMutex_Module__diagsMask__C
0086e19c   ti_sysbios_gates_GateMutex_Module__id__C
0086efd4   ti_sysbios_gates_GateMutex_Module__root__V
0086d904   ti_sysbios_gates_GateMutex_Object__DESC__C
0086db18   ti_sysbios_gates_GateMutex_Object__PARAMS__C
0082da60   ti_sysbios_gates_GateMutex_Object__create__S
00830920   ti_sysbios_gates_GateMutex_Object__delete__S
0086fe90   ti_sysbios_gates_GateMutex_Object__table__V
00824be0   ti_sysbios_gates_GateMutex_enter__E
00830960   ti_sysbios_gates_GateMutex_leave__E
00832700   ti_sysbios_gates_GateMutex_query__E
00832720   ti_sysbios_gates_GateMutex_query__F
0086df00   ti_sysbios_gates_GateSwi_A_badContext__C
008309a0   ti_sysbios_gates_GateSwi_Handle__label__S
00832740   ti_sysbios_gates_GateSwi_Instance_init__F
0086d608   ti_sysbios_gates_GateSwi_Module__FXNS__C
0086df04   ti_sysbios_gates_GateSwi_Module__diagsEnabled__C
0086df08   ti_sysbios_gates_GateSwi_Module__diagsIncluded__C
0086df0c   ti_sysbios_gates_GateSwi_Module__diagsMask__C
0086e1a0   ti_sysbios_gates_GateSwi_Module__id__C
0086efe4   ti_sysbios_gates_GateSwi_Module__root__V
0086d924   ti_sysbios_gates_GateSwi_Object__DESC__C
0086db30   ti_sysbios_gates_GateSwi_Object__PARAMS__C
0082dae0   ti_sysbios_gates_GateSwi_Object__create__S
008309e0   ti_sysbios_gates_GateSwi_Object__delete__S
00870020   ti_sysbios_gates_GateSwi_Object__table__V
00827920   ti_sysbios_gates_GateSwi_enter__E
0082db60   ti_sysbios_gates_GateSwi_leave__E
00832760   ti_sysbios_gates_GateSwi_query__E
00832780   ti_sysbios_gates_GateSwi_query__F
00830a20   ti_sysbios_hal_Cache_CacheProxy_inv__E
00830a60   ti_sysbios_hal_Cache_CacheProxy_wbInv__E
00830a20   ti_sysbios_hal_Cache_inv__E
00830a60   ti_sysbios_hal_Cache_wbInv__E
0086df10   ti_sysbios_hal_Hwi_E_stackOverflow__C
008327a0   ti_sysbios_hal_Hwi_HwiProxy_Module__startupDone__S
008327c0   ti_sysbios_hal_Hwi_HwiProxy_clearInterrupt__E
008327e0   ti_sysbios_hal_Hwi_HwiProxy_disableInterrupt__E
00832800   ti_sysbios_hal_Hwi_HwiProxy_enableInterrupt__E
00832820   ti_sysbios_hal_Hwi_HwiProxy_startup__E
00832840   ti_sysbios_hal_Hwi_HwiProxy_switchFromBootStack__E
0086e1a4   ti_sysbios_hal_Hwi_Module__id__C
0086efec   ti_sysbios_hal_Hwi_Module__root__V
00832860   ti_sysbios_hal_Hwi_Module_startup__E
00832880   ti_sysbios_hal_Hwi_Module_startup__F
00870030   ti_sysbios_hal_Hwi_Object__table__V
0082dbe0   ti_sysbios_hal_Hwi_checkStack
008327c0   ti_sysbios_hal_Hwi_clearInterrupt__E
008327e0   ti_sysbios_hal_Hwi_disableInterrupt__E
00832800   ti_sysbios_hal_Hwi_enableInterrupt__E
0082f020   ti_sysbios_hal_Hwi_initStack
00832820   ti_sysbios_hal_Hwi_startup__E
00832840   ti_sysbios_hal_Hwi_switchFromBootStack__E
0086eff4   ti_sysbios_hal_Timer_Module__root__V
00830aa0   ti_sysbios_hal_Timer_Module__startupDone__F
008328a0   ti_sysbios_hal_Timer_Module__startupDone__S
008328c0   ti_sysbios_hal_Timer_Module_startup__E
008328e0   ti_sysbios_hal_Timer_Module_startup__F
00870038   ti_sysbios_hal_Timer_Object__table__V
00832900   ti_sysbios_hal_Timer_TimerProxy_Module__startupDone__S
00832920   ti_sysbios_hal_Timer_TimerProxy_getExpiredCounts__E
00832940   ti_sysbios_hal_Timer_TimerProxy_getPeriod__E
00832960   ti_sysbios_hal_Timer_TimerProxy_setNextTick__E
00832980   ti_sysbios_hal_Timer_TimerProxy_startup__E
00832980   ti_sysbios_hal_Timer_startup__E
0086df14   ti_sysbios_heaps_HeapBuf_Instance_State_freeList__O
0086effc   ti_sysbios_heaps_HeapBuf_Module__root__V
0086f004   ti_sysbios_heaps_HeapBuf_Module__state__V
008329a0   ti_sysbios_heaps_HeapBuf_Module_startup__E
00825ca0   ti_sysbios_heaps_HeapBuf_Module_startup__F
0086df18   ti_sysbios_heaps_HeapBuf_Object__count__C
0082f080   ti_sysbios_heaps_HeapBuf_Object__get__S
0086df1c   ti_sysbios_heaps_HeapBuf_Object__table__C
0086df20   ti_sysbios_heaps_HeapBuf_numConstructedHeaps__C
0086df24   ti_sysbios_heaps_HeapMem_A_align__C
0086df28   ti_sysbios_heaps_HeapMem_A_heapSize__C
0086df2c   ti_sysbios_heaps_HeapMem_A_invalidFree__C
0086df30   ti_sysbios_heaps_HeapMem_A_zeroBlock__C
0086df34   ti_sysbios_heaps_HeapMem_E_memory__C
00830ae0   ti_sysbios_heaps_HeapMem_Handle__label__S
008334c0   ti_sysbios_heaps_HeapMem_Instance_State_0_buf__A
00825e20   ti_sysbios_heaps_HeapMem_Instance_init__F
008329c0   ti_sysbios_heaps_HeapMem_Module_GateProxy_enter__E
008329e0   ti_sysbios_heaps_HeapMem_Module_GateProxy_leave__E
00832a00   ti_sysbios_heaps_HeapMem_Module_GateProxy_query__E
0086d4bc   ti_sysbios_heaps_HeapMem_Module__FXNS__C
0086df38   ti_sysbios_heaps_HeapMem_Module__diagsEnabled__C
0086df3c   ti_sysbios_heaps_HeapMem_Module__diagsIncluded__C
0086df40   ti_sysbios_heaps_HeapMem_Module__diagsMask__C
0086df44   ti_sysbios_heaps_HeapMem_Module__gateObj__C
0086e1a8   ti_sysbios_heaps_HeapMem_Module__id__C
0086f008   ti_sysbios_heaps_HeapMem_Module__root__V
0086d944   ti_sysbios_heaps_HeapMem_Object__DESC__C
0086d964   ti_sysbios_heaps_HeapMem_Object__PARAMS__C
0086df48   ti_sysbios_heaps_HeapMem_Object__count__C
0082dc60   ti_sysbios_heaps_HeapMem_Object__create__S
00830b20   ti_sysbios_heaps_HeapMem_Object__delete__S
0082f0e0   ti_sysbios_heaps_HeapMem_Object__get__S
0086df4c   ti_sysbios_heaps_HeapMem_Object__table__C
0086ffd8   ti_sysbios_heaps_HeapMem_Object__table__V
00810de0   ti_sysbios_heaps_HeapMem_alloc__E
00810160   ti_sysbios_heaps_HeapMem_free__E
0082bba0   ti_sysbios_heaps_HeapMem_getStats__E
0082cd80   ti_sysbios_heaps_HeapMem_init__I
00832a20   ti_sysbios_heaps_HeapMem_isBlocking__E
0086df50   ti_sysbios_heaps_HeapMem_reqAlignMask__C
0086df54   ti_sysbios_heaps_HeapMem_reqAlign__C
0086df58   ti_sysbios_knl_Clock_A_badThreadType__C
00827a60   ti_sysbios_knl_Clock_Instance_finalize__F
0081e7e0   ti_sysbios_knl_Clock_Instance_init__F
0086df5c   ti_sysbios_knl_Clock_LM_begin__C
0086df60   ti_sysbios_knl_Clock_LM_tick__C
0086df64   ti_sysbios_knl_Clock_LW_delayed__C
0086df68   ti_sysbios_knl_Clock_Module_State_clockQ__O
0086df6c   ti_sysbios_knl_Clock_Module__diagsEnabled__C
0086df70   ti_sysbios_knl_Clock_Module__diagsIncluded__C
0086df74   ti_sysbios_knl_Clock_Module__diagsMask__C
0086e1ac   ti_sysbios_knl_Clock_Module__id__C
0086e1b0   ti_sysbios_knl_Clock_Module__loggerDefined__C
0086df78   ti_sysbios_knl_Clock_Module__loggerFxn1__C
0086df7c   ti_sysbios_knl_Clock_Module__loggerFxn2__C
0086df80   ti_sysbios_knl_Clock_Module__loggerObj__C
0086f010   ti_sysbios_knl_Clock_Module__root__V
0086f018   ti_sysbios_knl_Clock_Module__state__V
00832a60   ti_sysbios_knl_Clock_Module_startup__E
0082dce0   ti_sysbios_knl_Clock_Module_startup__F
0086d984   ti_sysbios_knl_Clock_Object__DESC__C
0086d62c   ti_sysbios_knl_Clock_Object__PARAMS__C
0082dd60   ti_sysbios_knl_Clock_Object__create__S
00830b60   ti_sysbios_knl_Clock_Object__destruct__S
00830ba0   ti_sysbios_knl_Clock_Params__init__S
0082f140   ti_sysbios_knl_Clock_doTick__I
0082dde0   ti_sysbios_knl_Clock_getTicks__E
0082bc60   ti_sysbios_knl_Clock_logTick__E
00829680   ti_sysbios_knl_Clock_startI__E
0082a620   ti_sysbios_knl_Clock_start__E
0086df84   ti_sysbios_knl_Clock_tickMode__C
0086df88   ti_sysbios_knl_Clock_tickSource__C
0081d8c0   ti_sysbios_knl_Clock_workFunc__E
0086df90   ti_sysbios_knl_Idle_funcList__A
0086dc1c   ti_sysbios_knl_Idle_funcList__C
0082de60   ti_sysbios_knl_Idle_loop__E
00832a80   ti_sysbios_knl_Queue_Instance_init__F
0086f044   ti_sysbios_knl_Queue_Module__root__V
0086d9a4   ti_sysbios_knl_Queue_Object__DESC__C
0086db48   ti_sysbios_knl_Queue_Object__PARAMS__C
0086df8c   ti_sysbios_knl_Queue_Object__count__C
0082dee0   ti_sysbios_knl_Queue_Object__create__S
00830be0   ti_sysbios_knl_Queue_Object__destruct__S
0082f1a0   ti_sysbios_knl_Queue_Object__get__S
0086df94   ti_sysbios_knl_Queue_Object__table__C
00832aa0   ti_sysbios_knl_Queue_empty__E
0086df98   ti_sysbios_knl_Semaphore_A_badContext__C
0086df9c   ti_sysbios_knl_Semaphore_A_noEvents__C
0086dfa0   ti_sysbios_knl_Semaphore_A_overflow__C
0086dfa4   ti_sysbios_knl_Semaphore_Instance_State_pendQ__O
00830c20   ti_sysbios_knl_Semaphore_Instance_finalize__F
00827ba0   ti_sysbios_knl_Semaphore_Instance_init__F
0086dfa8   ti_sysbios_knl_Semaphore_LM_pend__C
0086dfac   ti_sysbios_knl_Semaphore_LM_post__C
0086dfb0   ti_sysbios_knl_Semaphore_Module__diagsEnabled__C
0086dfb4   ti_sysbios_knl_Semaphore_Module__diagsIncluded__C
0086dfb8   ti_sysbios_knl_Semaphore_Module__diagsMask__C
0086e1b4   ti_sysbios_knl_Semaphore_Module__id__C
0086e1b8   ti_sysbios_knl_Semaphore_Module__loggerDefined__C
0086dfbc   ti_sysbios_knl_Semaphore_Module__loggerFxn2__C
0086dfc0   ti_sysbios_knl_Semaphore_Module__loggerFxn4__C
0086dfc4   ti_sysbios_knl_Semaphore_Module__loggerObj__C
0086f04c   ti_sysbios_knl_Semaphore_Module__root__V
0086d9c4   ti_sysbios_knl_Semaphore_Object__DESC__C
0086d650   ti_sysbios_knl_Semaphore_Object__PARAMS__C
0082df60   ti_sysbios_knl_Semaphore_Object__create__S
00830c60   ti_sysbios_knl_Semaphore_Object__delete__S
00830ca0   ti_sysbios_knl_Semaphore_Object__destruct__S
00830ce0   ti_sysbios_knl_Semaphore_Params__init__S
0082dfe0   ti_sysbios_knl_Semaphore_pendTimeout__I
00818200   ti_sysbios_knl_Semaphore_pend__E
00820480   ti_sysbios_knl_Semaphore_post__E
0086dfc8   ti_sysbios_knl_Swi_A_badPriority__C
0082bd20   ti_sysbios_knl_Swi_Instance_finalize__F
008239a0   ti_sysbios_knl_Swi_Instance_init__F
0086dfcc   ti_sysbios_knl_Swi_LD_end__C
0086dfd0   ti_sysbios_knl_Swi_LM_begin__C
0086dfd4   ti_sysbios_knl_Swi_LM_post__C
0086f8d0   ti_sysbios_knl_Swi_Module_State_0_readyQ__A
0086dfd8   ti_sysbios_knl_Swi_Module__diagsEnabled__C
0086dfdc   ti_sysbios_knl_Swi_Module__diagsIncluded__C
0086dfe0   ti_sysbios_knl_Swi_Module__diagsMask__C
0086e1bc   ti_sysbios_knl_Swi_Module__id__C
0086e1c0   ti_sysbios_knl_Swi_Module__loggerDefined__C
0086dfe4   ti_sysbios_knl_Swi_Module__loggerFxn1__C
0086dfe8   ti_sysbios_knl_Swi_Module__loggerFxn4__C
0086dfec   ti_sysbios_knl_Swi_Module__loggerObj__C
0086f054   ti_sysbios_knl_Swi_Module__root__V
0086f05c   ti_sysbios_knl_Swi_Module__state__V
00832ac0   ti_sysbios_knl_Swi_Module_startup__E
0082f200   ti_sysbios_knl_Swi_Module_startup__F
0086d9e4   ti_sysbios_knl_Swi_Object__DESC__C
0086d4e4   ti_sysbios_knl_Swi_Object__PARAMS__C
0086dff0   ti_sysbios_knl_Swi_Object__count__C
0082bde0   ti_sysbios_knl_Swi_Object__create__S
00830d20   ti_sysbios_knl_Swi_Object__destruct__S
0082f260   ti_sysbios_knl_Swi_Object__get__S
0086dff4   ti_sysbios_knl_Swi_Object__table__C
0086fed0   ti_sysbios_knl_Swi_Object__table__V
00830d60   ti_sysbios_knl_Swi_Params__init__S
00832ae0   ti_sysbios_knl_Swi_disable__E
00827ce0   ti_sysbios_knl_Swi_post__E
00829780   ti_sysbios_knl_Swi_restoreHwi__E
00820b00   ti_sysbios_knl_Swi_run__I
00825fa0   ti_sysbios_knl_Swi_schedule__I
0082e060   ti_sysbios_knl_Swi_startup__E
0086dff8   ti_sysbios_knl_Task_A_badPriority__C
0086dffc   ti_sysbios_knl_Task_A_badTaskState__C
0086e000   ti_sysbios_knl_Task_A_badThreadType__C
0086e004   ti_sysbios_knl_Task_A_noPendElem__C
0086e008   ti_sysbios_knl_Task_E_spOutOfBounds__C
0086e00c   ti_sysbios_knl_Task_E_stackOverflow__C
008690d8   ti_sysbios_knl_Task_Instance_State_0_hookEnv__A
008682a0   ti_sysbios_knl_Task_Instance_State_0_stack__A
00814ca0   ti_sysbios_knl_Task_Instance_finalize__F
00819540   ti_sysbios_knl_Task_Instance_init__F
0086e010   ti_sysbios_knl_Task_LD_block__C
0086e014   ti_sysbios_knl_Task_LD_exit__C
0086e018   ti_sysbios_knl_Task_LD_ready__C
0086e01c   ti_sysbios_knl_Task_LM_setPri__C
0086e020   ti_sysbios_knl_Task_LM_switch__C
0086e024   ti_sysbios_knl_Task_LM_yield__C
0086f950   ti_sysbios_knl_Task_Module_State_0_readyQ__A
0086e028   ti_sysbios_knl_Task_Module_State_inactiveQ__O
0086e02c   ti_sysbios_knl_Task_Module_State_terminatedQ__O
0086e030   ti_sysbios_knl_Task_Module__diagsEnabled__C
0086e034   ti_sysbios_knl_Task_Module__diagsIncluded__C
0086e038   ti_sysbios_knl_Task_Module__diagsMask__C
0086e1c4   ti_sysbios_knl_Task_Module__id__C
0086e1c8   ti_sysbios_knl_Task_Module__loggerDefined__C
0086e03c   ti_sysbios_knl_Task_Module__loggerFxn2__C
0086e040   ti_sysbios_knl_Task_Module__loggerFxn4__C
0086e044   ti_sysbios_knl_Task_Module__loggerObj__C
0086f078   ti_sysbios_knl_Task_Module__root__V
0086f080   ti_sysbios_knl_Task_Module__state__V
00832b00   ti_sysbios_knl_Task_Module_startup__E
0081c860   ti_sysbios_knl_Task_Module_startup__F
0086da04   ti_sysbios_knl_Task_Object__DESC__C
0086d204   ti_sysbios_knl_Task_Object__PARAMS__C
0086e048   ti_sysbios_knl_Task_Object__count__C
0082bea0   ti_sysbios_knl_Task_Object__create__S
00830da0   ti_sysbios_knl_Task_Object__first__S
0082f2c0   ti_sysbios_knl_Task_Object__get__S
0086e04c   ti_sysbios_knl_Task_Object__heap__C
00830de0   ti_sysbios_knl_Task_Object__next__S
0086e050   ti_sysbios_knl_Task_Object__table__C
0086fd08   ti_sysbios_knl_Task_Object__table__V
00830e20   ti_sysbios_knl_Task_Params__init__S
00832b20   ti_sysbios_knl_Task_SupportProxy_Module__startupDone__S
00832b40   ti_sysbios_knl_Task_SupportProxy_checkStack__E
00832b60   ti_sysbios_knl_Task_SupportProxy_getStackAlignment__E
00832b80   ti_sysbios_knl_Task_SupportProxy_start__E
00832ba0   ti_sysbios_knl_Task_SupportProxy_swap__E
0086e054   ti_sysbios_knl_Task_allBlockedFunc__C
0082f320   ti_sysbios_knl_Task_allBlockedFunction__I
00827e20   ti_sysbios_knl_Task_blockI__E
00823b60   ti_sysbios_knl_Task_checkStacks__E
0086e058   ti_sysbios_knl_Task_defaultStackHeap__C
0086e05c   ti_sysbios_knl_Task_defaultStackSize__C
0086e1cc   ti_sysbios_knl_Task_deleteTerminatedTasks__C
00832bc0   ti_sysbios_knl_Task_disable__E
0082f380   ti_sysbios_knl_Task_enter__I
0081ea60   ti_sysbios_knl_Task_exit__E
00832be0   ti_sysbios_knl_Task_getPri__E
0086db60   ti_sysbios_knl_Task_hooks__A
0086dc24   ti_sysbios_knl_Task_hooks__C
0086e1d0   ti_sysbios_knl_Task_initStackFlag__C
0086e060   ti_sysbios_knl_Task_numConstructedTasks__C
0086e064   ti_sysbios_knl_Task_numPriorities__C
00822d20   ti_sysbios_knl_Task_postInit__I
0082e0e0   ti_sysbios_knl_Task_restore__E
00820d20   ti_sysbios_knl_Task_schedule__I
00832c00   ti_sysbios_knl_Task_self__E
00819900   ti_sysbios_knl_Task_setPri__E
00820f40   ti_sysbios_knl_Task_startup__E
00826120   ti_sysbios_knl_Task_unblockI__E
00827f60   ti_sysbios_knl_Task_yield__E
0086f0b4   ti_sysbios_syncs_SyncSem_Module__root__V
0086e068   ti_sysbios_timers_timer64_Timer_A_notAvailable__C
0086e06c   ti_sysbios_timers_timer64_Timer_E_cannotSupport__C
0086f300   ti_sysbios_timers_timer64_Timer_Module_State_0_device__A
0086f9d0   ti_sysbios_timers_timer64_Timer_Module_State_0_gctrl__A
0086fa50   ti_sysbios_timers_timer64_Timer_Module_State_0_handles__A
0086fad0   ti_sysbios_timers_timer64_Timer_Module_State_0_intFreqs__A
0086e070   ti_sysbios_timers_timer64_Timer_Module__diagsEnabled__C
0086e074   ti_sysbios_timers_timer64_Timer_Module__diagsIncluded__C
0086e078   ti_sysbios_timers_timer64_Timer_Module__diagsMask__C
0086e1d4   ti_sysbios_timers_timer64_Timer_Module__id__C
0086f0bc   ti_sysbios_timers_timer64_Timer_Module__root__V
00830e60   ti_sysbios_timers_timer64_Timer_Module__startupDone__F
00832c20   ti_sysbios_timers_timer64_Timer_Module__startupDone__S
0086f0c4   ti_sysbios_timers_timer64_Timer_Module__state__V
00832c40   ti_sysbios_timers_timer64_Timer_Module_startup__E
008136a0   ti_sysbios_timers_timer64_Timer_Module_startup__F
0086fcb8   ti_sysbios_timers_timer64_Timer_Object__table__V
00832c60   ti_sysbios_timers_timer64_Timer_TimerSupportProxy_enable__E
0086e07c   ti_sysbios_timers_timer64_Timer_anyMask__C
0086e080   ti_sysbios_timers_timer64_Timer_freqDivisor__C
0082e160   ti_sysbios_timers_timer64_Timer_getCount__E
0082e160   ti_sysbios_timers_timer64_Timer_getExpiredCounts__E
00822f00   ti_sysbios_timers_timer64_Timer_getFreq__E
0082e1e0   ti_sysbios_timers_timer64_Timer_getPeriod__E
0086e084   ti_sysbios_timers_timer64_Timer_numLocalTimers__C
0086e088   ti_sysbios_timers_timer64_Timer_numTimerDevices__C
00832c80   ti_sysbios_timers_timer64_Timer_setNextTick__E
00823d20   ti_sysbios_timers_timer64_Timer_setPeriodMicroSecs__E
00824d80   ti_sysbios_timers_timer64_Timer_start__E
0086e1d8   ti_sysbios_timers_timer64_Timer_startupNeeded__C
0082a700   ti_sysbios_timers_timer64_Timer_startup__E
0082bf60   ti_sysbios_timers_timer64_Timer_stop__E
008326c0   ti_sysbios_xdcruntime_GateProcessSupport_query__F
0086e08c   ti_sysbios_xdcruntime_GateThreadSupport_Instance_State_gate__O
00830ea0   ti_sysbios_xdcruntime_GateThreadSupport_Instance_finalize__F
00830ee0   ti_sysbios_xdcruntime_GateThreadSupport_Instance_init__F
0086f0d8   ti_sysbios_xdcruntime_GateThreadSupport_Module__root__V
0086da24   ti_sysbios_xdcruntime_GateThreadSupport_Object__DESC__C
0086db78   ti_sysbios_xdcruntime_GateThreadSupport_Object__PARAMS__C
0082e260   ti_sysbios_xdcruntime_GateThreadSupport_Object__create__S
00830f20   ti_sysbios_xdcruntime_GateThreadSupport_Object__delete__S
00832ca0   ti_sysbios_xdcruntime_GateThreadSupport_enter__E
00830f60   ti_sysbios_xdcruntime_GateThreadSupport_enter__F
00832cc0   ti_sysbios_xdcruntime_GateThreadSupport_leave__E
00830fa0   ti_sysbios_xdcruntime_GateThreadSupport_leave__F
00832ce0   ti_sysbios_xdcruntime_GateThreadSupport_query__E
008326c0   ti_sysbios_xdcruntime_GateThreadSupport_query__F
00830fe0   time
00868b2c   to
80011f80   twiddle_1024
80011180   twiddle_128
80011380   twiddle_256
80011000   twiddle_32
80011780   twiddle_512
80011080   twiddle_64
008711d0   txData_char
008711cc   txData_int
0082e2e0   unlink
0082ce20   write
0082f3e0   writemsg
00871210   x1
0087120c   x_min
80000000   x_ref_float
80007000   x_short
0086e090   xdc_runtime_Assert_E_assertFailed__C
0082cec0   xdc_runtime_Assert_raise__I
0086e094   xdc_runtime_Core_A_initializedParams__C
0086e098   xdc_runtime_Core_Module__diagsEnabled__C
0086e09c   xdc_runtime_Core_Module__diagsIncluded__C
0086e0a0   xdc_runtime_Core_Module__diagsMask__C
0086e1dc   xdc_runtime_Core_Module__id__C
0082e360   xdc_runtime_Core_assignLabel__I
0082e3e0   xdc_runtime_Core_assignParams__I
0081ece0   xdc_runtime_Core_createObject__I
00829880   xdc_runtime_Core_deleteObject__I
0086e0a4   xdc_runtime_Error_E_generic__C
0086e0a8   xdc_runtime_Error_E_memory__C
0086e0ac   xdc_runtime_Error_Module__diagsEnabled__C
0086e0b0   xdc_runtime_Error_Module__diagsIncluded__C
0086e0b4   xdc_runtime_Error_Module__diagsMask__C
0086e1e0   xdc_runtime_Error_Module__loggerDefined__C
0086e0b8   xdc_runtime_Error_Module__loggerFxn8__C
0086e0bc   xdc_runtime_Error_Module__loggerObj__C
0086f0e0   xdc_runtime_Error_Module__state__V
00832d20   xdc_runtime_Error_check__E
00831020   xdc_runtime_Error_check__F
00832d40   xdc_runtime_Error_init__E
00831060   xdc_runtime_Error_init__F
0086e1e4   xdc_runtime_Error_maxDepth__C
0086e0c0   xdc_runtime_Error_policy__C
00832d60   xdc_runtime_Error_print__E
0082a7e0   xdc_runtime_Error_print__F
0086e0c4   xdc_runtime_Error_raiseHook__C
008310a0   xdc_runtime_Error_raiseX__E
0081ef60   xdc_runtime_Error_raiseX__F
008310e0   xdc_runtime_GateNull_Handle__label__S
0086d674   xdc_runtime_GateNull_Module__FXNS__C
0086f0e4   xdc_runtime_GateNull_Module__root__V
0086da44   xdc_runtime_GateNull_Object__DESC__C
0086db90   xdc_runtime_GateNull_Object__PARAMS__C
0082f440   xdc_runtime_GateNull_Object__create__S
00831120   xdc_runtime_GateNull_Object__delete__S
00870090   xdc_runtime_GateNull_Object__table__V
00832d80   xdc_runtime_GateNull_enter__E
00832da0   xdc_runtime_GateNull_enter__F
00832dc0   xdc_runtime_GateNull_leave__E
00832de0   xdc_runtime_GateNull_leave__F
00832e00   xdc_runtime_GateNull_query__E
00832e20   xdc_runtime_GateNull_query__F
00832e40   xdc_runtime_Gate_enterSystem__E
00832e60   xdc_runtime_Gate_enterSystem__F
00832e80   xdc_runtime_Gate_leaveSystem__E
00831160   xdc_runtime_Gate_leaveSystem__F
0086e0c8   xdc_runtime_IGateProvider_Interface__BASE__C
0086e0cc   xdc_runtime_IHeap_Interface__BASE__C
0086e0d0   xdc_runtime_IModule_Interface__BASE__C
0086e0d4   xdc_runtime_Log_L_error__C
00832ea0   xdc_runtime_Memory_HeapProxy_alloc__E
00832ec0   xdc_runtime_Memory_HeapProxy_free__E
0086e1e8   xdc_runtime_Memory_Module__id__C
0086f0ec   xdc_runtime_Memory_Module__state__V
00832ee0   xdc_runtime_Memory_alloc__E
0082a8c0   xdc_runtime_Memory_alloc__F
00832f00   xdc_runtime_Memory_calloc__E
0082f4a0   xdc_runtime_Memory_calloc__F
0086e0d8   xdc_runtime_Memory_defaultHeapInstance__C
00832f20   xdc_runtime_Memory_free__E
00831220   xdc_runtime_Memory_free__F
00832f40   xdc_runtime_Memory_getMaxDefaultTypeAlign__E
00832f60   xdc_runtime_Memory_getMaxDefaultTypeAlign__F
00831260   xdc_runtime_Memory_valloc__E
0082f500   xdc_runtime_Memory_valloc__F
0086f0f0   xdc_runtime_Registry_Module__state__V
00832f80   xdc_runtime_Registry_findById__E
008312a0   xdc_runtime_Registry_findById__F
00832fa0   xdc_runtime_Startup_Module__startupDone__S
0086f0f8   xdc_runtime_Startup_Module__state__V
00000001   xdc_runtime_Startup__EXECFXN__C
00000001   xdc_runtime_Startup__RESETFXN__C
0086e0dc   xdc_runtime_Startup_execImpl__C
00832fc0   xdc_runtime_Startup_exec__E
00829980   xdc_runtime_Startup_exec__F
008312e0   xdc_runtime_Startup_exec__I
0086dbf8   xdc_runtime_Startup_firstFxns__A
0086dc2c   xdc_runtime_Startup_firstFxns__C
0086e0e0   xdc_runtime_Startup_lastFxns__A
0086dc34   xdc_runtime_Startup_lastFxns__C
0086e0e4   xdc_runtime_Startup_maxPasses__C
00832fe0   xdc_runtime_Startup_reset__I
00833000   xdc_runtime_Startup_rtsDone__E
00833020   xdc_runtime_Startup_rtsDone__F
0086d6c0   xdc_runtime_Startup_sfxnRts__A
0086e0e8   xdc_runtime_Startup_sfxnRts__C
0086d150   xdc_runtime_Startup_sfxnTab__A
0086e0ec   xdc_runtime_Startup_sfxnTab__C
0086e0f0   xdc_runtime_Startup_startModsFxn__C
0081fb60   xdc_runtime_Startup_startMods__I
00833040   xdc_runtime_SysStd_abort__E
0082f560   xdc_runtime_SysStd_abort__F
00833060   xdc_runtime_SysStd_exit__E
00833080   xdc_runtime_SysStd_exit__F
008330a0   xdc_runtime_SysStd_putch__E
008330c0   xdc_runtime_SysStd_putch__F
008330e0   xdc_runtime_SysStd_ready__E
00833100   xdc_runtime_SysStd_ready__F
00833120   xdc_runtime_System_Module_GateProxy_enter__E
00833140   xdc_runtime_System_Module_GateProxy_leave__E
0086ffa0   xdc_runtime_System_Module_State_0_atexitHandlers__A
0086e0f4   xdc_runtime_System_Module__gateObj__C
0086f100   xdc_runtime_System_Module__state__V
00833160   xdc_runtime_System_Module_startup__E
00833180   xdc_runtime_System_Module_startup__F
008331a0   xdc_runtime_System_SupportProxy_abort__E
008331c0   xdc_runtime_System_SupportProxy_exit__E
008331e0   xdc_runtime_System_SupportProxy_putch__E
00833200   xdc_runtime_System_SupportProxy_ready__E
00833220   xdc_runtime_System_abort__E
00831320   xdc_runtime_System_abort__F
00831360   xdc_runtime_System_aprintf__E
0082f5c0   xdc_runtime_System_aprintf_va__F
00833240   xdc_runtime_System_atexit__E
0082e460   xdc_runtime_System_atexit__F
0082f5c0   xdc_runtime_System_avprintf__F
00809c60   xdc_runtime_System_doPrint__I
00833260   xdc_runtime_System_exit__E
00833280   xdc_runtime_System_exit__F
0086e0f8   xdc_runtime_System_extendFxn__C
0082c020   xdc_runtime_System_formatNum__I
008332a0   xdc_runtime_System_lastFxn__I
0086e0fc   xdc_runtime_System_maxAtexitHandlers__C
0081a3e0   xdc_runtime_System_printfExtend__I
008313a0   xdc_runtime_System_printf__E
0082f620   xdc_runtime_System_printf_va__F
0082e4e0   xdc_runtime_System_rtsExit__I
008332e0   xdc_runtime_System_sprintf_va__F
0082f620   xdc_runtime_System_vprintf__F
008332c0   xdc_runtime_System_vsprintf__E
008332e0   xdc_runtime_System_vsprintf__F
0086f10c   xdc_runtime_Text_Module__state__V
0086e1ec   xdc_runtime_Text_charCnt__C
008690f0   xdc_runtime_Text_charTab__A
0086e100   xdc_runtime_Text_charTab__C
00833300   xdc_runtime_Text_cordText__E
0082f680   xdc_runtime_Text_cordText__F
0086e1f0   xdc_runtime_Text_isLoaded__C
0086e104   xdc_runtime_Text_nameEmpty__C
0086e108   xdc_runtime_Text_nameStatic__C
0086e10c   xdc_runtime_Text_nameUnknown__C
0086cc08   xdc_runtime_Text_nodeTab__A
0086e110   xdc_runtime_Text_nodeTab__C
0082e560   xdc_runtime_Text_printVisFxn__I
00833320   xdc_runtime_Text_putLab__E
00828760   xdc_runtime_Text_putLab__F
00829a80   xdc_runtime_Text_putMod__F
00833340   xdc_runtime_Text_putSite__E
008262a0   xdc_runtime_Text_putSite__F
0086e1f4   xdc_runtime_Text_registryModsLastId__C
00833360   xdc_runtime_Text_ropeText__E
008313e0   xdc_runtime_Text_ropeText__F
0086e1f8   xdc_runtime_Text_unnamedModsLastId__C
00829b80   xdc_runtime_Text_visitRope2__I
0086e114   xdc_runtime_Text_visitRopeFxn__C
00831420   xdc_runtime_Text_visitRope__I
0082e5e0   xdc_runtime_Text_xprintf__I
00831460   xdc_runtime_knl_GateThread_Handle__label__S
008314a0   xdc_runtime_knl_GateThread_Instance_finalize__F
008314e0   xdc_runtime_knl_GateThread_Instance_init__F
0086d698   xdc_runtime_knl_GateThread_Module__FXNS__C
0086f114   xdc_runtime_knl_GateThread_Module__root__V
00833380   xdc_runtime_knl_GateThread_Module__startupDone__S
0086da64   xdc_runtime_knl_GateThread_Object__DESC__C
0086dba8   xdc_runtime_knl_GateThread_Object__PARAMS__C
0082c0e0   xdc_runtime_knl_GateThread_Object__create__S
00831520   xdc_runtime_knl_GateThread_Object__delete__S
00831560   xdc_runtime_knl_GateThread_Proxy_Object__create__S
008333a0   xdc_runtime_knl_GateThread_Proxy_Object__delete__S
008333c0   xdc_runtime_knl_GateThread_Proxy_enter__E
008333e0   xdc_runtime_knl_GateThread_Proxy_leave__E
00833400   xdc_runtime_knl_GateThread_Proxy_query__E
00833420   xdc_runtime_knl_GateThread_enter__E
00833440   xdc_runtime_knl_GateThread_enter__F
00833460   xdc_runtime_knl_GateThread_leave__E
00833480   xdc_runtime_knl_GateThread_leave__F
008334a0   xdc_runtime_knl_GateThread_query__E
00833400   xdc_runtime_knl_GateThread_query__F
00871200   xx
00863500   xxx
80005000   y_short
80001000   z_short


GLOBAL SYMBOLS: SORTED BY Symbol Address 

address    name
--------   ----
00000000   _argsize
00000001   __TI_args_main
00000001   xdc_runtime_Startup__EXECFXN__C
00000001   xdc_runtime_Startup__RESETFXN__C
00001000   __TI_STACK_SIZE
00800000   __ASM__
00800070   __ISA__
00800088   __PLAT__
008000b0   __TARG__
008000d8   __TRDR__
00801260   Srio_processReceivedBD
00801748   Srio_rxCompletionIsr
008018b0   Srio_dioCompletionIsr
00801b90   Srio_init
00802870   Srio_start
00802acc   Srio_sockOpen
008030c4   Srio_sockBind
008037f0   Srio_allocTransmitBuffer
00803834   Srio_freeTransmitBuffer
00803868   Srio_sockSend
00803eb0   Srio_sockRecv
00803f94   Srio_freeRxDrvBuffer
00803fe0   Srio_setSockOpt
008040d8   Srio_getSockOpt
008041e4   Srio_sockClose
00804584   Srio_getVersion
00804590   Srio_getVersionStr
00806100   ti_sdo_ipc_GateMP_Instance_init__F
00807548   enable_srio
00807588   system_init
008076d8   masterTaskInitialization
00807994   slaveTaskInitialization
00807c78   initializeMain
00807e80   ti_sdo_ipc_heaps_HeapMemMP_alloc__E
008088e0   ti_sdo_ipc_heaps_HeapMemMP_free__E
008092c0   Ipc_attach
00809c60   xdc_runtime_System_doPrint__I
0080a600   ti_sdo_ipc_transports_TransportShm_Instance_init__F
0080af20   ti_sdo_ipc_ListMP_Instance_init__F
0080b7c0   ti_sdo_ipc_GateMP_Instance_finalize__F
0080c020   MessageQ_put
0080c860   Qmss_insertMemoryRegion
0080d040   ti_sdo_ipc_heaps_HeapMemMP_Instance_init__F
0080d7c0   ti_sysbios_family_c64p_Exception_handler__I
0080e114   Osal_srioMalloc
0080e148   Osal_srioFree
0080e174   Osal_dataBufferInitMemory
0080e228   Osal_srioDataBufferMalloc
0080e2ec   Osal_srioDataBufferFree
0080e384   Osal_srioLog
0080e398   Osal_srioCreateSem
0080e3ac   Osal_srioDeleteSem
0080e3b8   Osal_srioPendSem
0080e3cc   Osal_srioPostSem
0080e3d8   Osal_srioEnterMultipleCoreCriticalSection
0080e3f4   Osal_srioExitMultipleCoreCriticalSection
0080e404   Osal_srioEnterSingleCoreCriticalSection
0080e428   Osal_srioExitSingleCoreCriticalSection
0080e448   Osal_srioBeginMemAccess
0080e480   Osal_srioEndMemAccess
0080e4b0   Osal_srioBeginDescriptorAccess
0080e4c4   Osal_srioEndDescriptorAccess
0080e4e0   Osal_cppiMalloc
0080e504   Osal_cppiFree
0080e528   Osal_cppiCsEnter
0080e544   Osal_cppiCsExit
0080e550   Osal_cppiBeginMemAccess
0080e588   Osal_cppiEndMemAccess
0080e5b8   Osal_qmssCsEnter
0080e5d4   Osal_qmssCsExit
0080e5e4   Osal_qmssMtCsEnter
0080e5e8   Osal_qmssMtCsExit
0080e5f8   Osal_qmssBeginMemAccess
0080e630   Osal_qmssEndMemAccess
0080e680   SrioDevice_init
0080eda0   ti_sdo_ipc_nsremote_NameServerRemoteNotify_Instance_init__F
0080f460   NameServer_add
0080fb00   Cppi_configureRxFlow
00810160   ti_sysbios_heaps_HeapMem_free__E
008107c0   Notify_sendEvent
00810de0   ti_sysbios_heaps_HeapMem_alloc__E
00811400   Notify_registerEventSingle
008119e0   ListMP_getHead
00811fa0   Notify_unregisterEventSingle
00812560   __c6xabi_divd
00812b20   DSP_fft16x16
008130e0   ti_sdo_ipc_SharedRegion_start__F
008136a0   ti_sysbios_timers_timer64_Timer_Module_startup__F
00813c60   ti_sdo_ipc_nsremote_NameServerRemoteNotify_get__F
008141e0   ti_sdo_ipc_transports_TransportShm_put__E
00814760   ti_sdo_ipc_Ipc_procSyncStart__I
00814ca0   ti_sysbios_knl_Task_Instance_finalize__F
008151a0   ti_sdo_ipc_notifyDrivers_NotifyDriverShm_Instance_init__F
00815680   Cppi_txChannelOpen
00815b40   ti_sdo_ipc_gates_GatePeterson_Instance_init__F
008160e0   initializeBufferControl
00816148   getNextfreeBuffer
008161ec   prepareData
00816258   test_multicoreMaster
00816440   ti_sdo_ipc_GateMP_setRegion0Reserved__F
008168a0   ti_sdo_ipc_Ipc_procSyncFinish__I
00816d00   Cppi_rxChannelOpen
00817140   ListMP_putTail
00817580   ti_sdo_ipc_heaps_HeapMemMP_getStats__E
008179c0   ti_sdo_ipc_heaps_HeapMemMP_postInit__I
00817e00   ti_sdo_ipc_Notify_Instance_init__F
00818200   ti_sysbios_knl_Semaphore_pend__E
008186b0   threadInitialization
008188b4   multicoreTestTask
00818944   startSlaveUtil
00818970   main
008189e0   test_multicoreUser
00818dc0   Cppi_initDescriptor
00819180   ti_sdo_ipc_SharedRegion_reserveMemory__F
00819540   ti_sysbios_knl_Task_Instance_init__F
00819900   ti_sysbios_knl_Task_setPri__E
00819d34   saveTime
00819d90   ranDelay
00819e28   coreNumberFromId
00819e94   IdFromCore
00819eb8   disableCaches
00819ec8   printMessages
00819f30   l2_global_address
00819f60   myStartupFxn
00819f74   printStartEnd
0081a060   HeapMemMP_sharedMemReq
0081a3e0   xdc_runtime_System_printfExtend__I
0081a740   GateMP_sharedMemReq
0081aa80   Qmss_init
0081adc0   ti_sdo_ipc_nsremote_NameServerRemoteNotify_swiFxn__I
0081b100   GateMP_openByAddr
0081b400   ti_sdo_ipc_transports_TransportShm_openByAddr__F
0081b700   ti_sysbios_family_c64p_Hwi_dispatchC__I
0081ba00   SharedRegion_getEntry
0081bce0   SharedRegion_getPtr
0081c054   gen_twiddle_fft16x16
0081c2a0   freeBuffer
0081c318   requestProcessingData
0081c580   ti_sysbios_gates_GateMutexPri_enter__E
0081c860   ti_sysbios_knl_Task_Module_startup__F
0081cb40   cos
0081ce00   generateShortInput
0081d030   seperateRealImg
0081d0c0   ti_sdo_ipc_notifyDrivers_NotifyDriverShm_isr__I
0081d380   Ipc_start
0081d620   NameServer_getLocal
0081d8c0   ti_sysbios_knl_Clock_workFunc__E
0081db60   SharedRegion_getSRPtr
0081dde0   __c6xabi_divf
0081e2e0   sin
0081e560   ti_sdo_ipc_notifyDrivers_NotifyDriverShm_sharedMemReq__F
0081e7e0   ti_sysbios_knl_Clock_Instance_init__F
0081ea60   ti_sysbios_knl_Task_exit__E
0081ece0   xdc_runtime_Core_createObject__I
0081ef60   xdc_runtime_Error_raiseX__F
0081f1e0   ListMP_sharedMemReq
0081f440   ti_sdo_ipc_ListMP_Instance_finalize__F
0081f6a0   ti_sdo_ipc_heaps_HeapMemMP_Instance_finalize__F
0081f900   ti_sdo_ipc_notifyDrivers_NotifyDriverShm_disableEvent__E
0081fb60   xdc_runtime_Startup_startMods__I
0081fdc0   Cppi_open
00820000   __c6xabi_divull
00820240   ti_sysbios_family_c64p_Exception_internalHandler__I
00820480   ti_sysbios_knl_Semaphore_post__E
008206c0   fputc
008208e0   ti_sysbios_family_c64p_Hwi_reconfig__E
00820b00   ti_sysbios_knl_Swi_run__I
00820d20   ti_sysbios_knl_Task_schedule__I
00820f40   ti_sysbios_knl_Task_startup__E
00821160   GateMP_enter
00821360   GateMP_leave
00821560   ListMP_openByAddr
00821960   Qmss_programAccumulator
00821b60   ti_sysbios_family_c64p_Hwi_dispatchAlways
00821f60   cppi_internal_heap_add
00822160   setvbuf
00822360   ti_sdo_ipc_family_c647x_MultiProcSetup_init__I
00822560   ti_sdo_ipc_notifyDrivers_NotifyDriverShm_sendEvent__E
00822760   ti_sdo_ipc_transports_TransportShm_Instance_finalize__F
00822960   ti_sdo_ipc_GateMP_attach__F
00822b40   ti_sdo_ipc_GateMP_getFreeResource__I
00822d20   ti_sysbios_knl_Task_postInit__I
00822f00   ti_sysbios_timers_timer64_Timer_getFreq__E
008230e0   Cppi_initCfg
008232a0   HeapMemMP_openByAddr
00823620   atan
008237e0   ti_sdo_ipc_notifyDrivers_NotifyDriverShm_registerEvent__E
008239a0   ti_sysbios_knl_Swi_Instance_init__F
00823b60   ti_sysbios_knl_Task_checkStacks__E
00823d20   ti_sysbios_timers_timer64_Timer_setPeriodMicroSecs__E
00823ee0   HOSTrename
00824080   SharedRegion_getCacheLineSize
00824220   SharedRegion_getHeap
008243c0   SharedRegion_isCacheEnabled
00824560   ti_sdo_ipc_GateMP_openRegion0Reserved__F
00824700   ti_sdo_ipc_notifyDrivers_NotifyDriverShm_enableEvent__E
008248a0   ti_sdo_ipc_notifyDrivers_NotifyDriverShm_unregisterEvent__E
00824a40   ti_sdo_ipc_nsremote_NameServerRemoteNotify_attach__E
00824be0   ti_sysbios_gates_GateMutex_enter__E
00824d80   ti_sysbios_timers_timer64_Timer_start__E
00824f20   MultiProc_setLocalId
008250a0   NameServer_getHandle
00825220   Notify_intLineRegistered
00825520   ti_sysbios_family_c64p_Exception_dispatch__E
008256a0   ti_sdo_ipc_MessageQ_registerTransport__F
00825820   ti_sdo_ipc_Notify_Module_startup__F
008259a0   ti_sdo_ipc_gates_GatePeterson_enter__E
00825b20   ti_sdo_utils_NameServer_Module_startup__F
00825ca0   ti_sysbios_heaps_HeapBuf_Module_startup__F
00825e20   ti_sysbios_heaps_HeapMem_Instance_init__F
00825fa0   ti_sysbios_knl_Swi_schedule__I
00826120   ti_sysbios_knl_Task_unblockI__E
008262a0   xdc_runtime_Text_putSite__F
00826420   Qmss_getMemoryRegionCfg
00826580   ti_sdo_ipc_GateMP_createLocal__F
008266e0   ti_sdo_ipc_MessageQ_unregisterTransport__F
00826840   ti_sdo_ipc_gates_GateHWSem_Instance_init__F
008269a0   ti_sdo_ipc_transports_TransportShm_sharedMemReq__F
00826b00   ti_sdo_utils_NameServer_isRegistered__E
00826c60   ti_sdo_utils_NameServer_registerRemoteDriver__E
00826dc0   ti_sdo_utils_NameServer_unregisterRemoteDriver__E
00826f20   CSL_chipReadReg
00827060   GateMP_close
008271a0   Notify_attach
008272e0   _auto_init_elf
00827560   ti_sdo_ipc_Notify_exec__F
008276a0   ti_sysbios_family_c64p_Hwi_Module_startup__F
008277e0   ti_sysbios_family_c66_Cache_Module_startup__F
00827920   ti_sysbios_gates_GateSwi_enter__E
00827a60   ti_sysbios_knl_Clock_Instance_finalize__F
00827ba0   ti_sysbios_knl_Semaphore_Instance_init__F
00827ce0   ti_sysbios_knl_Swi_post__E
00827e20   ti_sysbios_knl_Task_blockI__E
00827f60   ti_sysbios_knl_Task_yield__E
008280a0   _closefile
008281c0   fseek
00828400   ti_sdo_ipc_MessageQ_Module_startup__F
00828520   ti_sdo_ipc_family_c647x_Interrupt_intRegister__E
00828640   ti_sdo_ipc_nsremote_NameServerRemoteNotify_Instance_finalize__F
00828760   xdc_runtime_Text_putLab__F
00828880   HOSTlseek
00828980   _wrt_ok
00828b80   ti_sdo_ipc_GateMP_start__F
00828c80   ti_sdo_ipc_Notify_Instance_finalize__F
00828d80   ti_sdo_ipc_SharedRegion_attach__F
00828e80   ti_sdo_ipc_SharedRegion_clearReservedMemory__F
00828f80   ti_sdo_ipc_family_c647x_Interrupt_Module_startup__F
00829080   ti_sdo_ipc_gates_GateHWSem_Module_startup__F
00829180   ti_sdo_ipc_gates_GateMPSupportNull_enter__E
00829280   ti_sdo_ipc_gates_GateMPSupportNull_leave__E
00829380   ti_sdo_ipc_transports_TransportShmSetup_attach__E
00829480   ti_sysbios_family_c64p_EventCombiner_dispatch__F
00829580   ti_sysbios_gates_GateMutexPri_leave__E
00829680   ti_sysbios_knl_Clock_startI__E
00829780   ti_sysbios_knl_Swi_restoreHwi__E
00829880   xdc_runtime_Core_deleteObject__I
00829980   xdc_runtime_Startup_exec__F
00829a80   xdc_runtime_Text_putMod__F
00829b80   xdc_runtime_Text_visitRope2__I
00829c80   HOSTopen
00829d60   close
00829e40   __TI_zero_init
00829f20   fflush
0082a000   memset
0082a0e0   ti_sdo_ipc_Notify_Object__create__S
0082a1c0   ti_sdo_ipc_family_c647x_NotifySetup_attach__E
0082a2a0   ti_sdo_ipc_gates_GateHWSem_enter__E
0082a380   ti_sysbios_family_c64p_Hwi_Instance_finalize__F
0082a460   ti_sysbios_family_c64p_Hwi_Instance_init__F
0082a540   ti_sysbios_family_c64p_Hwi_Object__create__S
0082a620   ti_sysbios_knl_Clock_start__E
0082a700   ti_sysbios_timers_timer64_Timer_startup__E
0082a7e0   xdc_runtime_Error_print__F
0082a8c0   xdc_runtime_Memory_alloc__F
0082a9a0   HOSTread
0082aa60   HOSTunlink
0082ab20   HOSTwrite
0082abe0   HeapMemMP_create
0082aca0   ListMP_create
0082ad60   Qmss_setEoiVector
0082ae20   Qmss_setQueueThreshold
0082afa0   __cxa_finalize
0082b060   __c6xabi_divu
0082b060   __divu
0082b120   __c6xabi_remi
0082b120   __remi
0082b1e0   _doflush
0082b2a0   exit
0082b360   ti_sdo_ipc_GateMP_Object__create__S
0082b420   ti_sdo_ipc_GateMP_getRegion0ReservedSize__F
0082b4e0   ti_sdo_ipc_ListMP_Object__create__S
0082b5a0   ti_sdo_ipc_family_c647x_Interrupt_intShmStub__I
0082b660   ti_sdo_ipc_gates_GatePeterson_Object__create__S
0082b720   ti_sdo_ipc_heaps_HeapMemMP_Object__create__S
0082b7e0   ti_sdo_ipc_notifyDrivers_NotifyDriverShm_Object__create__S
0082b8a0   ti_sdo_ipc_nsremote_NameServerRemoteNotify_Object__create__S
0082b960   ti_sdo_ipc_transports_TransportShm_Object__create__S
0082ba20   ti_sysbios_BIOS_errorRaiseHook__I
0082bae0   ti_sysbios_gates_GateAll_leave__E
0082bba0   ti_sysbios_heaps_HeapMem_getStats__E
0082bc60   ti_sysbios_knl_Clock_logTick__E
0082bd20   ti_sysbios_knl_Swi_Instance_finalize__F
0082bde0   ti_sysbios_knl_Swi_Object__create__S
0082bea0   ti_sysbios_knl_Task_Object__create__S
0082bf60   ti_sysbios_timers_timer64_Timer_stop__E
0082c020   xdc_runtime_System_formatNum__I
0082c0e0   xdc_runtime_knl_GateThread_Object__create__S
0082c1a0   Cppi_channelEnable
0082c240   HOSTclose
0082c2e0   HOSTtime
0082c380   Qmss_queueClose
0082c420   Qmss_startCfg
0082c4c0   __c6xabi_nround
0082c560   __c6xabi_remu
0082c560   __remu
0082c600   _c_int00
0082c6a0   _cleanup
0082c740   ti_sysbios_family_c64p_Hwi_plug__E
0082c7e0   cppi_internal_heap_malloc
0082c880   cppi_list_cat
0082c9c0   lseek
0082ca60   memcpy
0082cb00   modf
0082cba0   ti_sdo_ipc_family_c647x_Interrupt_intUnregister__E
0082cc40   ti_sdo_ipc_gates_GatePeterson_leave__E
0082cce0   ti_sdo_ipc_notifyDrivers_NotifyDriverShm_Instance_finalize__F
0082cd80   ti_sysbios_heaps_HeapMem_init__I
0082ce20   write
0082cec0   xdc_runtime_Assert_raise__I
0082cf60   Cppi_setCpdmaLoopback
0082cfe0   Qmss_getMemRegQueueHandle
0082d060   Qmss_queueOpen
0082d0e0   __c6xabi_llshl
0082d160   ti_sysbios_family_c62_TaskSupport_swap__E
0082d1e0   cppi_internal_heap_cache_begin
0082d260   cppi_list_remove
0082d2e0   malloc
0082d360   rand
0082d3e0   readmsg
0082d460   ti_sdo_ipc_gates_GateHWSem_Object__create__S
0082d4e0   ti_sdo_ipc_gates_GateMPSupportNull_Object__create__S
0082d560   ti_sdo_ipc_nsremote_NameServerRemoteNotify_detach__E
0082d5e0   ti_sdo_ipc_transports_TransportShm_swiFxn__I
0082d660   ti_sdo_utils_List_Object__create__S
0082d6e0   ti_sysbios_family_c62_TaskSupport_start__E
0082d760   ti_sysbios_family_c64p_Exception_Module_startup__F
0082d7e0   ti_sysbios_family_c64p_Hwi_eventMap__E
0082d860   ti_sysbios_family_c66_Cache_invL1pAll__E
0082d8e0   ti_sysbios_gates_GateAll_Object__create__S
0082d960   ti_sysbios_gates_GateHwi_Object__create__S
0082d9e0   ti_sysbios_gates_GateMutexPri_Object__create__S
0082da60   ti_sysbios_gates_GateMutex_Object__create__S
0082dae0   ti_sysbios_gates_GateSwi_Object__create__S
0082db60   ti_sysbios_gates_GateSwi_leave__E
0082dbe0   ti_sysbios_hal_Hwi_checkStack
0082dc60   ti_sysbios_heaps_HeapMem_Object__create__S
0082dce0   ti_sysbios_knl_Clock_Module_startup__F
0082dd60   ti_sysbios_knl_Clock_Object__create__S
0082dde0   ti_sysbios_knl_Clock_getTicks__E
0082de60   ti_sysbios_knl_Idle_loop__E
0082dee0   ti_sysbios_knl_Queue_Object__create__S
0082df60   ti_sysbios_knl_Semaphore_Object__create__S
0082dfe0   ti_sysbios_knl_Semaphore_pendTimeout__I
0082e060   ti_sysbios_knl_Swi_startup__E
0082e0e0   ti_sysbios_knl_Task_restore__E
0082e160   ti_sysbios_timers_timer64_Timer_getCount__E
0082e160   ti_sysbios_timers_timer64_Timer_getExpiredCounts__E
0082e1e0   ti_sysbios_timers_timer64_Timer_getPeriod__E
0082e260   ti_sysbios_xdcruntime_GateThreadSupport_Object__create__S
0082e2e0   remove
0082e2e0   unlink
0082e360   xdc_runtime_Core_assignLabel__I
0082e3e0   xdc_runtime_Core_assignParams__I
0082e460   xdc_runtime_System_atexit__F
0082e4e0   xdc_runtime_System_rtsExit__I
0082e560   xdc_runtime_Text_printVisFxn__I
0082e5e0   xdc_runtime_Text_xprintf__I
0082e660   GateMP_Params_init
0082e6c0   HeapMemMP_Params_init
0082e720   Srio_listCat
0082e780   Srio_listRemoveNode
0082e7e0   __c6xabi_frcmpyd_div
0082e840   __c6xabi_llshru
0082e8a0   _subcull
0082e900   cppi_list_add
0082e960   cppi_list_cache_invalidate
0082e9c0   srand
0082ea20   ti_sdo_ipc_MessageQ_Object__get__S
0082ea80   ti_sdo_ipc_family_c647x_NotifySetup_sharedMemReq__E
0082eae0   ti_sdo_ipc_gates_GateHWSem_leave__E
0082eb40   ti_sdo_ipc_gates_GatePeterson_Instance_finalize__F
0082eba0   ti_sdo_ipc_gates_GatePeterson_sharedMemReq__E
0082ec00   ti_sdo_ipc_notifyDrivers_NotifyDriverShm_setNotifyHandle__E
0082ec60   ti_sdo_ipc_transports_TransportShmSetup_sharedMemReq__E
0082ecc0   ti_sdo_utils_List_Object__get__S
0082ed20   ti_sdo_utils_NameServer_Object__get__S
0082ed80   ti_sysbios_BIOS_exitFunc__I
0082ede0   ti_sysbios_BIOS_registerRTSLock__I
0082ee40   ti_sysbios_family_c64p_EventCombiner_Module_startup__F
0082eea0   ti_sysbios_family_c64p_EventCombiner_dispatchPlug__F
0082ef00   ti_sysbios_family_c64p_EventCombiner_unused__F
0082ef60   ti_sysbios_gates_GateAll_enter__E
0082efc0   ti_sysbios_gates_GateMutex_Instance_init__F
0082f020   ti_sysbios_hal_Hwi_initStack
0082f080   ti_sysbios_heaps_HeapBuf_Object__get__S
0082f0e0   ti_sysbios_heaps_HeapMem_Object__get__S
0082f140   ti_sysbios_knl_Clock_doTick__I
0082f1a0   ti_sysbios_knl_Queue_Object__get__S
0082f200   ti_sysbios_knl_Swi_Module_startup__F
0082f260   ti_sysbios_knl_Swi_Object__get__S
0082f2c0   ti_sysbios_knl_Task_Object__get__S
0082f320   ti_sysbios_knl_Task_allBlockedFunction__I
0082f380   ti_sysbios_knl_Task_enter__I
0082f3e0   writemsg
0082f438   C$$IO$$
0082f440   xdc_runtime_GateNull_Object__create__S
0082f4a0   xdc_runtime_Memory_calloc__F
0082f500   xdc_runtime_Memory_valloc__F
0082f560   xdc_runtime_SysStd_abort__F
0082f5c0   xdc_runtime_System_aprintf_va__F
0082f5c0   xdc_runtime_System_avprintf__F
0082f620   xdc_runtime_System_printf_va__F
0082f620   xdc_runtime_System_vprintf__F
0082f680   xdc_runtime_Text_cordText__F
0082f6e0   Qmss_ackInterrupt
0082f720   Qmss_getMemRegDescSize
0082f760   Srio_listAdd
0082f7a0   Srio_listRemove
0082f7e0   __c6xabi_strasgi_64plus
0082f7e0   __strasgi_64plus
0082f820   _args_main
0082f860   ti_sysbios_family_c62_TaskSupport_buildTaskStack
0082f8a0   ti_sysbios_family_xxx_Hwi_switchToIsrStack
0082f8e0   floor
0082f920   free
0082f9a0   ti_sdo_ipc_GateMP_Object__delete__S
0082f9e0   ti_sdo_ipc_GateMP_Params__init__S
0082fa20   ti_sdo_ipc_GateMP_RemoteCustom1Proxy_Object__create__S
0082fa60   ti_sdo_ipc_GateMP_RemoteCustom2Proxy_Object__create__S
0082faa0   ti_sdo_ipc_GateMP_RemoteSystemProxy_Object__create__S
0082fae0   ti_sdo_ipc_ListMP_Object__delete__S
0082fb20   ti_sdo_ipc_ListMP_Params__init__S
0082fb60   ti_sdo_ipc_MessageQ_registerTransport__E
0082fba0   ti_sdo_ipc_family_c647x_Interrupt_intClear__E
0082fbe0   ti_sdo_ipc_family_c647x_Interrupt_intSend__E
0082fc20   ti_sdo_ipc_gates_GateHWSem_Handle__label__S
0082fc60   ti_sdo_ipc_gates_GateHWSem_Object__delete__S
0082fca0   ti_sdo_ipc_gates_GateHWSem_Params__init__S
0082fce0   ti_sdo_ipc_gates_GateMPSupportNull_Handle__label__S
0082fd20   ti_sdo_ipc_gates_GateMPSupportNull_Object__delete__S
0082fd60   ti_sdo_ipc_gates_GateMPSupportNull_Params__init__S
0082fda0   ti_sdo_ipc_gates_GatePeterson_Handle__label__S
0082fde0   ti_sdo_ipc_gates_GatePeterson_Object__delete__S
0082fe20   ti_sdo_ipc_gates_GatePeterson_Params__init__S
0082fe60   ti_sdo_ipc_heaps_HeapMemMP_Handle__label__S
0082fea0   ti_sdo_ipc_heaps_HeapMemMP_Object__delete__S
0082fee0   ti_sdo_ipc_heaps_HeapMemMP_Params__init__S
0082ff20   ti_sdo_ipc_notifyDrivers_NotifyDriverShm_Handle__label__S
0082ff60   ti_sdo_ipc_notifyDrivers_NotifyDriverShm_InterruptProxy_intRegister__E
0082ffa0   ti_sdo_ipc_notifyDrivers_NotifyDriverShm_Object__delete__S
0082ffe0   ti_sdo_ipc_notifyDrivers_NotifyDriverShm_Params__init__S
00830020   ti_sdo_ipc_notifyDrivers_NotifyDriverShm_disable__E
00830060   ti_sdo_ipc_notifyDrivers_NotifyDriverShm_enable__E
008300a0   ti_sdo_ipc_nsremote_NameServerRemoteNotify_Handle__label__S
008300e0   ti_sdo_ipc_nsremote_NameServerRemoteNotify_Object__delete__S
00830120   ti_sdo_ipc_nsremote_NameServerRemoteNotify_Object__first__S
00830160   ti_sdo_ipc_nsremote_NameServerRemoteNotify_Object__next__S
008301a0   ti_sdo_ipc_nsremote_NameServerRemoteNotify_Params__init__S
008301e0   ti_sdo_ipc_nsremote_NameServerRemoteNotify_get__E
00830220   ti_sdo_ipc_nsremote_NameServerRemoteNotify_sharedMemReq__E
00830260   ti_sdo_ipc_transports_TransportShm_Handle__label__S
008302a0   ti_sdo_ipc_transports_TransportShm_Object__delete__S
008302e0   ti_sdo_ipc_transports_TransportShm_Params__init__S
00830320   ti_sdo_utils_List_Object__destruct__S
00830360   ti_sdo_utils_NameServer_Module__startupDone__F
008303a0   ti_sdo_utils_NameServer_Object__first__S
008303e0   ti_sdo_utils_NameServer_Object__next__S
00830420   ti_sysbios_BIOS_startFunc__I
00830460   ti_sysbios_BIOS_start__E
008304a0   ti_sysbios_family_c64p_EventCombiner_dispatchPlug__E
008304e0   ti_sysbios_family_c64p_EventCombiner_enableEvent__F
00830520   ti_sysbios_family_c64p_Hwi_Module__startupDone__F
00830560   ti_sysbios_family_c64p_Hwi_Object__delete__S
008305a0   ti_sysbios_family_c64p_Hwi_Params__init__S
008305e0   ti_sysbios_family_c64p_Hwi_disableInterrupt__E
00830620   ti_sysbios_family_c64p_Hwi_enableInterrupt__E
00830660   ti_sysbios_gates_GateAll_Handle__label__S
008306a0   ti_sysbios_gates_GateAll_Object__delete__S
008306e0   ti_sysbios_gates_GateHwi_Handle__label__S
00830720   ti_sysbios_gates_GateHwi_Object__delete__S
00830760   ti_sysbios_gates_GateMutexPri_Handle__label__S
008307a0   ti_sysbios_gates_GateMutexPri_Instance_finalize__F
008307e0   ti_sysbios_gates_GateMutexPri_Instance_init__F
00830820   ti_sysbios_gates_GateMutexPri_Object__delete__S
00830860   ti_sysbios_gates_GateMutexPri_Object__destruct__S
008308a0   ti_sysbios_gates_GateMutex_Handle__label__S
008308e0   ti_sysbios_gates_GateMutex_Instance_finalize__F
00830920   ti_sysbios_gates_GateMutex_Object__delete__S
00830960   ti_sysbios_gates_GateMutex_leave__E
008309a0   ti_sysbios_gates_GateSwi_Handle__label__S
008309e0   ti_sysbios_gates_GateSwi_Object__delete__S
00830a20   ti_sysbios_hal_Cache_CacheProxy_inv__E
00830a20   ti_sysbios_hal_Cache_inv__E
00830a60   ti_sysbios_hal_Cache_CacheProxy_wbInv__E
00830a60   ti_sysbios_hal_Cache_wbInv__E
00830aa0   ti_sysbios_hal_Timer_Module__startupDone__F
00830ae0   ti_sysbios_heaps_HeapMem_Handle__label__S
00830b20   ti_sysbios_heaps_HeapMem_Object__delete__S
00830b60   ti_sysbios_knl_Clock_Object__destruct__S
00830ba0   ti_sysbios_knl_Clock_Params__init__S
00830be0   ti_sysbios_knl_Queue_Object__destruct__S
00830c20   ti_sysbios_knl_Semaphore_Instance_finalize__F
00830c60   ti_sysbios_knl_Semaphore_Object__delete__S
00830ca0   ti_sysbios_knl_Semaphore_Object__destruct__S
00830ce0   ti_sysbios_knl_Semaphore_Params__init__S
00830d20   ti_sysbios_knl_Swi_Object__destruct__S
00830d60   ti_sysbios_knl_Swi_Params__init__S
00830da0   ti_sysbios_knl_Task_Object__first__S
00830de0   ti_sysbios_knl_Task_Object__next__S
00830e20   ti_sysbios_knl_Task_Params__init__S
00830e60   ti_sysbios_timers_timer64_Timer_Module__startupDone__F
00830ea0   ti_sysbios_xdcruntime_GateThreadSupport_Instance_finalize__F
00830ee0   ti_sysbios_xdcruntime_GateThreadSupport_Instance_init__F
00830f20   ti_sysbios_xdcruntime_GateThreadSupport_Object__delete__S
00830f60   ti_sysbios_xdcruntime_GateThreadSupport_enter__F
00830fa0   ti_sysbios_xdcruntime_GateThreadSupport_leave__F
00830fe0   time
00831020   xdc_runtime_Error_check__F
00831060   xdc_runtime_Error_init__F
008310a0   xdc_runtime_Error_raiseX__E
008310e0   xdc_runtime_GateNull_Handle__label__S
00831120   xdc_runtime_GateNull_Object__delete__S
00831160   xdc_runtime_Gate_leaveSystem__F
00831220   xdc_runtime_Memory_free__F
00831260   xdc_runtime_Memory_valloc__E
008312a0   xdc_runtime_Registry_findById__F
008312e0   xdc_runtime_Startup_exec__I
00831320   xdc_runtime_System_abort__F
00831360   xdc_runtime_System_aprintf__E
008313a0   xdc_runtime_System_printf__E
008313e0   xdc_runtime_Text_ropeText__F
00831420   xdc_runtime_Text_visitRope__I
00831460   xdc_runtime_knl_GateThread_Handle__label__S
008314a0   xdc_runtime_knl_GateThread_Instance_finalize__F
008314e0   xdc_runtime_knl_GateThread_Instance_init__F
00831520   xdc_runtime_knl_GateThread_Object__delete__S
00831560   xdc_runtime_knl_GateThread_Proxy_Object__create__S
008315a0   CSL_SRIO_Open
008315c0   Cppi_getFlowId
008315e0   Cppi_init
00831600   Qmss_getQueueHandle
00831620   Qmss_getQueueNumber
00831640   Qmss_start
00831660   Srio_listGetHead
00831680   Srio_listGetNext
008316a0   __c6xabi_trunc
008316c0   __cxa_atexit
008316e0   __cxa_ia64_exit
00831700   __xdc__init
00831720   _nop
00831740   _register_lock
00831760   _register_unlock
00831780   ti_sysbios_family_c62_TaskSupport_glue
008317a0   ti_sysbios_family_xxx_Hwi_switchToTaskStack
008317c0   C$$EXIT
008317c0   abort
008317e0   atexit
00831800   cppi_list_get_head
00831820   cppi_list_get_next
00831840   __TI_decompress_none
00831860   __TI_decompress_rle24
008318a0   putc
008318c0   putchar
008318e0   ti_sdo_ipc_GateMP_RemoteCustom1Proxy_Object__delete__S
00831900   ti_sdo_ipc_GateMP_RemoteCustom1Proxy_Params__init__S
00831920   ti_sdo_ipc_GateMP_RemoteCustom1Proxy_Proxy__abstract__S
00831940   ti_sdo_ipc_GateMP_RemoteCustom1Proxy_Proxy__delegate__S
00831960   ti_sdo_ipc_GateMP_RemoteCustom1Proxy_getReservedMask__E
00831980   ti_sdo_ipc_GateMP_RemoteCustom1Proxy_sharedMemReq__E
008319a0   ti_sdo_ipc_GateMP_RemoteCustom2Proxy_Object__delete__S
008319c0   ti_sdo_ipc_GateMP_RemoteCustom2Proxy_Params__init__S
008319e0   ti_sdo_ipc_GateMP_RemoteCustom2Proxy_Proxy__abstract__S
00831a00   ti_sdo_ipc_GateMP_RemoteCustom2Proxy_Proxy__delegate__S
00831a20   ti_sdo_ipc_GateMP_RemoteCustom2Proxy_getReservedMask__E
00831a40   ti_sdo_ipc_GateMP_RemoteCustom2Proxy_sharedMemReq__E
00831a60   ti_sdo_ipc_GateMP_RemoteSystemProxy_Object__delete__S
00831a80   ti_sdo_ipc_GateMP_RemoteSystemProxy_Params__init__S
00831aa0   ti_sdo_ipc_GateMP_RemoteSystemProxy_Proxy__abstract__S
00831ac0   ti_sdo_ipc_GateMP_RemoteSystemProxy_Proxy__delegate__S
00831ae0   ti_sdo_ipc_GateMP_RemoteSystemProxy_getReservedMask__E
00831b00   ti_sdo_ipc_GateMP_RemoteSystemProxy_sharedMemReq__E
00831b20   ti_sdo_ipc_GateMP_attach__E
00831b40   ti_sdo_ipc_GateMP_getRegion0ReservedSize__E
00831b60   ti_sdo_ipc_GateMP_getSharedAddr__E
00831b80   ti_sdo_ipc_GateMP_getSharedAddr__F
00831ba0   ti_sdo_ipc_GateMP_start__E
00831bc0   ti_sdo_ipc_MessageQ_Module_startup__E
00831be0   ti_sdo_ipc_MessageQ_SetupTransportProxy_attach__E
00831c00   ti_sdo_ipc_MessageQ_SetupTransportProxy_isRegistered__E
00831c20   ti_sdo_ipc_MessageQ_SetupTransportProxy_sharedMemReq__E
00831c40   ti_sdo_ipc_MessageQ_unregisterTransport__E
00831c60   ti_sdo_ipc_Notify_Module_GateProxy_enter__E
00831c80   ti_sdo_ipc_Notify_Module_GateProxy_leave__E
00831ca0   ti_sdo_ipc_Notify_Module_startup__E
00831cc0   ti_sdo_ipc_Notify_SetupProxy_attach__E
00831ce0   ti_sdo_ipc_Notify_SetupProxy_numIntLines__E
00831d00   ti_sdo_ipc_Notify_SetupProxy_sharedMemReq__E
00831d20   ti_sdo_ipc_Notify_exec__E
00831d40   ti_sdo_ipc_SharedRegion_attach__E
00831d60   ti_sdo_ipc_SharedRegion_clearReservedMemory__E
00831d80   ti_sdo_ipc_SharedRegion_reserveMemory__E
00831da0   ti_sdo_ipc_SharedRegion_start__E
00831dc0   ti_sdo_ipc_family_c647x_Interrupt_Module_startup__E
00831de0   ti_sdo_ipc_family_c647x_Interrupt_intDisable__E
00831e00   ti_sdo_ipc_family_c647x_Interrupt_intEnable__E
00831e20   ti_sdo_ipc_family_c647x_NotifySetup_numIntLines__E
00831e40   ti_sdo_ipc_gates_GateHWSem_Module_startup__E
00831e60   ti_sdo_ipc_gates_GateHWSem_getReservedMask__E
00831e80   ti_sdo_ipc_gates_GateHWSem_query__E
00831ea0   ti_sdo_ipc_gates_GateHWSem_query__F
00831ec0   ti_sdo_ipc_gates_GateHWSem_sharedMemReq__E
00831ee0   ti_sdo_ipc_gates_GateMPSupportNull_Instance_init__F
00831f00   ti_sdo_ipc_gates_GateMPSupportNull_getReservedMask__E
00831f20   ti_sdo_ipc_gates_GateMPSupportNull_query__E
00831f40   ti_sdo_ipc_gates_GateMPSupportNull_query__F
00831f60   ti_sdo_ipc_gates_GateMPSupportNull_sharedMemReq__E
00831f80   ti_sdo_ipc_gates_GatePeterson_getReservedMask__E
00831fa0   ti_sdo_ipc_gates_GatePeterson_query__E
00831fc0   ti_sdo_ipc_gates_GatePeterson_query__F
00831fe0   ti_sdo_ipc_heaps_HeapMemMP_isBlocking__E
00832000   ti_sdo_ipc_heaps_HeapMemMP_isBlocking__F
00832020   ti_sdo_ipc_notifyDrivers_NotifyDriverShm_InterruptProxy_intClear__E
00832040   ti_sdo_ipc_notifyDrivers_NotifyDriverShm_InterruptProxy_intDisable__E
00832060   ti_sdo_ipc_notifyDrivers_NotifyDriverShm_InterruptProxy_intEnable__E
00832080   ti_sdo_ipc_notifyDrivers_NotifyDriverShm_InterruptProxy_intSend__E
008320a0   ti_sdo_ipc_notifyDrivers_NotifyDriverShm_InterruptProxy_intUnregister__E
008320c0   ti_sdo_ipc_notifyDrivers_NotifyDriverShm_sharedMemReq__E
008320e0   ti_sdo_ipc_nsremote_NameServerRemoteNotify_cbFxn__I
00832100   ti_sdo_ipc_transports_TransportShmSetup_isRegistered__E
00832120   ti_sdo_ipc_transports_TransportShm_control__E
00832140   ti_sdo_ipc_transports_TransportShm_getStatus__E
00832160   ti_sdo_ipc_transports_TransportShm_notifyFxn__I
00832180   ti_sdo_ipc_transports_TransportShm_openByAddr__E
008321a0   ti_sdo_ipc_transports_TransportShm_setErrFxn__E
008321c0   ti_sdo_ipc_transports_TransportShm_setErrFxn__F
008321e0   ti_sdo_ipc_transports_TransportShm_sharedMemReq__E
00832200   ti_sdo_utils_List_Instance_init__F
00832220   ti_sdo_utils_MultiProc_getClusterId__E
00832240   ti_sdo_utils_MultiProc_getClusterId__F
00832260   ti_sdo_utils_NameServer_Module__startupDone__S
00832280   ti_sdo_utils_NameServer_Module_startup__E
008322a0   ti_sdo_utils_NameServer_SetupProxy_attach__E
008322c0   ti_sdo_utils_NameServer_SetupProxy_sharedMemReq__E
008322e0   ti_sysbios_BIOS_RtsGateProxy_enter__E
00832300   ti_sysbios_BIOS_RtsGateProxy_leave__E
00832320   ti_sysbios_BIOS_getThreadType__E
00832340   ti_sysbios_BIOS_setThreadType__E
00832360   ti_sysbios_family_c62_TaskSupport_Module__startupDone__S
00832380   ti_sysbios_family_c62_TaskSupport_checkStack__E
008323a0   ti_sysbios_family_c62_TaskSupport_getStackAlignment__E
008323c0   ti_sysbios_family_c64p_EventCombiner_Module_startup__E
008323e0   ti_sysbios_family_c64p_EventCombiner_dispatch__E
00832400   ti_sysbios_family_c64p_EventCombiner_enableEvent__E
00832420   ti_sysbios_family_c64p_EventCombiner_unused__E
00832440   ti_sysbios_family_c64p_Exception_Module_startup__E
00832460   ti_sysbios_family_c64p_Hwi_Module__startupDone__S
00832480   ti_sysbios_family_c64p_Hwi_Module_startup__E
008324a0   ti_sysbios_family_c64p_Hwi_clearInterrupt__E
008324c0   ti_sysbios_family_c64p_Hwi_getHandle__E
008324e0   ti_sysbios_family_c64p_Hwi_startup__E
00832500   ti_sysbios_family_c64p_Hwi_switchFromBootStack__E
00832520   ti_sysbios_family_c64p_Hwi_unPluggedInterrupt__I
00832540   ti_sysbios_family_c64p_tci6488_TimerSupport_enable__E
00832560   ti_sysbios_family_c66_Cache_Module_startup__E
00832580   ti_sysbios_family_c66_Cache_inv__E
008325a0   ti_sysbios_family_c66_Cache_wbInv__E
008325c0   ti_sysbios_gates_GateAll_Instance_init__F
008325e0   ti_sysbios_gates_GateAll_query__E
00832600   ti_sysbios_gates_GateAll_query__F
00832620   ti_sysbios_gates_GateHwi_Instance_init__F
00832640   ti_sysbios_gates_GateHwi_enter__E
00832660   ti_sysbios_gates_GateHwi_leave__E
00832680   ti_sysbios_gates_GateHwi_query__E
008326a0   ti_sysbios_gates_GateHwi_query__F
008326c0   ti_sysbios_gates_GateMutexPri_query__E
008326c0   ti_sysbios_xdcruntime_GateProcessSupport_query__F
008326c0   ti_sysbios_xdcruntime_GateThreadSupport_query__F
008326e0   ti_sysbios_gates_GateMutexPri_query__F
00832700   ti_sysbios_gates_GateMutex_query__E
00832720   ti_sysbios_gates_GateMutex_query__F
00832740   ti_sysbios_gates_GateSwi_Instance_init__F
00832760   ti_sysbios_gates_GateSwi_query__E
00832780   ti_sysbios_gates_GateSwi_query__F
008327a0   ti_sysbios_hal_Hwi_HwiProxy_Module__startupDone__S
008327c0   ti_sysbios_hal_Hwi_HwiProxy_clearInterrupt__E
008327c0   ti_sysbios_hal_Hwi_clearInterrupt__E
008327e0   ti_sysbios_hal_Hwi_HwiProxy_disableInterrupt__E
008327e0   ti_sysbios_hal_Hwi_disableInterrupt__E
00832800   ti_sysbios_hal_Hwi_HwiProxy_enableInterrupt__E
00832800   ti_sysbios_hal_Hwi_enableInterrupt__E
00832820   ti_sysbios_hal_Hwi_HwiProxy_startup__E
00832820   ti_sysbios_hal_Hwi_startup__E
00832840   ti_sysbios_hal_Hwi_HwiProxy_switchFromBootStack__E
00832840   ti_sysbios_hal_Hwi_switchFromBootStack__E
00832860   ti_sysbios_hal_Hwi_Module_startup__E
00832880   ti_sysbios_hal_Hwi_Module_startup__F
008328a0   ti_sysbios_hal_Timer_Module__startupDone__S
008328c0   ti_sysbios_hal_Timer_Module_startup__E
008328e0   ti_sysbios_hal_Timer_Module_startup__F
00832900   ti_sysbios_hal_Timer_TimerProxy_Module__startupDone__S
00832920   ti_sysbios_hal_Timer_TimerProxy_getExpiredCounts__E
00832940   ti_sysbios_hal_Timer_TimerProxy_getPeriod__E
00832960   ti_sysbios_hal_Timer_TimerProxy_setNextTick__E
00832980   ti_sysbios_hal_Timer_TimerProxy_startup__E
00832980   ti_sysbios_hal_Timer_startup__E
008329a0   ti_sysbios_heaps_HeapBuf_Module_startup__E
008329c0   ti_sysbios_heaps_HeapMem_Module_GateProxy_enter__E
008329e0   ti_sysbios_heaps_HeapMem_Module_GateProxy_leave__E
00832a00   ti_sysbios_heaps_HeapMem_Module_GateProxy_query__E
00832a20   ti_sysbios_heaps_HeapMem_isBlocking__E
00832a60   ti_sysbios_knl_Clock_Module_startup__E
00832a80   ti_sysbios_knl_Queue_Instance_init__F
00832aa0   ti_sysbios_knl_Queue_empty__E
00832ac0   ti_sysbios_knl_Swi_Module_startup__E
00832ae0   ti_sysbios_knl_Swi_disable__E
00832b00   ti_sysbios_knl_Task_Module_startup__E
00832b20   ti_sysbios_knl_Task_SupportProxy_Module__startupDone__S
00832b40   ti_sysbios_knl_Task_SupportProxy_checkStack__E
00832b60   ti_sysbios_knl_Task_SupportProxy_getStackAlignment__E
00832b80   ti_sysbios_knl_Task_SupportProxy_start__E
00832ba0   ti_sysbios_knl_Task_SupportProxy_swap__E
00832bc0   ti_sysbios_knl_Task_disable__E
00832be0   ti_sysbios_knl_Task_getPri__E
00832c00   ti_sysbios_knl_Task_self__E
00832c20   ti_sysbios_timers_timer64_Timer_Module__startupDone__S
00832c40   ti_sysbios_timers_timer64_Timer_Module_startup__E
00832c60   ti_sysbios_timers_timer64_Timer_TimerSupportProxy_enable__E
00832c80   ti_sysbios_timers_timer64_Timer_setNextTick__E
00832ca0   ti_sysbios_xdcruntime_GateThreadSupport_enter__E
00832cc0   ti_sysbios_xdcruntime_GateThreadSupport_leave__E
00832ce0   ti_sysbios_xdcruntime_GateThreadSupport_query__E
00832d20   xdc_runtime_Error_check__E
00832d40   xdc_runtime_Error_init__E
00832d60   xdc_runtime_Error_print__E
00832d80   xdc_runtime_GateNull_enter__E
00832da0   xdc_runtime_GateNull_enter__F
00832dc0   xdc_runtime_GateNull_leave__E
00832de0   xdc_runtime_GateNull_leave__F
00832e00   xdc_runtime_GateNull_query__E
00832e20   xdc_runtime_GateNull_query__F
00832e40   xdc_runtime_Gate_enterSystem__E
00832e60   xdc_runtime_Gate_enterSystem__F
00832e80   xdc_runtime_Gate_leaveSystem__E
00832ea0   xdc_runtime_Memory_HeapProxy_alloc__E
00832ec0   xdc_runtime_Memory_HeapProxy_free__E
00832ee0   xdc_runtime_Memory_alloc__E
00832f00   xdc_runtime_Memory_calloc__E
00832f20   xdc_runtime_Memory_free__E
00832f40   xdc_runtime_Memory_getMaxDefaultTypeAlign__E
00832f60   xdc_runtime_Memory_getMaxDefaultTypeAlign__F
00832f80   xdc_runtime_Registry_findById__E
00832fa0   xdc_runtime_Startup_Module__startupDone__S
00832fc0   xdc_runtime_Startup_exec__E
00832fe0   xdc_runtime_Startup_reset__I
00833000   xdc_runtime_Startup_rtsDone__E
00833020   xdc_runtime_Startup_rtsDone__F
00833040   xdc_runtime_SysStd_abort__E
00833060   xdc_runtime_SysStd_exit__E
00833080   xdc_runtime_SysStd_exit__F
008330a0   xdc_runtime_SysStd_putch__E
008330c0   xdc_runtime_SysStd_putch__F
008330e0   xdc_runtime_SysStd_ready__E
00833100   xdc_runtime_SysStd_ready__F
00833120   xdc_runtime_System_Module_GateProxy_enter__E
00833140   xdc_runtime_System_Module_GateProxy_leave__E
00833160   xdc_runtime_System_Module_startup__E
00833180   xdc_runtime_System_Module_startup__F
008331a0   xdc_runtime_System_SupportProxy_abort__E
008331c0   xdc_runtime_System_SupportProxy_exit__E
008331e0   xdc_runtime_System_SupportProxy_putch__E
00833200   xdc_runtime_System_SupportProxy_ready__E
00833220   xdc_runtime_System_abort__E
00833240   xdc_runtime_System_atexit__E
00833260   xdc_runtime_System_exit__E
00833280   xdc_runtime_System_exit__F
008332a0   xdc_runtime_System_lastFxn__I
008332c0   xdc_runtime_System_vsprintf__E
008332e0   xdc_runtime_System_sprintf_va__F
008332e0   xdc_runtime_System_vsprintf__F
00833300   xdc_runtime_Text_cordText__E
00833320   xdc_runtime_Text_putLab__E
00833340   xdc_runtime_Text_putSite__E
00833360   xdc_runtime_Text_ropeText__E
00833380   xdc_runtime_knl_GateThread_Module__startupDone__S
008333a0   xdc_runtime_knl_GateThread_Proxy_Object__delete__S
008333c0   xdc_runtime_knl_GateThread_Proxy_enter__E
008333e0   xdc_runtime_knl_GateThread_Proxy_leave__E
00833400   xdc_runtime_knl_GateThread_Proxy_query__E
00833400   xdc_runtime_knl_GateThread_query__F
00833420   xdc_runtime_knl_GateThread_enter__E
00833440   xdc_runtime_knl_GateThread_enter__F
00833460   xdc_runtime_knl_GateThread_leave__E
00833480   xdc_runtime_knl_GateThread_leave__F
008334a0   xdc_runtime_knl_GateThread_query__E
008334c0   ti_sysbios_heaps_HeapMem_Instance_State_0_buf__A
00863500   xxx
00867500   host_region
00868100   qmssInitConfig
00868180   buffer9
00868220   gHiPriAccumList
008682a0   ti_sysbios_knl_Task_Instance_State_0_stack__A
00868aa0   cfg
00868b20   bindInfo
00868b2c   to
00868b38   from
00868b48   coreDeviceID
00868b58   myBuffer
00868ce8   _tmpnams
00868e28   qmssLObj
00868f48   gDataBufferMemMgr
00869038   controlVector
008690b8   ti_sdo_utils_NameServer_Module_State_0_nsRemoteHandle__A
008690d8   ti_sysbios_knl_Task_Instance_State_0_hookEnv__A
008690e8   _lock
008690ec   _unlock
008690f0   xdc_runtime_Text_charTab__A
0086b6a8   acc48_le
0086c5dc   ti_sdo_ipc_GateMP_A_invalidClose__C
0086c5e0   ti_sysbios_family_c66_Cache_marvalues__C
0086cc08   xdc_runtime_Text_nodeTab__A
0086d150   xdc_runtime_Startup_sfxnTab__A
0086d1cc   ti_sdo_ipc_notifyDrivers_NotifyDriverShm_Module__FXNS__C
0086d204   ti_sysbios_knl_Task_Object__PARAMS__C
0086d23c   ti_sdo_ipc_GateMP_A_invalidDelete__C
0086d240   gSrioDriverVersionStr
0086d278   ti_sdo_ipc_GateMP_Object__PARAMS__C
0086d2ac   ti_sdo_ipc_notifyDrivers_NotifyDriverShm_Object__PARAMS__C
0086d2e0   ti_sdo_ipc_heaps_HeapMemMP_Object__PARAMS__C
0086d310   ti_sysbios_family_c64p_Hwi_Object__PARAMS__C
0086d36c   ti_sdo_ipc_ListMP_Object__PARAMS__C
0086d398   ti_sdo_ipc_gates_GateHWSem_Module__FXNS__C
0086d3c4   ti_sdo_ipc_gates_GateMPSupportNull_Module__FXNS__C
0086d3f0   ti_sdo_ipc_gates_GatePeterson_Module__FXNS__C
0086d41c   ti_sdo_ipc_heaps_HeapMemMP_Module__FXNS__C
0086d444   ti_sdo_ipc_nsremote_NameServerRemoteNotify_Module__FXNS__C
0086d46c   ti_sdo_ipc_transports_TransportShm_Module__FXNS__C
0086d494   ti_sdo_ipc_transports_TransportShm_Object__PARAMS__C
0086d4bc   ti_sysbios_heaps_HeapMem_Module__FXNS__C
0086d4e4   ti_sysbios_knl_Swi_Object__PARAMS__C
0086d50c   ti_sdo_ipc_gates_GateHWSem_Object__PARAMS__C
0086d530   ti_sdo_ipc_gates_GateMPSupportNull_Object__PARAMS__C
0086d554   ti_sdo_ipc_gates_GatePeterson_Object__PARAMS__C
0086d578   ti_sysbios_gates_GateAll_Module__FXNS__C
0086d59c   ti_sysbios_gates_GateHwi_Module__FXNS__C
0086d5c0   ti_sysbios_gates_GateMutexPri_Module__FXNS__C
0086d5e4   ti_sysbios_gates_GateMutex_Module__FXNS__C
0086d608   ti_sysbios_gates_GateSwi_Module__FXNS__C
0086d62c   ti_sysbios_knl_Clock_Object__PARAMS__C
0086d650   ti_sysbios_knl_Semaphore_Object__PARAMS__C
0086d674   xdc_runtime_GateNull_Module__FXNS__C
0086d698   xdc_runtime_knl_GateThread_Module__FXNS__C
0086d6bc   ti_sdo_ipc_GateMP_E_gateUnavailable__C
0086d6c0   xdc_runtime_Startup_sfxnRts__A
0086d704   ti_sdo_ipc_GateMP_Object__DESC__C
0086d724   ti_sdo_ipc_ListMP_Object__DESC__C
0086d744   ti_sdo_ipc_Notify_Object__DESC__C
0086d764   ti_sdo_ipc_gates_GateHWSem_Object__DESC__C
0086d784   ti_sdo_ipc_gates_GateMPSupportNull_Object__DESC__C
0086d7a4   ti_sdo_ipc_gates_GatePeterson_Object__DESC__C
0086d7c4   ti_sdo_ipc_heaps_HeapMemMP_Object__DESC__C
0086d7e4   ti_sdo_ipc_notifyDrivers_NotifyDriverShm_Object__DESC__C
0086d804   ti_sdo_ipc_nsremote_NameServerRemoteNotify_Object__DESC__C
0086d824   ti_sdo_ipc_nsremote_NameServerRemoteNotify_Object__PARAMS__C
0086d844   ti_sdo_ipc_transports_TransportShm_Object__DESC__C
0086d864   ti_sdo_utils_List_Object__DESC__C
0086d884   ti_sysbios_family_c64p_Hwi_Object__DESC__C
0086d8a4   ti_sysbios_gates_GateAll_Object__DESC__C
0086d8c4   ti_sysbios_gates_GateHwi_Object__DESC__C
0086d8e4   ti_sysbios_gates_GateMutexPri_Object__DESC__C
0086d904   ti_sysbios_gates_GateMutex_Object__DESC__C
0086d924   ti_sysbios_gates_GateSwi_Object__DESC__C
0086d944   ti_sysbios_heaps_HeapMem_Object__DESC__C
0086d964   ti_sysbios_heaps_HeapMem_Object__PARAMS__C
0086d984   ti_sysbios_knl_Clock_Object__DESC__C
0086d9a4   ti_sysbios_knl_Queue_Object__DESC__C
0086d9c4   ti_sysbios_knl_Semaphore_Object__DESC__C
0086d9e4   ti_sysbios_knl_Swi_Object__DESC__C
0086da04   ti_sysbios_knl_Task_Object__DESC__C
0086da24   ti_sysbios_xdcruntime_GateThreadSupport_Object__DESC__C
0086da44   xdc_runtime_GateNull_Object__DESC__C
0086da64   xdc_runtime_knl_GateThread_Object__DESC__C
0086da84   ti_sdo_ipc_GateMP_E_localGate__C
0086daa0   ti_sdo_ipc_Notify_Object__PARAMS__C
0086dab8   ti_sdo_utils_List_Object__PARAMS__C
0086dad0   ti_sysbios_gates_GateAll_Object__PARAMS__C
0086dae8   ti_sysbios_gates_GateHwi_Object__PARAMS__C
0086db00   ti_sysbios_gates_GateMutexPri_Object__PARAMS__C
0086db18   ti_sysbios_gates_GateMutex_Object__PARAMS__C
0086db30   ti_sysbios_gates_GateSwi_Object__PARAMS__C
0086db48   ti_sysbios_knl_Queue_Object__PARAMS__C
0086db60   ti_sysbios_knl_Task_hooks__A
0086db78   ti_sysbios_xdcruntime_GateThreadSupport_Object__PARAMS__C
0086db90   xdc_runtime_GateNull_Object__PARAMS__C
0086dba8   xdc_runtime_knl_GateThread_Object__PARAMS__C
0086dbd4   ti_sdo_ipc_GateMP_LM_create__C
0086dbd8   ti_sdo_ipc_family_c647x_MultiProcSetup_procMap__A
0086dbe8   ti_sysbios_family_c64p_EventCombiner_EVTMASK__C
0086dbf8   xdc_runtime_Startup_firstFxns__A
0086dc08   ti_sysbios_family_c66_Cache_initSize__C
0086dc1c   ti_sysbios_knl_Idle_funcList__C
0086dc24   ti_sysbios_knl_Task_hooks__C
0086dc2c   xdc_runtime_Startup_firstFxns__C
0086dc34   xdc_runtime_Startup_lastFxns__C
0086dc3c   ti_sdo_ipc_GateMP_LM_delete__C
0086dc40   ti_sdo_ipc_GateMP_LM_enter__C
0086dc44   ti_sdo_ipc_GateMP_LM_leave__C
0086dc48   ti_sdo_ipc_GateMP_LM_open__C
0086dc4c   ti_sdo_ipc_GateMP_Module__diagsEnabled__C
0086dc50   ti_sdo_ipc_GateMP_Module__diagsIncluded__C
0086dc54   ti_sdo_ipc_GateMP_Module__diagsMask__C
0086dc58   ti_sdo_ipc_GateMP_Module__loggerFxn2__C
0086dc5c   ti_sdo_ipc_GateMP_Module__loggerFxn4__C
0086dc60   ti_sdo_ipc_GateMP_Module__loggerObj__C
0086dc64   ti_sdo_ipc_Ipc_A_addrNotCacheAligned__C
0086dc68   ti_sdo_ipc_Ipc_A_addrNotInSharedRegion__C
0086dc6c   ti_sdo_ipc_Ipc_A_internal__C
0086dc70   ti_sdo_ipc_Ipc_A_invArgument__C
0086dc74   ti_sdo_ipc_Ipc_A_invParam__C
0086dc78   ti_sdo_ipc_Ipc_A_nullArgument__C
0086dc7c   ti_sdo_ipc_Ipc_A_nullPointer__C
0086dc80   ti_sdo_ipc_Ipc_E_internal__C
0086dc84   ti_sdo_ipc_Ipc_E_nameFailed__C
0086dc88   ti_sdo_ipc_Ipc_E_versionMismatch__C
0086dc8c   ti_sdo_ipc_Ipc_Module__diagsEnabled__C
0086dc90   ti_sdo_ipc_Ipc_Module__diagsIncluded__C
0086dc94   ti_sdo_ipc_Ipc_Module__diagsMask__C
0086dc98   ti_sdo_ipc_Ipc_numUserFxns__C
0086dc9c   ti_sdo_ipc_Ipc_procSync__C
0086dca0   ti_sdo_ipc_Ipc_userFxns__C
0086dca4   ti_sdo_ipc_ListMP_Module__diagsEnabled__C
0086dca8   ti_sdo_ipc_ListMP_Module__diagsIncluded__C
0086dcac   ti_sdo_ipc_ListMP_Module__diagsMask__C
0086dcb0   ti_sdo_ipc_MessageQ_A_invalidMsg__C
0086dcb4   ti_sdo_ipc_MessageQ_A_invalidObj__C
0086dcb8   ti_sdo_ipc_MessageQ_A_invalidQueueId__C
0086dcbc   ti_sdo_ipc_MessageQ_A_procIdInvalid__C
0086dcc0   ti_sdo_ipc_MessageQ_A_unregisteredTransport__C
0086dcc4   ti_sdo_ipc_MessageQ_Instance_State_highList__O
0086dcc8   ti_sdo_ipc_MessageQ_Instance_State_normalList__O
0086dccc   ti_sdo_ipc_MessageQ_LM_putLocal__C
0086dcd0   ti_sdo_ipc_MessageQ_Module__diagsEnabled__C
0086dcd4   ti_sdo_ipc_MessageQ_Module__diagsIncluded__C
0086dcd8   ti_sdo_ipc_MessageQ_Module__diagsMask__C
0086dcdc   ti_sdo_ipc_MessageQ_Module__loggerFxn4__C
0086dce0   ti_sdo_ipc_MessageQ_Module__loggerObj__C
0086dce4   ti_sdo_ipc_MessageQ_Object__count__C
0086dce8   ti_sdo_ipc_MessageQ_Object__table__C
0086dcec   ti_sdo_ipc_Notify_A_alreadyRegistered__C
0086dcf0   ti_sdo_ipc_Notify_A_internal__C
0086dcf4   ti_sdo_ipc_Notify_A_invArgument__C
0086dcf8   ti_sdo_ipc_Notify_A_notRegistered__C
0086dcfc   ti_sdo_ipc_Notify_A_reservedEvent__C
0086dd00   ti_sdo_ipc_Notify_Module__diagsEnabled__C
0086dd04   ti_sdo_ipc_Notify_Module__diagsIncluded__C
0086dd08   ti_sdo_ipc_Notify_Module__diagsMask__C
0086dd0c   ti_sdo_ipc_Notify_Module__gateObj__C
0086dd10   ti_sdo_ipc_Notify_Object__heap__C
0086dd14   ti_sdo_ipc_Notify_numEvents__C
0086dd18   ti_sdo_ipc_Notify_sendEventPollCount__C
0086dd1c   ti_sdo_ipc_SharedRegion_A_addrOutOfRange__C
0086dd20   ti_sdo_ipc_SharedRegion_A_idTooLarge__C
0086dd24   ti_sdo_ipc_SharedRegion_A_noHeap__C
0086dd28   ti_sdo_ipc_SharedRegion_A_region0Invalid__C
0086dd2c   ti_sdo_ipc_SharedRegion_A_regionInvalid__C
0086dd30   ti_sdo_ipc_SharedRegion_A_reserveTooMuch__C
0086dd34   ti_sdo_ipc_SharedRegion_INVALIDSRPTR__C
0086dd38   ti_sdo_ipc_SharedRegion_Module__diagsEnabled__C
0086dd3c   ti_sdo_ipc_SharedRegion_Module__diagsIncluded__C
0086dd40   ti_sdo_ipc_SharedRegion_Module__diagsMask__C
0086dd44   ti_sdo_ipc_SharedRegion_cacheLineSize__C
0086dd48   ti_sdo_ipc_SharedRegion_numOffsetBits__C
0086dd4c   ti_sdo_ipc_SharedRegion_offsetMask__C
0086dd50   ti_sdo_ipc_family_c647x_Interrupt_INTERDSPINT__C
0086dd54   ti_sdo_ipc_family_c647x_Interrupt_IPCAR0__C
0086dd58   ti_sdo_ipc_family_c647x_Interrupt_IPCGR0__C
0086dd5c   ti_sdo_ipc_family_c647x_Interrupt_KICK0__C
0086dd60   ti_sdo_ipc_family_c647x_Interrupt_KICK1__C
0086dd64   ti_sdo_ipc_family_c647x_MultiProcSetup_A_invalidProcessor__C
0086dd68   ti_sdo_ipc_family_c647x_MultiProcSetup_Module__diagsEnabled__C
0086dd6c   ti_sdo_ipc_family_c647x_MultiProcSetup_Module__diagsIncluded__C
0086dd70   ti_sdo_ipc_family_c647x_MultiProcSetup_Module__diagsMask__C
0086dd74   ti_sdo_ipc_family_c647x_MultiProcSetup_procMap__C
0086dd78   ti_sdo_ipc_family_c647x_NotifySetup_dspIntVectId__C
0086dd7c   ti_sdo_ipc_gates_GateHWSem_A_invSemNum__C
0086dd80   ti_sdo_ipc_gates_GateHWSem_Module__diagsEnabled__C
0086dd84   ti_sdo_ipc_gates_GateHWSem_Module__diagsIncluded__C
0086dd88   ti_sdo_ipc_gates_GateHWSem_Module__diagsMask__C
0086dd8c   ti_sdo_ipc_gates_GateHWSem_baseAddr__C
0086dd90   ti_sdo_ipc_gates_GateHWSem_numSems__C
0086dd94   ti_sdo_ipc_gates_GateHWSem_reservedMaskArr__C
0086dd98   ti_sdo_ipc_gates_GateHWSem_reservedMaskArr__A
0086dd9c   ti_sdo_ipc_gates_GateMPSupportNull_A_invalidAction__C
0086dda0   ti_sdo_ipc_gates_GateMPSupportNull_Module__diagsEnabled__C
0086dda4   ti_sdo_ipc_gates_GateMPSupportNull_Module__diagsIncluded__C
0086dda8   ti_sdo_ipc_gates_GateMPSupportNull_Module__diagsMask__C
0086ddac   ti_sdo_ipc_gates_GateMPSupportNull_action__C
0086ddb0   ti_sdo_ipc_gates_GatePeterson_E_gateRemotelyOpened__C
0086ddb4   ti_sdo_ipc_gates_GatePeterson_Module__diagsEnabled__C
0086ddb8   ti_sdo_ipc_gates_GatePeterson_Module__diagsIncluded__C
0086ddbc   ti_sdo_ipc_gates_GatePeterson_Module__diagsMask__C
0086ddc0   ti_sdo_ipc_gates_GatePeterson_numInstances__C
0086ddc4   ti_sdo_ipc_heaps_HeapMemMP_A_align__C
0086ddc8   ti_sdo_ipc_heaps_HeapMemMP_A_heapSize__C
0086ddcc   ti_sdo_ipc_heaps_HeapMemMP_A_invalidFree__C
0086ddd0   ti_sdo_ipc_heaps_HeapMemMP_A_zeroBlock__C
0086ddd4   ti_sdo_ipc_heaps_HeapMemMP_E_memory__C
0086ddd8   ti_sdo_ipc_heaps_HeapMemMP_Module__diagsEnabled__C
0086dddc   ti_sdo_ipc_heaps_HeapMemMP_Module__diagsIncluded__C
0086dde0   ti_sdo_ipc_heaps_HeapMemMP_Module__diagsMask__C
0086dde4   ti_sdo_ipc_interfaces_IGateMPSupport_Interface__BASE__C
0086dde8   ti_sdo_ipc_interfaces_IMessageQTransport_Interface__BASE__C
0086ddec   ti_sdo_ipc_interfaces_INotifyDriver_Interface__BASE__C
0086ddf0   ti_sdo_ipc_notifyDrivers_NotifyDriverShm_Module__diagsEnabled__C
0086ddf4   ti_sdo_ipc_notifyDrivers_NotifyDriverShm_Module__diagsIncluded__C
0086ddf8   ti_sdo_ipc_notifyDrivers_NotifyDriverShm_Module__diagsMask__C
0086ddfc   ti_sdo_ipc_notifyDrivers_NotifyDriverShm_Object__heap__C
0086de00   ti_sdo_ipc_nsremote_NameServerRemoteNotify_A_invalidValueLen__C
0086de04   ti_sdo_ipc_nsremote_NameServerRemoteNotify_Instance_State_semMultiBlock__O
0086de08   ti_sdo_ipc_nsremote_NameServerRemoteNotify_Instance_State_semRemoteWait__O
0086de0c   ti_sdo_ipc_nsremote_NameServerRemoteNotify_Instance_State_swiObj__O
0086de10   ti_sdo_ipc_nsremote_NameServerRemoteNotify_Module__diagsEnabled__C
0086de14   ti_sdo_ipc_nsremote_NameServerRemoteNotify_Module__diagsIncluded__C
0086de18   ti_sdo_ipc_nsremote_NameServerRemoteNotify_Module__diagsMask__C
0086de1c   ti_sdo_ipc_nsremote_NameServerRemoteNotify_notifyEventId__C
0086de20   ti_sdo_ipc_nsremote_NameServerRemoteNotify_timeout__C
0086de24   ti_sdo_ipc_transports_TransportShmSetup_priority__C
0086de28   ti_sdo_ipc_transports_TransportShm_Instance_State_swiObj__O
0086de2c   ti_sdo_ipc_transports_TransportShm_Module__diagsEnabled__C
0086de30   ti_sdo_ipc_transports_TransportShm_Module__diagsIncluded__C
0086de34   ti_sdo_ipc_transports_TransportShm_Module__diagsMask__C
0086de38   ti_sdo_utils_INameServerRemote_Interface__BASE__C
0086de3c   ti_sdo_utils_List_Object__count__C
0086de40   ti_sdo_utils_List_Object__table__C
0086de44   ti_sdo_utils_MultiProc_A_invalidMultiProcId__C
0086de48   ti_sdo_utils_MultiProc_Module__diagsEnabled__C
0086de4c   ti_sdo_utils_MultiProc_Module__diagsIncluded__C
0086de50   ti_sdo_utils_MultiProc_Module__diagsMask__C
0086de54   ti_sdo_utils_NameServer_A_invArgument__C
0086de58   ti_sdo_utils_NameServer_A_invalidLen__C
0086de5c   ti_sdo_utils_NameServer_E_entryExists__C
0086de60   ti_sdo_utils_NameServer_E_maxReached__C
0086de64   ti_sdo_utils_NameServer_Instance_State_freeList__O
0086de68   ti_sdo_utils_NameServer_Instance_State_nameList__O
0086de6c   ti_sdo_utils_NameServer_Module__diagsEnabled__C
0086de70   ti_sdo_utils_NameServer_Module__diagsIncluded__C
0086de74   ti_sdo_utils_NameServer_Module__diagsMask__C
0086de78   ti_sdo_utils_NameServer_Object__count__C
0086de7c   ti_sdo_utils_NameServer_Object__table__C
0086de80   ti_sysbios_BIOS_Module__diagsEnabled__C
0086de84   ti_sysbios_BIOS_Module__diagsIncluded__C
0086de88   ti_sysbios_BIOS_Module__diagsMask__C
0086de8c   ti_sysbios_BIOS_installedErrorHook__C
0086de90   ti_sysbios_family_c62_TaskSupport_stackAlignment__C
0086de94   ti_sysbios_family_c64p_EventCombiner_E_unpluggedEvent__C
0086de98   ti_sysbios_family_c64p_Exception_E_exceptionMin__C
0086de9c   ti_sysbios_family_c64p_Exception_exceptionHook__C
0086dea0   ti_sysbios_family_c64p_Exception_externalHook__C
0086dea4   ti_sysbios_family_c64p_Exception_internalHook__C
0086dea8   ti_sysbios_family_c64p_Exception_nmiHook__C
0086deac   ti_sysbios_family_c64p_Hwi_E_alreadyDefined__C
0086deb0   ti_sysbios_family_c64p_Hwi_E_handleNotFound__C
0086deb4   ti_sysbios_family_c64p_Hwi_LD_end__C
0086deb8   ti_sysbios_family_c64p_Hwi_LM_begin__C
0086debc   ti_sysbios_family_c64p_Hwi_Module__diagsEnabled__C
0086dec0   ti_sysbios_family_c64p_Hwi_Module__diagsIncluded__C
0086dec4   ti_sysbios_family_c64p_Hwi_Module__diagsMask__C
0086dec8   ti_sysbios_family_c64p_Hwi_Module__loggerFxn1__C
0086decc   ti_sysbios_family_c64p_Hwi_Module__loggerFxn8__C
0086ded0   ti_sysbios_family_c64p_Hwi_Module__loggerObj__C
0086ded4   ti_sysbios_family_c66_Cache_atomicBlockSize__C
0086ded8   ti_sysbios_gates_GateMutexPri_A_badContext__C
0086dedc   ti_sysbios_gates_GateMutexPri_Instance_State_pendQ__O
0086dee0   ti_sysbios_gates_GateMutexPri_Module__diagsEnabled__C
0086dee4   ti_sysbios_gates_GateMutexPri_Module__diagsIncluded__C
0086dee8   ti_sysbios_gates_GateMutexPri_Module__diagsMask__C
0086deec   ti_sysbios_gates_GateMutex_A_badContext__C
0086def0   ti_sysbios_gates_GateMutex_Instance_State_sem__O
0086def4   ti_sysbios_gates_GateMutex_Module__diagsEnabled__C
0086def8   ti_sysbios_gates_GateMutex_Module__diagsIncluded__C
0086defc   ti_sysbios_gates_GateMutex_Module__diagsMask__C
0086df00   ti_sysbios_gates_GateSwi_A_badContext__C
0086df04   ti_sysbios_gates_GateSwi_Module__diagsEnabled__C
0086df08   ti_sysbios_gates_GateSwi_Module__diagsIncluded__C
0086df0c   ti_sysbios_gates_GateSwi_Module__diagsMask__C
0086df10   ti_sysbios_hal_Hwi_E_stackOverflow__C
0086df14   ti_sysbios_heaps_HeapBuf_Instance_State_freeList__O
0086df18   ti_sysbios_heaps_HeapBuf_Object__count__C
0086df1c   ti_sysbios_heaps_HeapBuf_Object__table__C
0086df20   ti_sysbios_heaps_HeapBuf_numConstructedHeaps__C
0086df24   ti_sysbios_heaps_HeapMem_A_align__C
0086df28   ti_sysbios_heaps_HeapMem_A_heapSize__C
0086df2c   ti_sysbios_heaps_HeapMem_A_invalidFree__C
0086df30   ti_sysbios_heaps_HeapMem_A_zeroBlock__C
0086df34   ti_sysbios_heaps_HeapMem_E_memory__C
0086df38   ti_sysbios_heaps_HeapMem_Module__diagsEnabled__C
0086df3c   ti_sysbios_heaps_HeapMem_Module__diagsIncluded__C
0086df40   ti_sysbios_heaps_HeapMem_Module__diagsMask__C
0086df44   ti_sysbios_heaps_HeapMem_Module__gateObj__C
0086df48   ti_sysbios_heaps_HeapMem_Object__count__C
0086df4c   ti_sysbios_heaps_HeapMem_Object__table__C
0086df50   ti_sysbios_heaps_HeapMem_reqAlignMask__C
0086df54   ti_sysbios_heaps_HeapMem_reqAlign__C
0086df58   ti_sysbios_knl_Clock_A_badThreadType__C
0086df5c   ti_sysbios_knl_Clock_LM_begin__C
0086df60   ti_sysbios_knl_Clock_LM_tick__C
0086df64   ti_sysbios_knl_Clock_LW_delayed__C
0086df68   ti_sysbios_knl_Clock_Module_State_clockQ__O
0086df6c   ti_sysbios_knl_Clock_Module__diagsEnabled__C
0086df70   ti_sysbios_knl_Clock_Module__diagsIncluded__C
0086df74   ti_sysbios_knl_Clock_Module__diagsMask__C
0086df78   ti_sysbios_knl_Clock_Module__loggerFxn1__C
0086df7c   ti_sysbios_knl_Clock_Module__loggerFxn2__C
0086df80   ti_sysbios_knl_Clock_Module__loggerObj__C
0086df84   ti_sysbios_knl_Clock_tickMode__C
0086df88   ti_sysbios_knl_Clock_tickSource__C
0086df8c   ti_sysbios_knl_Queue_Object__count__C
0086df90   ti_sysbios_knl_Idle_funcList__A
0086df94   ti_sysbios_knl_Queue_Object__table__C
0086df98   ti_sysbios_knl_Semaphore_A_badContext__C
0086df9c   ti_sysbios_knl_Semaphore_A_noEvents__C
0086dfa0   ti_sysbios_knl_Semaphore_A_overflow__C
0086dfa4   ti_sysbios_knl_Semaphore_Instance_State_pendQ__O
0086dfa8   ti_sysbios_knl_Semaphore_LM_pend__C
0086dfac   ti_sysbios_knl_Semaphore_LM_post__C
0086dfb0   ti_sysbios_knl_Semaphore_Module__diagsEnabled__C
0086dfb4   ti_sysbios_knl_Semaphore_Module__diagsIncluded__C
0086dfb8   ti_sysbios_knl_Semaphore_Module__diagsMask__C
0086dfbc   ti_sysbios_knl_Semaphore_Module__loggerFxn2__C
0086dfc0   ti_sysbios_knl_Semaphore_Module__loggerFxn4__C
0086dfc4   ti_sysbios_knl_Semaphore_Module__loggerObj__C
0086dfc8   ti_sysbios_knl_Swi_A_badPriority__C
0086dfcc   ti_sysbios_knl_Swi_LD_end__C
0086dfd0   ti_sysbios_knl_Swi_LM_begin__C
0086dfd4   ti_sysbios_knl_Swi_LM_post__C
0086dfd8   ti_sysbios_knl_Swi_Module__diagsEnabled__C
0086dfdc   ti_sysbios_knl_Swi_Module__diagsIncluded__C
0086dfe0   ti_sysbios_knl_Swi_Module__diagsMask__C
0086dfe4   ti_sysbios_knl_Swi_Module__loggerFxn1__C
0086dfe8   ti_sysbios_knl_Swi_Module__loggerFxn4__C
0086dfec   ti_sysbios_knl_Swi_Module__loggerObj__C
0086dff0   ti_sysbios_knl_Swi_Object__count__C
0086dff4   ti_sysbios_knl_Swi_Object__table__C
0086dff8   ti_sysbios_knl_Task_A_badPriority__C
0086dffc   ti_sysbios_knl_Task_A_badTaskState__C
0086e000   ti_sysbios_knl_Task_A_badThreadType__C
0086e004   ti_sysbios_knl_Task_A_noPendElem__C
0086e008   ti_sysbios_knl_Task_E_spOutOfBounds__C
0086e00c   ti_sysbios_knl_Task_E_stackOverflow__C
0086e010   ti_sysbios_knl_Task_LD_block__C
0086e014   ti_sysbios_knl_Task_LD_exit__C
0086e018   ti_sysbios_knl_Task_LD_ready__C
0086e01c   ti_sysbios_knl_Task_LM_setPri__C
0086e020   ti_sysbios_knl_Task_LM_switch__C
0086e024   ti_sysbios_knl_Task_LM_yield__C
0086e028   ti_sysbios_knl_Task_Module_State_inactiveQ__O
0086e02c   ti_sysbios_knl_Task_Module_State_terminatedQ__O
0086e030   ti_sysbios_knl_Task_Module__diagsEnabled__C
0086e034   ti_sysbios_knl_Task_Module__diagsIncluded__C
0086e038   ti_sysbios_knl_Task_Module__diagsMask__C
0086e03c   ti_sysbios_knl_Task_Module__loggerFxn2__C
0086e040   ti_sysbios_knl_Task_Module__loggerFxn4__C
0086e044   ti_sysbios_knl_Task_Module__loggerObj__C
0086e048   ti_sysbios_knl_Task_Object__count__C
0086e04c   ti_sysbios_knl_Task_Object__heap__C
0086e050   ti_sysbios_knl_Task_Object__table__C
0086e054   ti_sysbios_knl_Task_allBlockedFunc__C
0086e058   ti_sysbios_knl_Task_defaultStackHeap__C
0086e05c   ti_sysbios_knl_Task_defaultStackSize__C
0086e060   ti_sysbios_knl_Task_numConstructedTasks__C
0086e064   ti_sysbios_knl_Task_numPriorities__C
0086e068   ti_sysbios_timers_timer64_Timer_A_notAvailable__C
0086e06c   ti_sysbios_timers_timer64_Timer_E_cannotSupport__C
0086e070   ti_sysbios_timers_timer64_Timer_Module__diagsEnabled__C
0086e074   ti_sysbios_timers_timer64_Timer_Module__diagsIncluded__C
0086e078   ti_sysbios_timers_timer64_Timer_Module__diagsMask__C
0086e07c   ti_sysbios_timers_timer64_Timer_anyMask__C
0086e080   ti_sysbios_timers_timer64_Timer_freqDivisor__C
0086e084   ti_sysbios_timers_timer64_Timer_numLocalTimers__C
0086e088   ti_sysbios_timers_timer64_Timer_numTimerDevices__C
0086e08c   ti_sysbios_xdcruntime_GateThreadSupport_Instance_State_gate__O
0086e090   xdc_runtime_Assert_E_assertFailed__C
0086e094   xdc_runtime_Core_A_initializedParams__C
0086e098   xdc_runtime_Core_Module__diagsEnabled__C
0086e09c   xdc_runtime_Core_Module__diagsIncluded__C
0086e0a0   xdc_runtime_Core_Module__diagsMask__C
0086e0a4   xdc_runtime_Error_E_generic__C
0086e0a8   xdc_runtime_Error_E_memory__C
0086e0ac   xdc_runtime_Error_Module__diagsEnabled__C
0086e0b0   xdc_runtime_Error_Module__diagsIncluded__C
0086e0b4   xdc_runtime_Error_Module__diagsMask__C
0086e0b8   xdc_runtime_Error_Module__loggerFxn8__C
0086e0bc   xdc_runtime_Error_Module__loggerObj__C
0086e0c0   xdc_runtime_Error_policy__C
0086e0c4   xdc_runtime_Error_raiseHook__C
0086e0c8   xdc_runtime_IGateProvider_Interface__BASE__C
0086e0cc   xdc_runtime_IHeap_Interface__BASE__C
0086e0d0   xdc_runtime_IModule_Interface__BASE__C
0086e0d4   xdc_runtime_Log_L_error__C
0086e0d8   xdc_runtime_Memory_defaultHeapInstance__C
0086e0dc   xdc_runtime_Startup_execImpl__C
0086e0e0   xdc_runtime_Startup_lastFxns__A
0086e0e4   xdc_runtime_Startup_maxPasses__C
0086e0e8   xdc_runtime_Startup_sfxnRts__C
0086e0ec   xdc_runtime_Startup_sfxnTab__C
0086e0f0   xdc_runtime_Startup_startModsFxn__C
0086e0f4   xdc_runtime_System_Module__gateObj__C
0086e0f8   xdc_runtime_System_extendFxn__C
0086e0fc   xdc_runtime_System_maxAtexitHandlers__C
0086e100   xdc_runtime_Text_charTab__C
0086e104   xdc_runtime_Text_nameEmpty__C
0086e108   xdc_runtime_Text_nameStatic__C
0086e10c   xdc_runtime_Text_nameUnknown__C
0086e110   xdc_runtime_Text_nodeTab__C
0086e114   xdc_runtime_Text_visitRopeFxn__C
0086e118   ti_sdo_ipc_GateMP_Module__id__C
0086e11c   ti_sdo_ipc_GateMP_Module__loggerDefined__C
0086e120   ti_sdo_ipc_Ipc_Module__id__C
0086e124   ti_sdo_ipc_Ipc_generateSlaveDataForHost__C
0086e128   ti_sdo_ipc_ListMP_Module__id__C
0086e12c   ti_sdo_ipc_MessageQ_Module__id__C
0086e130   ti_sdo_ipc_MessageQ_Module__loggerDefined__C
0086e134   ti_sdo_ipc_Notify_Module__id__C
0086e138   ti_sdo_ipc_Notify_numLines__C
0086e13c   ti_sdo_ipc_Notify_reservedEvents__C
0086e140   ti_sdo_ipc_SharedRegion_Module__id__C
0086e144   ti_sdo_ipc_SharedRegion_numEntries__C
0086e148   ti_sdo_ipc_SharedRegion_translate__C
0086e14c   ti_sdo_ipc_family_c647x_Interrupt_enableKick__C
0086e150   ti_sdo_ipc_family_c647x_MultiProcSetup_Module__id__C
0086e154   ti_sdo_ipc_gates_GateHWSem_Module__id__C
0086e158   ti_sdo_ipc_gates_GateMPSupportNull_Module__id__C
0086e15c   ti_sdo_ipc_gates_GatePeterson_Module__id__C
0086e160   ti_sdo_ipc_heaps_HeapMemMP_Module__id__C
0086e164   ti_sdo_ipc_notifyDrivers_NotifyDriverShm_Module__id__C
0086e168   ti_sdo_ipc_nsremote_NameServerRemoteNotify_Module__id__C
0086e16c   ti_sdo_ipc_transports_TransportShm_Module__id__C
0086e170   ti_sdo_ipc_transports_TransportShm_notifyEventId__C
0086e174   ti_sdo_utils_MultiProc_Module__id__C
0086e178   ti_sdo_utils_MultiProc_numProcessors__C
0086e17c   ti_sdo_utils_MultiProc_numProcsInCluster__C
0086e180   ti_sdo_utils_NameServer_Module__id__C
0086e184   ti_sysbios_BIOS_Module__id__C
0086e188   ti_sysbios_family_c64p_EventCombiner_Module__id__C
0086e18c   ti_sysbios_family_c64p_Exception_Module__id__C
0086e190   ti_sysbios_family_c64p_Hwi_Module__id__C
0086e194   ti_sysbios_family_c64p_Hwi_Module__loggerDefined__C
0086e198   ti_sysbios_gates_GateMutexPri_Module__id__C
0086e19c   ti_sysbios_gates_GateMutex_Module__id__C
0086e1a0   ti_sysbios_gates_GateSwi_Module__id__C
0086e1a4   ti_sysbios_hal_Hwi_Module__id__C
0086e1a8   ti_sysbios_heaps_HeapMem_Module__id__C
0086e1ac   ti_sysbios_knl_Clock_Module__id__C
0086e1b0   ti_sysbios_knl_Clock_Module__loggerDefined__C
0086e1b4   ti_sysbios_knl_Semaphore_Module__id__C
0086e1b8   ti_sysbios_knl_Semaphore_Module__loggerDefined__C
0086e1bc   ti_sysbios_knl_Swi_Module__id__C
0086e1c0   ti_sysbios_knl_Swi_Module__loggerDefined__C
0086e1c4   ti_sysbios_knl_Task_Module__id__C
0086e1c8   ti_sysbios_knl_Task_Module__loggerDefined__C
0086e1cc   ti_sysbios_knl_Task_deleteTerminatedTasks__C
0086e1d0   ti_sysbios_knl_Task_initStackFlag__C
0086e1d4   ti_sysbios_timers_timer64_Timer_Module__id__C
0086e1d8   ti_sysbios_timers_timer64_Timer_startupNeeded__C
0086e1dc   xdc_runtime_Core_Module__id__C
0086e1e0   xdc_runtime_Error_Module__loggerDefined__C
0086e1e4   xdc_runtime_Error_maxDepth__C
0086e1e8   xdc_runtime_Memory_Module__id__C
0086e1ec   xdc_runtime_Text_charCnt__C
0086e1f0   xdc_runtime_Text_isLoaded__C
0086e1f4   xdc_runtime_Text_registryModsLastId__C
0086e1f8   xdc_runtime_Text_unnamedModsLastId__C
0086e200   ti_sdo_ipc_GateMP_Module_State_0_remoteCustom1Gates__A
0086ea00   ti_sdo_ipc_GateMP_Module__root__V
0086ea08   ti_sdo_ipc_GateMP_Module__state__V
0086ea50   ti_sdo_ipc_Ipc_Module__state__V
0086ea5c   ti_sdo_ipc_ListMP_Module__root__V
0086ea64   ti_sdo_ipc_ListMP_Module__state__V
0086ea68   ti_sdo_ipc_MessageQ_Module__root__V
0086ea70   ti_sdo_ipc_MessageQ_Module__state__V
0086ea8c   ti_sdo_ipc_Notify_Module__root__V
0086ea94   ti_sdo_ipc_Notify_Module__state__V
0086ea9c   ti_sdo_ipc_SharedRegion_Module__state__V
0086eaa0   ti_sdo_ipc_family_c647x_Interrupt_Module__state__V
0086eaa8   ti_sdo_ipc_gates_GateHWSem_Module__root__V
0086eab0   ti_sdo_ipc_gates_GateMPSupportNull_Module__root__V
0086eab8   ti_sdo_ipc_gates_GatePeterson_Module__root__V
0086eac0   ti_sdo_ipc_heaps_HeapMemMP_Module__root__V
0086eac8   ti_sdo_ipc_heaps_HeapMemMP_Module__state__V
0086eacc   ti_sdo_ipc_notifyDrivers_NotifyDriverShm_Module__root__V
0086ead4   ti_sdo_ipc_nsremote_NameServerRemoteNotify_Module__root__V
0086eadc   ti_sdo_ipc_transports_TransportShm_Module__root__V
0086eae4   ti_sdo_ipc_transports_TransportShmSetup_Module__state__V
0086eae8   ti_sdo_utils_List_Module__root__V
0086eaf0   ti_sdo_utils_MultiProc_Module__state__V
0086eaf4   ti_sdo_utils_NameServer_Module__root__V
0086eafc   ti_sdo_utils_NameServer_Module__state__V
0086eb04   ti_sdo_utils_NameServerRemoteNull_Module__root__V
0086eb0c   ti_sysbios_BIOS_Module__state__V
0086eb28   ti_sysbios_family_c64p_EventCombiner_Module__state__V
0086ef28   ti_sysbios_family_c64p_Exception_Module__state__V
0086ef54   ti_sysbios_family_c64p_Hwi_Module__root__V
0086ef5c   ti_sysbios_family_c64p_Hwi_Module__state__V
0086efc4   ti_sysbios_gates_GateAll_Module__root__V
0086efcc   ti_sysbios_gates_GateHwi_Module__root__V
0086efd4   ti_sysbios_gates_GateMutex_Module__root__V
0086efdc   ti_sysbios_gates_GateMutexPri_Module__root__V
0086efe4   ti_sysbios_gates_GateSwi_Module__root__V
0086efec   ti_sysbios_hal_Hwi_Module__root__V
0086eff4   ti_sysbios_hal_Timer_Module__root__V
0086effc   ti_sysbios_heaps_HeapBuf_Module__root__V
0086f004   ti_sysbios_heaps_HeapBuf_Module__state__V
0086f008   ti_sysbios_heaps_HeapMem_Module__root__V
0086f010   ti_sysbios_knl_Clock_Module__root__V
0086f018   ti_sysbios_knl_Clock_Module__state__V
0086f044   ti_sysbios_knl_Queue_Module__root__V
0086f04c   ti_sysbios_knl_Semaphore_Module__root__V
0086f054   ti_sysbios_knl_Swi_Module__root__V
0086f05c   ti_sysbios_knl_Swi_Module__state__V
0086f078   ti_sysbios_knl_Task_Module__root__V
0086f080   ti_sysbios_knl_Task_Module__state__V
0086f0b4   ti_sysbios_syncs_SyncSem_Module__root__V
0086f0bc   ti_sysbios_timers_timer64_Timer_Module__root__V
0086f0c4   ti_sysbios_timers_timer64_Timer_Module__state__V
0086f0d8   ti_sysbios_xdcruntime_GateThreadSupport_Module__root__V
0086f0e0   xdc_runtime_Error_Module__state__V
0086f0e4   xdc_runtime_GateNull_Module__root__V
0086f0ec   xdc_runtime_Memory_Module__state__V
0086f0f0   xdc_runtime_Registry_Module__state__V
0086f0f8   xdc_runtime_Startup_Module__state__V
0086f100   xdc_runtime_System_Module__state__V
0086f10c   xdc_runtime_Text_Module__state__V
0086f114   xdc_runtime_knl_GateThread_Module__root__V
0086f11c   __xdc__init__addr
0086f120   _ftable
0086f300   ti_sysbios_timers_timer64_Timer_Module_State_0_device__A
0086f480   qmssGblCfgParams
0086f5a0   ti_sdo_utils_NameServer_Object__table__V
0086f720   ti_sdo_ipc_Ipc_Module_State_0_procEntry__A
0086f7c0   ti_sdo_ipc_SharedRegion_Module_State_0_regions__A
0086f850   ti_sdo_ipc_GateMP_Module_State_0_remoteSystemGates__A
0086f8d0   ti_sysbios_knl_Swi_Module_State_0_readyQ__A
0086f950   ti_sysbios_knl_Task_Module_State_0_readyQ__A
0086f9d0   ti_sysbios_timers_timer64_Timer_Module_State_0_gctrl__A
0086fa50   ti_sysbios_timers_timer64_Timer_Module_State_0_handles__A
0086fad0   ti_sysbios_timers_timer64_Timer_Module_State_0_intFreqs__A
0086fbc8   cppiGblCfgParams
0086fc40   ti_sysbios_family_c64p_Hwi_Object__table__V
0086fcb8   ti_sysbios_timers_timer64_Timer_Object__table__V
0086fd04   _ft_end
0086fd08   TSK_idle
0086fd08   ti_sysbios_knl_Task_Object__table__V
0086fe10   ti_sdo_ipc_MessageQ_Module_State_0_transports__A
0086fe50   ti_sdo_ipc_family_c647x_Interrupt_Module_State_0_fxnTable__A
0086fe90   ti_sysbios_gates_GateMutex_Object__table__V
0086fed0   ti_sysbios_knl_Swi_Object__table__V
0086ff20   Qmss_highEoiVector
0086ff40   ti_sdo_ipc_MessageQ_Module_State_0_heaps__A
0086ff60   ti_sdo_ipc_Notify_Module_State_0_notifyHandles__A
0086ff80   ti_sdo_ipc_transports_TransportShmSetup_Module_State_0_handles__A
0086ffa0   xdc_runtime_System_Module_State_0_atexitHandlers__A
0086ffc0   ti_sysbios_gates_GateMutexPri_Object__table__V
0086ffd8   ti_sysbios_heaps_HeapMem_Object__table__V
0086fff0   Qmss_lowEoiVector
00870000   ti_sysbios_gates_GateAll_Object__table__V
00870010   _cleanup_ptr
00870014   _dtors_ptr
00870018   __TI_enable_exit_profile_output
0087001c   cppiLObj
00870020   ti_sysbios_gates_GateSwi_Object__table__V
00870030   ti_sysbios_hal_Hwi_Object__table__V
00870038   ti_sysbios_hal_Timer_Object__table__V
00870040   ti_sdo_ipc_GateMP_Module_State_0_remoteCustom2Gates__A
00870048   ti_sdo_ipc_Notify_Module_State_0_notifyHandles_0__A
00870050   ti_sdo_ipc_Notify_Module_State_0_notifyHandles_1__A
00870058   ti_sdo_ipc_Notify_Module_State_0_notifyHandles_2__A
00870060   ti_sdo_ipc_Notify_Module_State_0_notifyHandles_3__A
00870068   ti_sdo_ipc_Notify_Module_State_0_notifyHandles_4__A
00870070   ti_sdo_ipc_Notify_Module_State_0_notifyHandles_5__A
00870078   ti_sdo_ipc_Notify_Module_State_0_notifyHandles_6__A
00870080   ti_sdo_ipc_Notify_Module_State_0_notifyHandles_7__A
00870088   ti_sysbios_gates_GateHwi_Object__table__V
00870090   xdc_runtime_GateNull_Object__table__V
00870098   Qmss_cdmaEoiVector
008700a0   _stack
008710a0   __CIOBUF_
008710a0   __TI_STACK_END
008711c0   __TI_STATIC_BASE
008711c0   hSrioDriver
008711c4   isAllocated
008711c8   srioSocket
008711cc   txData_int
008711d0   txData_char
008711d4   idx
008711d8   num_bytes
008711dc   ptr_rxDataPayload
008711e0   sendToCore
008711e4   hDrvBuffer
008711e8   allocatedLen
008711ec   messageSource
008711f0   coreLoop
008711f4   randomValue
008711f8   firstSendStart
008711fc   iterationCounter
00871200   xx
00871204   myStatus
00871208   recvFromCore
0087120c   x_min
00871210   x1
00871214   Ipc_sr0MemorySetup
00871218   coreNum
0087121c   runFlag
00871220   pp1
00871224   bufferCounter
00871228   gDataBufferMemMgrMaxSize
0087122c   malloc_counter
00871230   free_counter
00871234   messageValue
00871238   processingCounter
0087123c   lastOne
00871240   qmssLObjIsValid
00871244   DEVICE_ID1_16BIT
00871248   DEVICE_ID1_8BIT
0087124c   DEVICE_ID2_16BIT
00871250   DEVICE_ID2_8BIT
00871254   DEVICE_ID3_16BIT
00871258   DEVICE_ID3_8BIT
0087125c   DEVICE_ID4_16BIT
00871260   DEVICE_ID4_8BIT
00871264   DEVICE_ID5_16BIT
00871268   DEVICE_ID5_8BIT
0087126c   DEVICE_ID6_16BIT
00871270   DEVICE_ID6_8BIT
00871274   DEVICE_ID7_16BIT
00871278   DEVICE_ID7_8BIT
0087127c   DEVICE_ID8_16BIT
00871280   DEVICE_ID8_8BIT
00871400   ti_sysbios_family_c64p_Hwi0
00871420   ti_sysbios_family_c64p_Hwi1
00871440   ti_sysbios_family_c64p_Hwi2
00871460   ti_sysbios_family_c64p_Hwi3
00871480   ti_sysbios_family_c64p_Hwi4
008714a0   ti_sysbios_family_c64p_Hwi5
008714c0   ti_sysbios_family_c64p_Hwi6
008714e0   ti_sysbios_family_c64p_Hwi7
00871500   ti_sysbios_family_c64p_Hwi8
00871520   ti_sysbios_family_c64p_Hwi9
00871540   ti_sysbios_family_c64p_Hwi10
00871560   ti_sysbios_family_c64p_Hwi11
00871580   ti_sysbios_family_c64p_Hwi12
008715a0   ti_sysbios_family_c64p_Hwi13
008715c0   ti_sysbios_family_c64p_Hwi14
008715e0   ti_sysbios_family_c64p_Hwi15
0087249c   __TI_Handler_Table_Base
008724a8   __TI_Handler_Table_Limit
008724ec   __TI_CINIT_Base
0087254c   __TI_CINIT_Limit
0c000000   queueFree
0c002000   qmssGObj
0c002400   gSRIODriverMCB
0c002500   isSRIOInitialized
0c002580   isSRIOSocketsCreated
0c002600   cppiObject
80000000   x_ref_float
80001000   z_short
80005000   y_short
80007000   x_short
80009000   fftBuffer
80011000   twiddle_32
80011080   twiddle_64
80011180   twiddle_128
80011380   twiddle_256
80011780   twiddle_512
80011f80   twiddle_1024
ffffffff   __TI_pprof_out_hndl
ffffffff   __TI_prof_data_size
ffffffff   __TI_prof_data_start
ffffffff   __binit__
ffffffff   __c_args__
ffffffff   binit
UNDEFED    __TI_INITARRAY_Base
UNDEFED    __TI_INITARRAY_Limit

[1491 symbols]
